 Align

 Timestamp is 57c8d156 (Fri Sep  2 04:09:42 2016)

 Preferred load address is 10000000

 Start         Length     Name                   Class
 0001:00000000 00000004H .00cfg                  CODE
 0001:00000004 00000004H .CRT$XCA                CODE
 0001:00000008 00000004H .CRT$XCZ                CODE
 0001:0000000c 00000004H .CRT$XIA                CODE
 0001:00000010 0000000cH .CRT$XIC                CODE
 0001:0000001c 00000004H .CRT$XIZ                CODE
 0001:00000020 00000004H .CRT$XPA                CODE
 0001:00000024 00000008H .CRT$XPX                CODE
 0001:0000002c 00000004H .CRT$XPXA               CODE
 0001:00000030 00000004H .CRT$XPZ                CODE
 0001:00000034 00000004H .CRT$XTA                CODE
 0001:00000038 00000008H .CRT$XTZ                CODE
 0001:00000040 00004bdcH .rdata                  CODE
 0001:00004c1c 00000134H .rdata$r                CODE
 0001:00004d50 0000000cH .rdata$sxdata           CODE
 0001:00004d5c 000002b0H .rdata$zzzdbg           CODE
 0001:0000500c 00000004H .rtc$IAA                CODE
 0001:00005010 00000004H .rtc$IZZ                CODE
 0001:00005014 00000004H .rtc$TAA                CODE
 0001:00005018 00000008H .rtc$TZZ                CODE
 0001:00005020 0000c4c8H .text$mn                CODE
 0001:000114e8 00000428H .xdata$x                CODE
 0001:00011910 0000008eH .edata                  CODE
 0002:00000000 00000770H .data                   DATA
 0002:00000770 00000078H .data$r                 DATA
 0002:000007e8 00000bbcH .bss                    DATA
 0003:00000000 000000f8H .idata$5                DATA
 0003:000000f8 00000014H .idata$2                DATA
 0003:0000010c 00000014H .idata$3                DATA
 0003:00000120 000000f8H .idata$4                DATA
 0003:00000218 00000466H .idata$6                DATA
 0004:00000000 0000008cH .gfids$x                DATA
 0004:0000008c 00000044H .gfids$y                DATA
 0005:00000000 00000060H .rsrc$01                DATA
 0005:00000060 00000360H .rsrc$02                DATA

  Address         Publics by Value              Rva+Base       Lib:Object

 0000:00000000       ___guard_fids_count        00000000     <absolute>
 0000:00000000       ___guard_longjmp_count     00000000     <absolute>
 0000:00000000       ___guard_longjmp_table     00000000     <absolute>
 0000:00000000       __except_list              00000000     <absolute>
 0000:00000000       ___guard_iat_table         00000000     <absolute>
 0000:00000000       ___guard_iat_count         00000000     <absolute>
 0000:00000000       ___guard_fids_table        00000000     <absolute>
 0000:00000000       ___dynamic_value_reloc_table 00000000     <absolute>
 0000:00000003       ___safe_se_handler_count   00000003     <absolute>
 0000:00000100       ___guard_flags             00000100     <absolute>
 0000:00000000       ___ImageBase               10000000     <linker-defined>
 0001:00000000       ___guard_check_icall_fptr  10001000     LIBCMT:guard_support.obj
 0001:00000004       ___xc_a                    10001004     LIBCMT:initializers.obj
 0001:00000008       ___xc_z                    10001008     LIBCMT:initializers.obj
 0001:0000000c       ___xi_a                    1000100c     LIBCMT:initializers.obj
 0001:00000010       ___acrt_multibyte_initializer 10001010     libucrt:multibyte_initializer.obj
 0001:00000014       ___acrt_stdio_initializer  10001014     libucrt:stdio_initializer.obj
 0001:00000018       ___acrt_tran_sse2_initializer 10001018     libucrt:sse2_initializer.obj
 0001:0000001c       ___xi_z                    1000101c     LIBCMT:initializers.obj
 0001:00000020       ___xp_a                    10001020     LIBCMT:initializers.obj
 0001:00000024       ___acrt_locale_terminator  10001024     libucrt:locale_initializer.obj
 0001:00000028       ___dcrt_console_output_terminator 10001028     libucrt:console_output_initializer.obj
 0001:0000002c       ___acrt_stdio_terminator   1000102c     libucrt:stdio_initializer.obj
 0001:00000030       ___xp_z                    10001030     LIBCMT:initializers.obj
 0001:00000034       ___xt_a                    10001034     LIBCMT:initializers.obj
 0001:00000038       ___xt_z                    10001038     LIBCMT:initializers.obj
 0001:00000040       _MainGuid                  10001040     Align.obj
 0001:00000050       _MenuGuid                  10001050     Align.obj
 0001:00000060       _DialogGuid                10001060     Align.obj
 0001:00000070       ??_7?$DialogItemBinding@UFarDialogItem@@@@6B@ 10001070     Align.obj
 0001:00000078       ??_7PluginCheckBoxBinding@@6B@ 10001078     Align.obj
 0001:00000080       ??_7PluginRadioButtonBinding@@6B@ 10001080     Align.obj
 0001:00000088       ??_7PluginIntEditFieldBinding@@6B@ 10001088     Align.obj
 0001:00000090       ??_C@_15EFLNJKHH@?$AA?$CF?$AAu?$AA?$AA@ 10001090     Align.obj
 0001:00000098       ??_7PluginUIntEditFieldBinding@@6B@ 10001098     Align.obj
 0001:000000a0       ??_7?$DialogBuilderBase@UFarDialogItem@@@@6B@ 100010a0     Align.obj
 0001:000000c4       ??_7PluginDialogBuilder@@6B@ 100010c4     Align.obj
 0001:000000e8       ??_C@_11LOCGONAA@?$AA?$AA@ 100010e8     Align.obj
 0001:000000ec       ??_C@_1M@OFJLCCLD@?$AAA?$AAl?$AAi?$AAg?$AAn?$AA?$AA@ 100010ec     Align.obj
 0001:000000f8       ??_C@_1DI@GCKLIMEF@?$AAA?$AAl?$AAi?$AAg?$AAn?$AA?5?$AAb?$AAl?$AAo?$AAc?$AAk?$AA?5?$AAf?$AAo?$AAr?$AA?5?$AAF?$AAa?$AAr?$AA?5?$AAM?$AAa?$AAn?$AAa?$AAg?$AAe?$AAr?$AA?$AA@ 100010f8     Align.obj
 0001:00000130       ??_C@_1DE@BGKMIKPD@?$AAE?$AAu?$AAg?$AAe?$AAn?$AAe?$AA?5?$AAR?$AAo?$AAs?$AAh?$AAa?$AAl?$AA?5?$AA?$CG?$AA?5?$AAF?$AAa?$AAr?$AA?5?$AAG?$AAr?$AAo?$AAu?$AAp?$AA?$AA@ 10001130     Align.obj
 0001:00000164       ??_C@_1BI@JMKBMFLI@?$AAR?$AAi?$AAg?$AAh?$AAt?$AAM?$AAa?$AAr?$AAg?$AAi?$AAn?$AA?$AA@ 10001164     Align.obj
 0001:0000017c       ??_C@_1BC@PKHIBLMF@?$AAR?$AAe?$AAf?$AAo?$AAr?$AAm?$AAa?$AAt?$AA?$AA@ 1000117c     Align.obj
 0001:00000190       ??_C@_1BE@NIKLIADP@?$AAS?$AAm?$AAa?$AAr?$AAt?$AAM?$AAo?$AAd?$AAe?$AA?$AA@ 10001190     Align.obj
 0001:000001a4       ??_C@_1BA@MANOLHD@?$AAJ?$AAu?$AAs?$AAt?$AAi?$AAf?$AAy?$AA?$AA@ 100011a4     Align.obj
 0001:000001c0       __imp__EncodePointer@4     100011c0     vc_crt_fix.obj
 0001:000001c4       __imp__DecodePointer@4     100011c4     vc_crt_fix.obj
 0001:000001c8       __imp__GetModuleHandleExW@12 100011c8     vc_crt_fix.obj
 0001:000001cc       __imp__InitializeSListHead@4 100011cc     vc_crt_fix.obj
 0001:000001d0       __imp__InterlockedFlushSList@4 100011d0     vc_crt_fix.obj
 0001:000001d4       __imp__InterlockedPopEntrySList@4 100011d4     vc_crt_fix.obj
 0001:000001d8       __imp__InterlockedPushEntrySList@8 100011d8     vc_crt_fix.obj
 0001:000001dc       __imp__InterlockedPushListSListEx@16 100011dc     vc_crt_fix.obj
 0001:000001e0       __imp__RtlFirstEntrySList@4 100011e0     vc_crt_fix.obj
 0001:000001e4       __imp__QueryDepthSList@4   100011e4     vc_crt_fix.obj
 0001:000001fc       ??_C@_0O@NLDKAIKN@EncodePointer?$AA@ 100011fc     vc_crt_fix_impl.obj
 0001:0000020c       ??_C@_0O@KBPMFGHI@DecodePointer?$AA@ 1000120c     vc_crt_fix_impl.obj
 0001:0000021c       ??_C@_0BD@GIGEJCNH@GetModuleHandleExW?$AA@ 1000121c     vc_crt_fix_impl.obj
 0001:00000230       ??_C@_0BE@NBEJPEJA@InitializeSListHead?$AA@ 10001230     vc_crt_fix_impl.obj
 0001:00000244       ??_C@_0BG@PLLPFLHB@InterlockedFlushSList?$AA@ 10001244     vc_crt_fix_impl.obj
 0001:0000025c       ??_C@_0BJ@PNEEKDOK@InterlockedPopEntrySList?$AA@ 1000125c     vc_crt_fix_impl.obj
 0001:00000278       ??_C@_0BK@JFGGAIOA@InterlockedPushEntrySList?$AA@ 10001278     vc_crt_fix_impl.obj
 0001:00000294       ??_C@_0BL@FOECAEGO@InterlockedPushListSListEx?$AA@ 10001294     vc_crt_fix_impl.obj
 0001:000002b0       ??_C@_0BD@FHMMIGCI@RtlFirstEntrySList?$AA@ 100012b0     vc_crt_fix_impl.obj
 0001:000002c4       ??_C@_0BA@FGPHPMJB@QueryDepthSList?$AA@ 100012c4     vc_crt_fix_impl.obj
 0001:000002d4       __pDefaultRawDllMain       100012d4     LIBCMT:dll_dllmain.obj
 0001:000002d4       __pRawDllMain              100012d4     LIBCMT:dll_dllmain.obj
 0001:000002dc       ??_7exception@std@@6B@     100012dc     LIBCMT:throw_bad_alloc.obj
 0001:000002e4       ??_C@_0BC@EOODALEL@Unknown?5exception?$AA@ 100012e4     LIBCMT:throw_bad_alloc.obj
 0001:000002fc       ??_7bad_alloc@std@@6B@     100012fc     LIBCMT:throw_bad_alloc.obj
 0001:00000304       ??_C@_0P@GHFPNOJB@bad?5allocation?$AA@ 10001304     LIBCMT:throw_bad_alloc.obj
 0001:00000318       ??_7bad_array_new_length@std@@6B@ 10001318     LIBCMT:throw_bad_alloc.obj
 0001:00000320       ??_C@_0BF@KINCDENJ@bad?5array?5new?5length?$AA@ 10001320     LIBCMT:throw_bad_alloc.obj
 0001:0000033c       ??_7type_info@@6B@         1000133c     LIBCMT:std_type_info_static.obj
 0001:00000378       ??_C@_1BC@DNHGCMLG@?$AAa?$AAd?$AAv?$AAa?$AAp?$AAi?$AA3?$AA2?$AA?$AA@ 10001378     libvcruntime:winapi_downlevel.obj
 0001:0000038c       ??_C@_1DM@KHCHBNEB@?$AAa?$AAp?$AAi?$AA?9?$AAm?$AAs?$AA?9?$AAw?$AAi?$AAn?$AA?9?$AAc?$AAo?$AAr?$AAe?$AA?9?$AAf?$AAi?$AAb?$AAe?$AAr?$AAs?$AA?9?$AAl?$AA1?$AA?9?$AA1?$AA?9?$AA1?$AA?$AA@ 1000138c     libvcruntime:winapi_downlevel.obj
 0001:000003c8       ??_C@_1DK@LPPGFMPP@?$AAa?$AAp?$AAi?$AA?9?$AAm?$AAs?$AA?9?$AAw?$AAi?$AAn?$AA?9?$AAc?$AAo?$AAr?$AAe?$AA?9?$AAs?$AAy?$AAn?$AAc?$AAh?$AA?9?$AAl?$AA1?$AA?9?$AA2?$AA?9?$AA0?$AA?$AA@ 100013c8     libvcruntime:winapi_downlevel.obj
 0001:00000404       ??_C@_1BC@GDMECMAK@?$AAk?$AAe?$AAr?$AAn?$AAe?$AAl?$AA3?$AA2?$AA?$AA@ 10001404     libvcruntime:winapi_downlevel.obj
 0001:00000420       ??_C@_08KNHFBNJ@FlsAlloc?$AA@ 10001420     libvcruntime:winapi_downlevel.obj
 0001:00000434       ??_C@_07PEJMOBNF@FlsFree?$AA@ 10001434     libvcruntime:winapi_downlevel.obj
 0001:00000444       ??_C@_0M@GDNOONDI@FlsGetValue?$AA@ 10001444     libvcruntime:winapi_downlevel.obj
 0001:00000458       ??_C@_0M@JCPCPOEF@FlsSetValue?$AA@ 10001458     libvcruntime:winapi_downlevel.obj
 0001:0000046c       ??_C@_0BM@HCFOFFN@InitializeCriticalSectionEx?$AA@ 1000146c     libvcruntime:winapi_downlevel.obj
 0001:00000618       ??_C@_08EHJDFFNH@__based?$CI?$AA@ 10001618     libvcruntime:undname.obj
 0001:00000624       ??_C@_07KOLFKCDI@__cdecl?$AA@ 10001624     libvcruntime:undname.obj
 0001:0000062c       ??_C@_08GHMPAG@__pascal?$AA@ 1000162c     libvcruntime:undname.obj
 0001:00000638       ??_C@_09IFJBGAPI@__stdcall?$AA@ 10001638     libvcruntime:undname.obj
 0001:00000644       ??_C@_0L@NPHFGOKO@__thiscall?$AA@ 10001644     libvcruntime:undname.obj
 0001:00000650       ??_C@_0L@JMKHOMEK@__fastcall?$AA@ 10001650     libvcruntime:undname.obj
 0001:0000065c       ??_C@_0N@BCKKPABJ@__vectorcall?$AA@ 1000165c     libvcruntime:undname.obj
 0001:0000066c       ??_C@_09HIJEGCPM@__clrcall?$AA@ 1000166c     libvcruntime:undname.obj
 0001:00000678       ??_C@_06GHPCKEAG@__eabi?$AA@ 10001678     libvcruntime:undname.obj
 0001:00000680       ??_C@_07JOMMBBKO@__ptr64?$AA@ 10001680     libvcruntime:undname.obj
 0001:00000688       ??_C@_0L@PILCLIHE@__restrict?$AA@ 10001688     libvcruntime:undname.obj
 0001:00000694       ??_C@_0M@GFIIJFMG@__unaligned?$AA@ 10001694     libvcruntime:undname.obj
 0001:000006a0       ??_C@_09DHDLOLLB@restrict?$CI?$AA@ 100016a0     libvcruntime:undname.obj
 0001:000006aa       ??_C@_00CNPNBAHC@?$AA@     100016aa     libvcruntime:undname.obj
 0001:000006ac       ??_C@_04NIHEBCM@?5new?$AA@ 100016ac     libvcruntime:undname.obj
 0001:000006b4       ??_C@_07FPCDHGMM@?5delete?$AA@ 100016b4     libvcruntime:undname.obj
 0001:000006bc       ??_C@_01NEMOKFLO@?$DN?$AA@ 100016bc     libvcruntime:undname.obj
 0001:000006c0       ??_C@_02GPIOPFAK@?$DO?$DO?$AA@ 100016c0     libvcruntime:undname.obj
 0001:000006c4       ??_C@_02FODMEDOG@?$DM?$DM?$AA@ 100016c4     libvcruntime:undname.obj
 0001:000006c8       ??_C@_01DCLJPIOD@?$CB?$AA@ 100016c8     libvcruntime:undname.obj
 0001:000006cc       ??_C@_02EGOFBIJA@?$DN?$DN?$AA@ 100016cc     libvcruntime:undname.obj
 0001:000006d0       ??_C@_02FDNJECIE@?$CB?$DN?$AA@ 100016d0     libvcruntime:undname.obj
 0001:000006d4       ??_C@_02GPECMEKF@?$FL?$FN?$AA@ 100016d4     libvcruntime:undname.obj
 0001:000006d8       ??_C@_08LHJFAFGD@operator?$AA@ 100016d8     libvcruntime:undname.obj
 0001:000006e4       ??_C@_02HBOOOICD@?9?$DO?$AA@ 100016e4     libvcruntime:undname.obj
 0001:000006e8       ??_C@_01NBENCBCI@?$CK?$AA@ 100016e8     libvcruntime:undname.obj
 0001:000006ec       ??_C@_02ECNGHCIF@?$CL?$CL?$AA@ 100016ec     libvcruntime:undname.obj
 0001:000006f0       ??_C@_02BAABKJLB@?9?9?$AA@ 100016f0     libvcruntime:undname.obj
 0001:000006f4       ??_C@_01JOAMLHOP@?9?$AA@   100016f4     libvcruntime:undname.obj
 0001:000006f8       ??_C@_01MIFGBAGJ@?$CL?$AA@ 100016f8     libvcruntime:undname.obj
 0001:000006fc       ??_C@_01HNPIGOCE@?$CG?$AA@ 100016fc     libvcruntime:undname.obj
 0001:00000700       ??_C@_03MNHNFDLC@?9?$DO?$CK?$AA@ 10001700     libvcruntime:undname.obj
 0001:00000704       ??_C@_01KMDKNFGN@?1?$AA@   10001704     libvcruntime:undname.obj
 0001:00000708       ??_C@_01FGNFDNOH@?$CF?$AA@ 10001708     libvcruntime:undname.obj
 0001:0000070c       ??_C@_01MNNFJEPP@?$DM?$AA@ 1000170c     libvcruntime:undname.obj
 0001:00000710       ??_C@_02EHCHHCKH@?$DM?$DN?$AA@ 10001710     libvcruntime:undname.obj
 0001:00000714       ??_C@_01PPODPGHN@?$DO?$AA@ 10001714     libvcruntime:undname.obj
 0001:00000718       ??_C@_02EEKDKGMJ@?$DO?$DN?$AA@ 10001718     libvcruntime:undname.obj
 0001:0000071c       ??_C@_01IHBHIGKO@?0?$AA@   1000171c     libvcruntime:undname.obj
 0001:00000720       ??_C@_02HCKGKOFO@?$CI?$CJ?$AA@ 10001720     libvcruntime:undname.obj
 0001:00000724       ??_C@_01PJKLJHI@?$HO?$AA@  10001724     libvcruntime:undname.obj
 0001:00000728       ??_C@_01JKBOJNNK@?$FO?$AA@ 10001728     libvcruntime:undname.obj
 0001:0000072c       ??_C@_01DNKMNLPK@?$HM?$AA@ 1000172c     libvcruntime:undname.obj
 0001:00000730       ??_C@_02PPKAJPJL@?$CG?$CG?$AA@ 10001730     libvcruntime:undname.obj
 0001:00000734       ??_C@_02NONPIBCD@?$HM?$HM?$AA@ 10001734     libvcruntime:undname.obj
 0001:00000738       ??_C@_02FPIMKNGF@?$CK?$DN?$AA@ 10001738     libvcruntime:undname.obj
 0001:0000073c       ??_C@_02FOEOMHFC@?$CL?$DN?$AA@ 1000173c     libvcruntime:undname.obj
 0001:00000740       ??_C@_02FKMDLLOA@?9?$DN?$AA@ 10001740     libvcruntime:undname.obj
 0001:00000744       ??_C@_02FJEHGPIO@?1?$DN?$AA@ 10001744     libvcruntime:undname.obj
 0001:00000748       ??_C@_02FENAOKFI@?$CF?$DN?$AA@ 10001748     libvcruntime:undname.obj
 0001:0000074c       ??_C@_03IKFCCPFF@?$DO?$DO?$DN?$AA@ 1000174c     libvcruntime:undname.obj
 0001:00000750       ??_C@_03CDNPDDLA@?$DM?$DM?$DN?$AA@ 10001750     libvcruntime:undname.obj
 0001:00000754       ??_C@_02FGJGFEAB@?$CG?$DN?$AA@ 10001754     libvcruntime:undname.obj
 0001:00000758       ??_C@_02DHLNPPGH@?$HM?$DN?$AA@ 10001758     libvcruntime:undname.obj
 0001:0000075c       ??_C@_02MHEGNOJ@?$FO?$DN?$AA@ 1000175c     libvcruntime:undname.obj
 0001:00000760       ??_C@_09IFPLHPGF@?$GAvftable?8?$AA@ 10001760     libvcruntime:undname.obj
 0001:0000076c       ??_C@_09BLBHBJP@?$GAvbtable?8?$AA@ 1000176c     libvcruntime:undname.obj
 0001:00000778       ??_C@_07FEEIOKP@?$GAvcall?8?$AA@ 10001778     libvcruntime:undname.obj
 0001:00000780       ??_C@_08LLFFHHDJ@?$GAtypeof?8?$AA@ 10001780     libvcruntime:undname.obj
 0001:0000078c       ??_C@_0BF@KDPPACIK@?$GAlocal?5static?5guard?8?$AA@ 1000178c     libvcruntime:undname.obj
 0001:000007a4       ??_C@_08OBABFOLI@?$GAstring?8?$AA@ 100017a4     libvcruntime:undname.obj
 0001:000007b0       ??_C@_0BD@JDLKDPAB@?$GAvbase?5destructor?8?$AA@ 100017b0     libvcruntime:undname.obj
 0001:000007c4       ??_C@_0BN@DEGPLNFK@?$GAvector?5deleting?5destructor?8?$AA@ 100017c4     libvcruntime:undname.obj
 0001:000007e4       ??_C@_0BO@OBMKPJIG@?$GAdefault?5constructor?5closure?8?$AA@ 100017e4     libvcruntime:undname.obj
 0001:00000804       ??_C@_0BN@IMDCHIKM@?$GAscalar?5deleting?5destructor?8?$AA@ 10001804     libvcruntime:undname.obj
 0001:00000824       ??_C@_0BO@PFGOCPJJ@?$GAvector?5constructor?5iterator?8?$AA@ 10001824     libvcruntime:undname.obj
 0001:00000844       ??_C@_0BN@LFPFMEDL@?$GAvector?5destructor?5iterator?8?$AA@ 10001844     libvcruntime:undname.obj
 0001:00000864       ??_C@_0CE@IKBNEHA@?$GAvector?5vbase?5constructor?5iterat@ 10001864     libvcruntime:undname.obj
 0001:00000888       ??_C@_0BL@NILFHHPC@?$GAvirtual?5displacement?5map?8?$AA@ 10001888     libvcruntime:undname.obj
 0001:000008a4       ??_C@_0CB@JONCMFFK@?$GAeh?5vector?5constructor?5iterator?8@ 100018a4     libvcruntime:undname.obj
 0001:000008c8       ??_C@_0CA@GCEOPDGL@?$GAeh?5vector?5destructor?5iterator?8?$AA@ 100018c8     libvcruntime:undname.obj
 0001:000008e8       ??_C@_0CH@OOJPLCPH@?$GAeh?5vector?5vbase?5constructor?5ite@ 100018e8     libvcruntime:undname.obj
 0001:00000910       ??_C@_0BL@LLKPOHJI@?$GAcopy?5constructor?5closure?8?$AA@ 10001910     libvcruntime:undname.obj
 0001:0000092c       ??_C@_0BA@KBCDOMBN@?$GAudt?5returning?8?$AA@ 1000192c     libvcruntime:undname.obj
 0001:0000093c       ??_C@_03KLGMFNMG@?$GAEH?$AA@ 1000193c     libvcruntime:undname.obj
 0001:00000940       ??_C@_05KHLCHHI@?$GARTTI?$AA@ 10001940     libvcruntime:undname.obj
 0001:00000948       ??_C@_0BA@KKLDJDLB@?$GAlocal?5vftable?8?$AA@ 10001948     libvcruntime:undname.obj
 0001:00000958       ??_C@_0CE@IIHCMGGL@?$GAlocal?5vftable?5constructor?5closu@ 10001958     libvcruntime:undname.obj
 0001:0000097c       ??_C@_06FHBGPFGH@?5new?$FL?$FN?$AA@ 1000197c     libvcruntime:undname.obj
 0001:00000984       ??_C@_09LBNFPBCA@?5delete?$FL?$FN?$AA@ 10001984     libvcruntime:undname.obj
 0001:00000990       ??_C@_0P@HJKNJFNN@?$GAomni?5callsig?8?$AA@ 10001990     libvcruntime:undname.obj
 0001:000009a0       ??_C@_0BL@CNOONJFP@?$GAplacement?5delete?5closure?8?$AA@ 100019a0     libvcruntime:undname.obj
 0001:000009bc       ??_C@_0BN@CKNJLHMB@?$GAplacement?5delete?$FL?$FN?5closure?8?$AA@ 100019bc     libvcruntime:undname.obj
 0001:000009dc       ??_C@_0CG@CFDHKGGD@?$GAmanaged?5vector?5constructor?5iter@ 100019dc     libvcruntime:undname.obj
 0001:00000a04       ??_C@_0CF@IMGKMJNO@?$GAmanaged?5vector?5destructor?5itera@ 10001a04     libvcruntime:undname.obj
 0001:00000a2c       ??_C@_0CG@HLDDJMAG@?$GAeh?5vector?5copy?5constructor?5iter@ 10001a2c     libvcruntime:undname.obj
 0001:00000a54       ??_C@_0CM@FCBBDIGB@?$GAeh?5vector?5vbase?5copy?5constructo@ 10001a54     libvcruntime:undname.obj
 0001:00000a80       ??_C@_0BL@CLIPGLGB@?$GAdynamic?5initializer?5for?5?8?$AA@ 10001a80     libvcruntime:undname.obj
 0001:00000a9c       ??_C@_0CB@PDBIFEP@?$GAdynamic?5atexit?5destructor?5for?5?8@ 10001a9c     libvcruntime:undname.obj
 0001:00000ac0       ??_C@_0CD@CGAJBKEJ@?$GAvector?5copy?5constructor?5iterato@ 10001ac0     libvcruntime:undname.obj
 0001:00000ae4       ??_C@_0CJ@GJELGAMM@?$GAvector?5vbase?5copy?5constructor?5i@ 10001ae4     libvcruntime:undname.obj
 0001:00000b10       ??_C@_0CL@FGIJHLCE@?$GAmanaged?5vector?5copy?5constructor@ 10001b10     libvcruntime:undname.obj
 0001:00000b3c       ??_C@_0BM@PMGGMLDN@?$GAlocal?5static?5thread?5guard?8?$AA@ 10001b3c     libvcruntime:undname.obj
 0001:00000b58       ??_C@_0N@BDNMDMOL@operator?5?$CC?$CC?5?$AA@ 10001b58     libvcruntime:undname.obj
 0001:00000b68       ??_C@_0BC@DAFEJGAK@?5Type?5Descriptor?8?$AA@ 10001b68     libvcruntime:undname.obj
 0001:00000b7c       ??_C@_0BM@LDKODKLH@?5Base?5Class?5Descriptor?5at?5?$CI?$AA@ 10001b7c     libvcruntime:undname.obj
 0001:00000b98       ??_C@_0BD@LGICGFMM@?5Base?5Class?5Array?8?$AA@ 10001b98     libvcruntime:undname.obj
 0001:00000bac       ??_C@_0BN@MECKDCOJ@?5Class?5Hierarchy?5Descriptor?8?$AA@ 10001bac     libvcruntime:undname.obj
 0001:00000bcc       ??_C@_0BK@CFCOFLF@?5Complete?5Object?5Locator?8?$AA@ 10001bcc     libvcruntime:undname.obj
 0001:00000be8       ___acrt_exception_action_table 10001be8     libucrt:exception_filter.obj
 0001:00000c78       ___acrt_signal_action_table_count 10001c78     libucrt:exception_filter.obj
 0001:00000c7c       ___acrt_signal_action_first_fpe_index 10001c7c     libucrt:exception_filter.obj
 0001:00000c80       ___acrt_signal_action_fpe_count 10001c80     libucrt:exception_filter.obj
 0001:00000c84       ??_C@_1BI@BGOHAHKC@?$AAm?$AAs?$AAc?$AAo?$AAr?$AAe?$AAe?$AA?4?$AAd?$AAl?$AAl?$AA?$AA@ 10001c84     libucrt:exit.obj
 0001:00000c9c       ??_C@_0P@MIGLKIOC@CorExitProcess?$AA@ 10001c9c     libucrt:exit.obj
 0001:00000d78       ??_C@_1EG@CNNIPFIM@?$AAa?$AAp?$AAi?$AA?9?$AAm?$AAs?$AA?9?$AAw?$AAi?$AAn?$AA?9?$AAa?$AAp?$AAp?$AAm?$AAo?$AAd?$AAe?$AAl?$AA?9?$AAr?$AAu?$AAn?$AAt?$AAi?$AAm?$AAe?$AA?9?$AAl?$AA1?$AA?9?$AA1@ 10001d78     libucrt:winapi_thunks.obj
 0001:00000dc0       ??_C@_1EA@JGEFHKEI@?$AAa?$AAp?$AAi?$AA?9?$AAm?$AAs?$AA?9?$AAw?$AAi?$AAn?$AA?9?$AAc?$AAo?$AAr?$AAe?$AA?9?$AAd?$AAa?$AAt?$AAe?$AAt?$AAi?$AAm?$AAe?$AA?9?$AAl?$AA1?$AA?9?$AA1?$AA?9?$AA1?$AA?$AA@ 10001dc0     libucrt:winapi_thunks.obj
 0001:00000e00       ??_C@_1DI@GCIAAENM@?$AAa?$AAp?$AAi?$AA?9?$AAm?$AAs?$AA?9?$AAw?$AAi?$AAn?$AA?9?$AAc?$AAo?$AAr?$AAe?$AA?9?$AAf?$AAi?$AAl?$AAe?$AA?9?$AAl?$AA2?$AA?9?$AA1?$AA?9?$AA1?$AA?$AA@ 10001e00     libucrt:winapi_thunks.obj
 0001:00000e38       ??_C@_1EI@MPIAOHOC@?$AAa?$AAp?$AAi?$AA?9?$AAm?$AAs?$AA?9?$AAw?$AAi?$AAn?$AA?9?$AAc?$AAo?$AAr?$AAe?$AA?9?$AAl?$AAo?$AAc?$AAa?$AAl?$AAi?$AAz?$AAa?$AAt?$AAi?$AAo?$AAn?$AA?9?$AAl?$AA1?$AA?9@ 10001e38     libucrt:winapi_thunks.obj
 0001:00000e80       ??_C@_1FK@FPHCKFIE@?$AAa?$AAp?$AAi?$AA?9?$AAm?$AAs?$AA?9?$AAw?$AAi?$AAn?$AA?9?$AAc?$AAo?$AAr?$AAe?$AA?9?$AAl?$AAo?$AAc?$AAa?$AAl?$AAi?$AAz?$AAa?$AAt?$AAi?$AAo?$AAn?$AA?9?$AAo?$AAb?$AAs@ 10001e80     libucrt:winapi_thunks.obj
 0001:00000ee0       ??_C@_1EM@DILCGIIO@?$AAa?$AAp?$AAi?$AA?9?$AAm?$AAs?$AA?9?$AAw?$AAi?$AAn?$AA?9?$AAc?$AAo?$AAr?$AAe?$AA?9?$AAp?$AAr?$AAo?$AAc?$AAe?$AAs?$AAs?$AAt?$AAh?$AAr?$AAe?$AAa?$AAd?$AAs?$AA?9?$AAl@ 10001ee0     libucrt:winapi_thunks.obj
 0001:00000f2c       ??_C@_1DM@LNCGDDPN@?$AAa?$AAp?$AAi?$AA?9?$AAm?$AAs?$AA?9?$AAw?$AAi?$AAn?$AA?9?$AAc?$AAo?$AAr?$AAe?$AA?9?$AAs?$AAt?$AAr?$AAi?$AAn?$AAg?$AA?9?$AAl?$AA1?$AA?9?$AA1?$AA?9?$AA0?$AA?$AA@ 10001f2c     libucrt:winapi_thunks.obj
 0001:00000f68       ??_C@_1DO@FPAPJEMD@?$AAa?$AAp?$AAi?$AA?9?$AAm?$AAs?$AA?9?$AAw?$AAi?$AAn?$AA?9?$AAc?$AAo?$AAr?$AAe?$AA?9?$AAs?$AAy?$AAs?$AAi?$AAn?$AAf?$AAo?$AA?9?$AAl?$AA1?$AA?9?$AA2?$AA?9?$AA1?$AA?$AA@ 10001f68     libucrt:winapi_thunks.obj
 0001:00000fa8       ??_C@_1DK@NDHNAHIO@?$AAa?$AAp?$AAi?$AA?9?$AAm?$AAs?$AA?9?$AAw?$AAi?$AAn?$AA?9?$AAc?$AAo?$AAr?$AAe?$AA?9?$AAw?$AAi?$AAn?$AAr?$AAt?$AA?9?$AAl?$AA1?$AA?9?$AA1?$AA?9?$AA0?$AA?$AA@ 10001fa8     libucrt:winapi_thunks.obj
 0001:00000fe4       ??_C@_1DM@KGHDGBCM@?$AAa?$AAp?$AAi?$AA?9?$AAm?$AAs?$AA?9?$AAw?$AAi?$AAn?$AA?9?$AAc?$AAo?$AAr?$AAe?$AA?9?$AAx?$AAs?$AAt?$AAa?$AAt?$AAe?$AA?9?$AAl?$AA2?$AA?9?$AA1?$AA?9?$AA0?$AA?$AA@ 10001fe4     libucrt:winapi_thunks.obj
 0001:00001020       ??_C@_1EO@IJIOEFOH@?$AAa?$AAp?$AAi?$AA?9?$AAm?$AAs?$AA?9?$AAw?$AAi?$AAn?$AA?9?$AAr?$AAt?$AAc?$AAo?$AAr?$AAe?$AA?9?$AAn?$AAt?$AAu?$AAs?$AAe?$AAr?$AA?9?$AAw?$AAi?$AAn?$AAd?$AAo?$AAw?$AA?9@ 10002020     libucrt:winapi_thunks.obj
 0001:00001070       ??_C@_1FG@HHGEKANL@?$AAa?$AAp?$AAi?$AA?9?$AAm?$AAs?$AA?9?$AAw?$AAi?$AAn?$AA?9?$AAs?$AAe?$AAc?$AAu?$AAr?$AAi?$AAt?$AAy?$AA?9?$AAs?$AAy?$AAs?$AAt?$AAe?$AAm?$AAf?$AAu?$AAn?$AAc?$AAt?$AAi@ 10002070     libucrt:winapi_thunks.obj
 0001:000010c8       ??_C@_1FG@NCKKOLKO@?$AAe?$AAx?$AAt?$AA?9?$AAm?$AAs?$AA?9?$AAw?$AAi?$AAn?$AA?9?$AAk?$AAe?$AAr?$AAn?$AAe?$AAl?$AA3?$AA2?$AA?9?$AAp?$AAa?$AAc?$AAk?$AAa?$AAg?$AAe?$AA?9?$AAc?$AAu?$AAr?$AAr@ 100020c8     libucrt:winapi_thunks.obj
 0001:00001120       ??_C@_1EG@DBIOJECG@?$AAe?$AAx?$AAt?$AA?9?$AAm?$AAs?$AA?9?$AAw?$AAi?$AAn?$AA?9?$AAn?$AAt?$AAu?$AAs?$AAe?$AAr?$AA?9?$AAd?$AAi?$AAa?$AAl?$AAo?$AAg?$AAb?$AAo?$AAx?$AA?9?$AAl?$AA1?$AA?9?$AA1@ 10002120     libucrt:winapi_thunks.obj
 0001:00001168       ??_C@_1EO@FIHMJCLF@?$AAe?$AAx?$AAt?$AA?9?$AAm?$AAs?$AA?9?$AAw?$AAi?$AAn?$AA?9?$AAn?$AAt?$AAu?$AAs?$AAe?$AAr?$AA?9?$AAw?$AAi?$AAn?$AAd?$AAo?$AAw?$AAs?$AAt?$AAa?$AAt?$AAi?$AAo?$AAn?$AA?9@ 10002168     libucrt:winapi_thunks.obj
 0001:000011b8       ??_C@_1O@BCCLBEOE@?$AAu?$AAs?$AAe?$AAr?$AA3?$AA2?$AA?$AA@ 100021b8     libucrt:winapi_thunks.obj
 0001:000011f0       ??_C@_0BE@JOGNEJCI@GetCurrentPackageId?$AA@ 100021f0     libucrt:winapi_thunks.obj
 0001:00001214       ??_C@_0O@KKBNKAPF@LCMapStringEx?$AA@ 10002214     libucrt:winapi_thunks.obj
 0001:0000122c       ??_C@_0BB@HBDEELFH@LocaleNameToLCID?$AA@ 1000222c     libucrt:winapi_thunks.obj
 0001:000013b8       ??_C@_1M@HPNHIDJI@?$AAj?$AAa?$AA?9?$AAJ?$AAP?$AA?$AA@ 100023b8     libucrt:mbctype.obj
 0001:000013c4       ??_C@_1M@BIBDDEMK@?$AAz?$AAh?$AA?9?$AAC?$AAN?$AA?$AA@ 100023c4     libucrt:mbctype.obj
 0001:000013d0       ??_C@_1M@JLOOOEGK@?$AAk?$AAo?$AA?9?$AAK?$AAR?$AA?$AA@ 100023d0     libucrt:mbctype.obj
 0001:000013dc       ??_C@_1M@CLNBBOPM@?$AAz?$AAh?$AA?9?$AAT?$AAW?$AA?$AA@ 100023dc     libucrt:mbctype.obj
 0001:000013e8       ??_C@_03KOEHGMDN@Sun?$AA@  100023e8     libucrt:nlsdata.obj
 0001:000013ec       ??_C@_03PDAGKDH@Mon?$AA@   100023ec     libucrt:nlsdata.obj
 0001:000013f0       ??_C@_03NAGEINEP@Tue?$AA@  100023f0     libucrt:nlsdata.obj
 0001:000013f4       ??_C@_03MHOMLAJA@Wed?$AA@  100023f4     libucrt:nlsdata.obj
 0001:000013f8       ??_C@_03IOFIKPDN@Thu?$AA@  100023f8     libucrt:nlsdata.obj
 0001:000013fc       ??_C@_03IDIOELNC@Fri?$AA@  100023fc     libucrt:nlsdata.obj
 0001:00001400       ??_C@_03FEFJNEK@Sat?$AA@   10002400     libucrt:nlsdata.obj
 0001:00001404       ??_C@_06OOPIFAJ@Sunday?$AA@ 10002404     libucrt:nlsdata.obj
 0001:0000140c       ??_C@_06JLEDEDGH@Monday?$AA@ 1000240c     libucrt:nlsdata.obj
 0001:00001414       ??_C@_07BAAGCFCM@Tuesday?$AA@ 10002414     libucrt:nlsdata.obj
 0001:0000141c       ??_C@_09DLIGFAKA@Wednesday?$AA@ 1000241c     libucrt:nlsdata.obj
 0001:00001428       ??_C@_08HACCIKIA@Thursday?$AA@ 10002428     libucrt:nlsdata.obj
 0001:00001434       ??_C@_06JECMNKMI@Friday?$AA@ 10002434     libucrt:nlsdata.obj
 0001:0000143c       ??_C@_08INBOOONO@Saturday?$AA@ 1000243c     libucrt:nlsdata.obj
 0001:00001448       ??_C@_03JIHJHPIE@Jan?$AA@  10002448     libucrt:nlsdata.obj
 0001:0000144c       ??_C@_03HJBDCHOM@Feb?$AA@  1000244c     libucrt:nlsdata.obj
 0001:00001450       ??_C@_03ODNJBKGA@Mar?$AA@  10002450     libucrt:nlsdata.obj
 0001:00001454       ??_C@_03LEOLGMJP@Apr?$AA@  10002454     libucrt:nlsdata.obj
 0001:00001458       ??_C@_03CNMDKL@May?$AA@    10002458     libucrt:nlsdata.obj
 0001:0000145c       ??_C@_03IDFGHECI@Jun?$AA@  1000245c     libucrt:nlsdata.obj
 0001:00001460       ??_C@_03LBGABGKK@Jul?$AA@  10002460     libucrt:nlsdata.obj
 0001:00001464       ??_C@_03IFJFEIGA@Aug?$AA@  10002464     libucrt:nlsdata.obj
 0001:00001468       ??_C@_03GGCAPAJC@Sep?$AA@  10002468     libucrt:nlsdata.obj
 0001:0000146c       ??_C@_03BMAOKBAD@Oct?$AA@  1000246c     libucrt:nlsdata.obj
 0001:00001470       ??_C@_03JPJOFNIA@Nov?$AA@  10002470     libucrt:nlsdata.obj
 0001:00001474       ??_C@_03MKABNOCG@Dec?$AA@  10002474     libucrt:nlsdata.obj
 0001:00001478       ??_C@_07CGJPFGJA@January?$AA@ 10002478     libucrt:nlsdata.obj
 0001:00001480       ??_C@_08GNJGEPFN@February?$AA@ 10002480     libucrt:nlsdata.obj
 0001:0000148c       ??_C@_05HPCKOFNC@March?$AA@ 1000248c     libucrt:nlsdata.obj
 0001:00001494       ??_C@_05DMJDNLEJ@April?$AA@ 10002494     libucrt:nlsdata.obj
 0001:0000149c       ??_C@_04CNLMGBGM@June?$AA@ 1000249c     libucrt:nlsdata.obj
 0001:000014a4       ??_C@_04MIEPOIFP@July?$AA@ 100024a4     libucrt:nlsdata.obj
 0001:000014ac       ??_C@_06LBBHFDDG@August?$AA@ 100024ac     libucrt:nlsdata.obj
 0001:000014b4       ??_C@_09BHHEALKD@September?$AA@ 100024b4     libucrt:nlsdata.obj
 0001:000014c0       ??_C@_07JJNFCEND@October?$AA@ 100024c0     libucrt:nlsdata.obj
 0001:000014c8       ??_C@_08HCHEGEOA@November?$AA@ 100024c8     libucrt:nlsdata.obj
 0001:000014d4       ??_C@_08EDHMEBNP@December?$AA@ 100024d4     libucrt:nlsdata.obj
 0001:000014e0       ??_C@_02DEDBPAFC@AM?$AA@   100024e0     libucrt:nlsdata.obj
 0001:000014e4       ??_C@_02CJNFDJBF@PM?$AA@   100024e4     libucrt:nlsdata.obj
 0001:000014e8       ??_C@_08BPBNCDIB@MM?1dd?1yy?$AA@ 100024e8     libucrt:nlsdata.obj
 0001:000014f4       ??_C@_0BE@CKGJFCPC@dddd?0?5MMMM?5dd?0?5yyyy?$AA@ 100024f4     libucrt:nlsdata.obj
 0001:00001508       ??_C@_08JCCMCCIL@HH?3mm?3ss?$AA@ 10002508     libucrt:nlsdata.obj
 0001:00001514       ??_C@_17MBGCMIPB@?$AAS?$AAu?$AAn?$AA?$AA@ 10002514     libucrt:nlsdata.obj
 0001:0000151c       ??_C@_17KBOMKBF@?$AAM?$AAo?$AAn?$AA?$AA@ 1000251c     libucrt:nlsdata.obj
 0001:00001524       ??_C@_17BMKGEGOJ@?$AAT?$AAu?$AAe?$AA?$AA@ 10002524     libucrt:nlsdata.obj
 0001:0000152c       ??_C@_17CJEDCEPE@?$AAW?$AAe?$AAd?$AA?$AA@ 1000252c     libucrt:nlsdata.obj
 0001:00001534       ??_C@_17PDPHAADD@?$AAT?$AAh?$AAu?$AA?$AA@ 10002534     libucrt:nlsdata.obj
 0001:0000153c       ??_C@_17HFOLPPLP@?$AAF?$AAr?$AAi?$AA?$AA@ 1000253c     libucrt:nlsdata.obj
 0001:00001544       ??_C@_17GGIBDPIH@?$AAS?$AAa?$AAt?$AA?$AA@ 10002544     libucrt:nlsdata.obj
 0001:0000154c       ??_C@_1O@IHNHDHPB@?$AAS?$AAu?$AAn?$AAd?$AAa?$AAy?$AA?$AA@ 1000254c     libucrt:nlsdata.obj
 0001:0000155c       ??_C@_1O@MMNBFLIA@?$AAM?$AAo?$AAn?$AAd?$AAa?$AAy?$AA?$AA@ 1000255c     libucrt:nlsdata.obj
 0001:0000156c       ??_C@_1BA@ENFBFFEK@?$AAT?$AAu?$AAe?$AAs?$AAd?$AAa?$AAy?$AA?$AA@ 1000256c     libucrt:nlsdata.obj
 0001:0000157c       ??_C@_1BE@EBOGMDOH@?$AAW?$AAe?$AAd?$AAn?$AAe?$AAs?$AAd?$AAa?$AAy?$AA?$AA@ 1000257c     libucrt:nlsdata.obj
 0001:00001590       ??_C@_1BC@HHMNLIHE@?$AAT?$AAh?$AAu?$AAr?$AAs?$AAd?$AAa?$AAy?$AA?$AA@ 10002590     libucrt:nlsdata.obj
 0001:000015a4       ??_C@_1O@PDICJHAG@?$AAF?$AAr?$AAi?$AAd?$AAa?$AAy?$AA?$AA@ 100025a4     libucrt:nlsdata.obj
 0001:000015b4       ??_C@_1BC@ENMNNPAJ@?$AAS?$AAa?$AAt?$AAu?$AAr?$AAd?$AAa?$AAy?$AA?$AA@ 100025b4     libucrt:nlsdata.obj
 0001:000015c8       ??_C@_17DKNBKCHM@?$AAJ?$AAa?$AAn?$AA?$AA@ 100025c8     libucrt:nlsdata.obj
 0001:000015d0       ??_C@_17LMDJEKJN@?$AAF?$AAe?$AAb?$AA?$AA@ 100025d0     libucrt:nlsdata.obj
 0001:000015d8       ??_C@_17CKNLEDEC@?$AAM?$AAa?$AAr?$AA?$AA@ 100025d8     libucrt:nlsdata.obj
 0001:000015e0       ??_C@_17LFPOIHDD@?$AAA?$AAp?$AAr?$AA?$AA@ 100025e0     libucrt:nlsdata.obj
 0001:000015e8       ??_C@_17PNNKMEED@?$AAM?$AAa?$AAy?$AA?$AA@ 100025e8     libucrt:nlsdata.obj
 0001:000015f0       ??_C@_17KCJGOCPB@?$AAJ?$AAu?$AAn?$AA?$AA@ 100025f0     libucrt:nlsdata.obj
 0001:000015f8       ??_C@_17IJPCKHK@?$AAJ?$AAu?$AAl?$AA?$AA@ 100025f8     libucrt:nlsdata.obj
 0001:00001600       ??_C@_17ICPELBCN@?$AAA?$AAu?$AAg?$AA?$AA@ 10002600     libucrt:nlsdata.obj
 0001:00001608       ??_C@_17HCHCOKMG@?$AAS?$AAe?$AAp?$AA?$AA@ 10002608     libucrt:nlsdata.obj
 0001:00001610       ??_C@_17FNLKOI@?$AAO?$AAc?$AAt?$AA?$AA@ 10002610     libucrt:nlsdata.obj
 0001:00001618       ??_C@_17BBDMLCIG@?$AAN?$AAo?$AAv?$AA?$AA@ 10002618     libucrt:nlsdata.obj
 0001:00001620       ??_C@_17EGKACKIF@?$AAD?$AAe?$AAc?$AA?$AA@ 10002620     libucrt:nlsdata.obj
 0001:00001628       ??_C@_1BA@EFMEIEBA@?$AAJ?$AAa?$AAn?$AAu?$AAa?$AAr?$AAy?$AA?$AA@ 10002628     libucrt:nlsdata.obj
 0001:00001638       ??_C@_1BC@JGDDFFAM@?$AAF?$AAe?$AAb?$AAr?$AAu?$AAa?$AAr?$AAy?$AA?$AA@ 10002638     libucrt:nlsdata.obj
 0001:0000164c       ??_C@_1M@IKEENEDF@?$AAM?$AAa?$AAr?$AAc?$AAh?$AA?$AA@ 1000264c     libucrt:nlsdata.obj
 0001:00001658       ??_C@_1M@GJNLMHFD@?$AAA?$AAp?$AAr?$AAi?$AAl?$AA?$AA@ 10002658     libucrt:nlsdata.obj
 0001:00001664       ??_C@_19EPFLPGAP@?$AAJ?$AAu?$AAn?$AAe?$AA?$AA@ 10002664     libucrt:nlsdata.obj
 0001:00001670       ??_C@_19BIFMLPCD@?$AAJ?$AAu?$AAl?$AAy?$AA?$AA@ 10002670     libucrt:nlsdata.obj
 0001:0000167c       ??_C@_1O@PAHLKOAC@?$AAA?$AAu?$AAg?$AAu?$AAs?$AAt?$AA?$AA@ 1000267c     libucrt:nlsdata.obj
 0001:0000168c       ??_C@_1BE@DKAAMBJL@?$AAS?$AAe?$AAp?$AAt?$AAe?$AAm?$AAb?$AAe?$AAr?$AA?$AA@ 1000268c     libucrt:nlsdata.obj
 0001:000016a0       ??_C@_1BA@EPANDLNG@?$AAO?$AAc?$AAt?$AAo?$AAb?$AAe?$AAr?$AA?$AA@ 100026a0     libucrt:nlsdata.obj
 0001:000016b0       ??_C@_1BC@BGLIFPF@?$AAN?$AAo?$AAv?$AAe?$AAm?$AAb?$AAe?$AAr?$AA?$AA@ 100026b0     libucrt:nlsdata.obj
 0001:000016c4       ??_C@_1BC@FEMKIFH@?$AAD?$AAe?$AAc?$AAe?$AAm?$AAb?$AAe?$AAr?$AA?$AA@ 100026c4     libucrt:nlsdata.obj
 0001:000016d8       ??_C@_15ODEHAHHF@?$AAA?$AAM?$AA?$AA@ 100026d8     libucrt:nlsdata.obj
 0001:000016e0       ??_C@_15CLMNNGEL@?$AAP?$AAM?$AA?$AA@ 100026e0     libucrt:nlsdata.obj
 0001:000016e8       ??_C@_1BC@IEBCMHCM@?$AAM?$AAM?$AA?1?$AAd?$AAd?$AA?1?$AAy?$AAy?$AA?$AA@ 100026e8     libucrt:nlsdata.obj
 0001:000016fc       ??_C@_1CI@KNAKOEBC@?$AAd?$AAd?$AAd?$AAd?$AA?0?$AA?5?$AAM?$AAM?$AAM?$AAM?$AA?5?$AAd?$AAd?$AA?0?$AA?5?$AAy?$AAy?$AAy?$AAy?$AA?$AA@ 100026fc     libucrt:nlsdata.obj
 0001:00001724       ??_C@_1BC@GDGBMEMK@?$AAH?$AAH?$AA?3?$AAm?$AAm?$AA?3?$AAs?$AAs?$AA?$AA@ 10002724     libucrt:nlsdata.obj
 0001:00001738       ??_C@_1M@BMHNFIME@?$AAe?$AAn?$AA?9?$AAU?$AAS?$AA?$AA@ 10002738     libucrt:nlsdata.obj
 0001:00001748       ___lc_time_c               10002748     libucrt:nlsdata.obj
 0001:000018b0       ___newctype                100028b0     libucrt:ctype.obj
 0001:00001bb0       ___newclmap                10002bb0     libucrt:ctype.obj
 0001:00001d30       ___newcumap                10002d30     libucrt:ctype.obj
 0001:000025d0       ??_C@_15EMKDOKLE@?$AAa?$AAr?$AA?$AA@ 100035d0     libucrt:lcidtoname_downlevel.obj
 0001:000025d8       ??_C@_15KNPADPLH@?$AAb?$AAg?$AA?$AA@ 100035d8     libucrt:lcidtoname_downlevel.obj
 0001:000025e0       ??_C@_15EDMHLDMO@?$AAc?$AAa?$AA?$AA@ 100035e0     libucrt:lcidtoname_downlevel.obj
 0001:000025e8       ??_C@_1O@BPEAJADD@?$AAz?$AAh?$AA?9?$AAC?$AAH?$AAS?$AA?$AA@ 100035e8     libucrt:lcidtoname_downlevel.obj
 0001:000025f8       ??_C@_15LJNHCMNK@?$AAc?$AAs?$AA?$AA@ 100035f8     libucrt:lcidtoname_downlevel.obj
 0001:00002600       ??_C@_15FOMCIDHG@?$AAd?$AAa?$AA?$AA@ 10003600     libucrt:lcidtoname_downlevel.obj
 0001:00002608       ??_C@_15NBKABECB@?$AAd?$AAe?$AA?$AA@ 10003608     libucrt:lcidtoname_downlevel.obj
 0001:00002610       ??_C@_15GHPEIIAO@?$AAe?$AAl?$AA?$AA@ 10003610     libucrt:lcidtoname_downlevel.obj
 0001:00002618       ??_C@_15MNPNEAIF@?$AAe?$AAn?$AA?$AA@ 10003618     libucrt:lcidtoname_downlevel.obj
 0001:00002620       ??_C@_15GPIOMPMH@?$AAe?$AAs?$AA?$AA@ 10003620     libucrt:lcidtoname_downlevel.obj
 0001:00002628       ??_C@_15NGLOAKJC@?$AAf?$AAi?$AA?$AA@ 10003628     libucrt:lcidtoname_downlevel.obj
 0001:00002630       ??_C@_15FBKGNKAM@?$AAf?$AAr?$AA?$AA@ 10003630     libucrt:lcidtoname_downlevel.obj
 0001:00002638       ??_C@_15KGGCNEFK@?$AAh?$AAe?$AA?$AA@ 10003638     libucrt:lcidtoname_downlevel.obj
 0001:00002640       ??_C@_15PGHLIDMF@?$AAh?$AAu?$AA?$AA@ 10003640     libucrt:lcidtoname_downlevel.obj
 0001:00002648       ??_C@_15BIEMAPLM@?$AAi?$AAs?$AA?$AA@ 10003648     libucrt:lcidtoname_downlevel.obj
 0001:00002650       ??_C@_15IFJLDHAF@?$AAi?$AAt?$AA?$AA@ 10003650     libucrt:lcidtoname_downlevel.obj
 0001:00002658       ??_C@_15GEMIOCAG@?$AAj?$AAa?$AA?$AA@ 10003658     libucrt:lcidtoname_downlevel.obj
 0001:00002660       ??_C@_15EPELEGJA@?$AAk?$AAo?$AA?$AA@ 10003660     libucrt:lcidtoname_downlevel.obj
 0001:00002668       ??_C@_15NDDHIMN@?$AAn?$AAl?$AA?$AA@ 10003668     libucrt:lcidtoname_downlevel.obj
 0001:00002670       ??_C@_15BPIGNHCD@?$AAn?$AAo?$AA?$AA@ 10003670     libucrt:lcidtoname_downlevel.obj
 0001:00002678       ??_C@_15DEOPBLCG@?$AAp?$AAl?$AA?$AA@ 10003678     libucrt:lcidtoname_downlevel.obj
 0001:00002680       ??_C@_15KBECGEFG@?$AAp?$AAt?$AA?$AA@ 10003680     libucrt:lcidtoname_downlevel.obj
 0001:00002688       ??_C@_15GLJCBFMD@?$AAr?$AAo?$AA?$AA@ 10003688     libucrt:lcidtoname_downlevel.obj
 0001:00002690       ??_C@_15FEDGKCDI@?$AAr?$AAu?$AA?$AA@ 10003690     libucrt:lcidtoname_downlevel.obj
 0001:00002698       ??_C@_15GLKMLLHM@?$AAh?$AAr?$AA?$AA@ 10003698     libucrt:lcidtoname_downlevel.obj
 0001:000026a0       ??_C@_15CPKMFBDB@?$AAs?$AAk?$AA?$AA@ 100036a0     libucrt:lcidtoname_downlevel.obj
 0001:000026a8       ??_C@_15BAAIOGMK@?$AAs?$AAq?$AA?$AA@ 100036a8     libucrt:lcidtoname_downlevel.obj
 0001:000026b0       ??_C@_15INNPNOHD@?$AAs?$AAv?$AA?$AA@ 100036b0     libucrt:lcidtoname_downlevel.obj
 0001:000026b8       ??_C@_15CABMMOGH@?$AAt?$AAh?$AA?$AA@ 100036b8     libucrt:lcidtoname_downlevel.obj
 0001:000026c0       ??_C@_15BPLIHJJM@?$AAt?$AAr?$AA?$AA@ 100036c0     libucrt:lcidtoname_downlevel.obj
 0001:000026c8       ??_C@_15NEOEKKDJ@?$AAu?$AAr?$AA?$AA@ 100036c8     libucrt:lcidtoname_downlevel.obj
 0001:000026d0       ??_C@_15NFICGAJK@?$AAi?$AAd?$AA?$AA@ 100036d0     libucrt:lcidtoname_downlevel.obj
 0001:000026d8       ??_C@_15PJPFLCCM@?$AAu?$AAk?$AA?$AA@ 100036d8     libucrt:lcidtoname_downlevel.obj
 0001:000026e0       ??_C@_15HPJPHDM@?$AAb?$AAe?$AA?$AA@ 100036e0     libucrt:lcidtoname_downlevel.obj
 0001:000026e8       ??_C@_15LCHLGJII@?$AAs?$AAl?$AA?$AA@ 100036e8     libucrt:lcidtoname_downlevel.obj
 0001:000026f0       ??_C@_15PCFJPHHO@?$AAe?$AAt?$AA?$AA@ 100036f0     libucrt:lcidtoname_downlevel.obj
 0001:000026f8       ??_C@_15HPFPGODN@?$AAl?$AAv?$AA?$AA@ 100036f8     libucrt:lcidtoname_downlevel.obj
 0001:00002700       ??_C@_15NFFGKGLG@?$AAl?$AAt?$AA?$AA@ 10003700     libucrt:lcidtoname_downlevel.obj
 0001:00002708       ??_C@_15BDAKCCHN@?$AAf?$AAa?$AA?$AA@ 10003708     libucrt:lcidtoname_downlevel.obj
 0001:00002710       ??_C@_15NFGIAIAJ@?$AAv?$AAi?$AA?$AA@ 10003710     libucrt:lcidtoname_downlevel.obj
 0001:00002718       ??_C@_15LMKNDMHN@?$AAh?$AAy?$AA?$AA@ 10003718     libucrt:lcidtoname_downlevel.obj
 0001:00002720       ??_C@_15IJBHMCFL@?$AAa?$AAz?$AA?$AA@ 10003720     libucrt:lcidtoname_downlevel.obj
 0001:00002728       ??_C@_15EKOFJABL@?$AAe?$AAu?$AA?$AA@ 10003728     libucrt:lcidtoname_downlevel.obj
 0001:00002730       ??_C@_15BGHADCNK@?$AAm?$AAk?$AA?$AA@ 10003730     libucrt:lcidtoname_downlevel.obj
 0001:00002738       ??_C@_15JDNICKHM@?$AAa?$AAf?$AA?$AA@ 10003738     libucrt:lcidtoname_downlevel.obj
 0001:00002740       ??_C@_15KPJEDBKD@?$AAk?$AAa?$AA?$AA@ 10003740     libucrt:lcidtoname_downlevel.obj
 0001:00002748       ??_C@_15PDNFFFEO@?$AAf?$AAo?$AA?$AA@ 10003748     libucrt:lcidtoname_downlevel.obj
 0001:00002750       ??_C@_15OMLEGLOC@?$AAh?$AAi?$AA?$AA@ 10003750     libucrt:lcidtoname_downlevel.obj
 0001:00002758       ??_C@_15IDNNENKK@?$AAm?$AAs?$AA?$AA@ 10003758     libucrt:lcidtoname_downlevel.obj
 0001:00002760       ??_C@_15MACJNBMH@?$AAk?$AAk?$AA?$AA@ 10003760     libucrt:lcidtoname_downlevel.obj
 0001:00002768       ??_C@_15DKDJEOND@?$AAk?$AAy?$AA?$AA@ 10003768     libucrt:lcidtoname_downlevel.obj
 0001:00002770       ??_C@_15DFGDLJBG@?$AAs?$AAw?$AA?$AA@ 10003770     libucrt:lcidtoname_downlevel.obj
 0001:00002778       ??_C@_15BBFAICNG@?$AAu?$AAz?$AA?$AA@ 10003778     libucrt:lcidtoname_downlevel.obj
 0001:00002780       ??_C@_15DKNDCGEA@?$AAt?$AAt?$AA?$AA@ 10003780     libucrt:lcidtoname_downlevel.obj
 0001:00002788       ??_C@_15MGIFMDPL@?$AAp?$AAa?$AA?$AA@ 10003788     libucrt:lcidtoname_downlevel.obj
 0001:00002790       ??_C@_15HCNDBBA@?$AAg?$AAu?$AA?$AA@ 10003790     libucrt:lcidtoname_downlevel.obj
 0001:00002798       ??_C@_15FNBEIBON@?$AAt?$AAa?$AA?$AA@ 10003798     libucrt:lcidtoname_downlevel.obj
 0001:000027a0       ??_C@_15NCHGBGLK@?$AAt?$AAe?$AA?$AA@ 100037a0     libucrt:lcidtoname_downlevel.obj
 0001:000027a8       ??_C@_15PHPHCBPF@?$AAk?$AAn?$AA?$AA@ 100037a8     libucrt:lcidtoname_downlevel.obj
 0001:000027b0       ??_C@_15DLGBCKMP@?$AAm?$AAr?$AA?$AA@ 100037b0     libucrt:lcidtoname_downlevel.obj
 0001:000027b8       ??_C@_15EABBLBFF@?$AAs?$AAa?$AA?$AA@ 100037b8     libucrt:lcidtoname_downlevel.obj
 0001:000027c0       ??_C@_15CBKOMCOI@?$AAm?$AAn?$AA?$AA@ 100037c0     libucrt:lcidtoname_downlevel.obj
 0001:000027c8       ??_C@_15CKDMCJAF@?$AAg?$AAl?$AA?$AA@ 100037c8     libucrt:lcidtoname_downlevel.obj
 0001:000027d0       ??_C@_17CNJFBPG@?$AAk?$AAo?$AAk?$AA?$AA@ 100037d0     libucrt:lcidtoname_downlevel.obj
 0001:000027d8       ??_C@_17FFBJICPL@?$AAs?$AAy?$AAr?$AA?$AA@ 100037d8     libucrt:lcidtoname_downlevel.obj
 0001:000027e0       ??_C@_17KPNDCPAF@?$AAd?$AAi?$AAv?$AA?$AA@ 100037e0     libucrt:lcidtoname_downlevel.obj
 0001:000027e8       ??_C@_1M@OKAHONE@?$AAa?$AAr?$AA?9?$AAS?$AAA?$AA?$AA@ 100037e8     libucrt:lcidtoname_downlevel.obj
 0001:000027f4       ??_C@_1M@FFFIGIGK@?$AAb?$AAg?$AA?9?$AAB?$AAG?$AA?$AA@ 100037f4     libucrt:lcidtoname_downlevel.obj
 0001:00002800       ??_C@_1M@BJNKEDC@?$AAc?$AAa?$AA?9?$AAE?$AAS?$AA?$AA@ 10003800     libucrt:lcidtoname_downlevel.obj
 0001:0000280c       ??_C@_1M@IJJHFJHA@?$AAc?$AAs?$AA?9?$AAC?$AAZ?$AA?$AA@ 1000380c     libucrt:lcidtoname_downlevel.obj
 0001:00002818       ??_C@_1M@CLPEOBGI@?$AAd?$AAa?$AA?9?$AAD?$AAK?$AA?$AA@ 10003818     libucrt:lcidtoname_downlevel.obj
 0001:00002824       ??_C@_1M@MCMADGCB@?$AAd?$AAe?$AA?9?$AAD?$AAE?$AA?$AA@ 10003824     libucrt:lcidtoname_downlevel.obj
 0001:00002830       ??_C@_1M@OOCKEMAM@?$AAe?$AAl?$AA?9?$AAG?$AAR?$AA?$AA@ 10003830     libucrt:lcidtoname_downlevel.obj
 0001:0000283c       ??_C@_1M@DDNJFGID@?$AAf?$AAi?$AA?9?$AAF?$AAI?$AA?$AA@ 1000383c     libucrt:lcidtoname_downlevel.obj
 0001:00002848       ??_C@_1M@GLIPPMAC@?$AAf?$AAr?$AA?9?$AAF?$AAR?$AA?$AA@ 10003848     libucrt:lcidtoname_downlevel.obj
 0001:00002854       ??_C@_1M@GFMCHPE@?$AAh?$AAe?$AA?9?$AAI?$AAL?$AA?$AA@ 10003854     libucrt:lcidtoname_downlevel.obj
 0001:00002860       ??_C@_1M@MHLPGNKM@?$AAh?$AAu?$AA?9?$AAH?$AAU?$AA?$AA@ 10003860     libucrt:lcidtoname_downlevel.obj
 0001:0000286c       ??_C@_1M@LPDDNNPN@?$AAi?$AAs?$AA?9?$AAI?$AAS?$AA?$AA@ 1000386c     libucrt:lcidtoname_downlevel.obj
 0001:00002878       ??_C@_1M@MADIPODN@?$AAi?$AAt?$AA?9?$AAI?$AAT?$AA?$AA@ 10003878     libucrt:lcidtoname_downlevel.obj
 0001:00002884       ??_C@_1M@IHBJJGG@?$AAn?$AAl?$AA?9?$AAN?$AAL?$AA?$AA@ 10003884     libucrt:lcidtoname_downlevel.obj
 0001:00002890       ??_C@_1M@EANAGDL@?$AAn?$AAb?$AA?9?$AAN?$AAO?$AA?$AA@ 10003890     libucrt:lcidtoname_downlevel.obj
 0001:0000289c       ??_C@_1M@NEIEMEGP@?$AAp?$AAl?$AA?9?$AAP?$AAL?$AA?$AA@ 1000389c     libucrt:lcidtoname_downlevel.obj
 0001:000028a8       ??_C@_1M@BOCFIGEP@?$AAp?$AAt?$AA?9?$AAB?$AAR?$AA?$AA@ 100038a8     libucrt:lcidtoname_downlevel.obj
 0001:000028b4       ??_C@_1M@IMPFOPBG@?$AAr?$AAo?$AA?9?$AAR?$AAO?$AA?$AA@ 100038b4     libucrt:lcidtoname_downlevel.obj
 0001:000028c0       ??_C@_1M@IDNNEJMM@?$AAr?$AAu?$AA?9?$AAR?$AAU?$AA?$AA@ 100038c0     libucrt:lcidtoname_downlevel.obj
 0001:000028cc       ??_C@_1M@LILEEOGM@?$AAh?$AAr?$AA?9?$AAH?$AAR?$AA?$AA@ 100038cc     libucrt:lcidtoname_downlevel.obj
 0001:000028d8       ??_C@_1M@FKIFEHPB@?$AAs?$AAk?$AA?9?$AAS?$AAK?$AA?$AA@ 100038d8     libucrt:lcidtoname_downlevel.obj
 0001:000028e4       ??_C@_1M@LJMAMNPJ@?$AAs?$AAq?$AA?9?$AAA?$AAL?$AA?$AA@ 100038e4     libucrt:lcidtoname_downlevel.obj
 0001:000028f0       ??_C@_1M@GIAKDKJK@?$AAs?$AAv?$AA?9?$AAS?$AAE?$AA?$AA@ 100038f0     libucrt:lcidtoname_downlevel.obj
 0001:000028fc       ??_C@_1M@MKJKIKCL@?$AAt?$AAh?$AA?9?$AAT?$AAH?$AA?$AA@ 100038fc     libucrt:lcidtoname_downlevel.obj
 0001:00002908       ??_C@_1M@MFLCCMPB@?$AAt?$AAr?$AA?9?$AAT?$AAR?$AA?$AA@ 10003908     libucrt:lcidtoname_downlevel.obj
 0001:00002914       ??_C@_1M@OIJHDKJN@?$AAu?$AAr?$AA?9?$AAP?$AAK?$AA?$AA@ 10003914     libucrt:lcidtoname_downlevel.obj
 0001:00002920       ??_C@_1M@LHIPCIEK@?$AAi?$AAd?$AA?9?$AAI?$AAD?$AA?$AA@ 10003920     libucrt:lcidtoname_downlevel.obj
 0001:0000292c       ??_C@_1M@MFMOBGI@?$AAu?$AAk?$AA?9?$AAU?$AAA?$AA?$AA@ 1000392c     libucrt:lcidtoname_downlevel.obj
 0001:00002938       ??_C@_1M@OBGLJIPL@?$AAb?$AAe?$AA?9?$AAB?$AAY?$AA?$AA@ 10003938     libucrt:lcidtoname_downlevel.obj
 0001:00002944       ??_C@_1M@BCFAJEAD@?$AAs?$AAl?$AA?9?$AAS?$AAI?$AA?$AA@ 10003944     libucrt:lcidtoname_downlevel.obj
 0001:00002950       ??_C@_1M@FKFFEDDN@?$AAe?$AAt?$AA?9?$AAE?$AAE?$AA?$AA@ 10003950     libucrt:lcidtoname_downlevel.obj
 0001:0000295c       ??_C@_1M@KGKKAACI@?$AAl?$AAv?$AA?9?$AAL?$AAV?$AA?$AA@ 1000395c     libucrt:lcidtoname_downlevel.obj
 0001:00002968       ??_C@_1M@IFGBIJO@?$AAl?$AAt?$AA?9?$AAL?$AAT?$AA?$AA@ 10003968     libucrt:lcidtoname_downlevel.obj
 0001:00002974       ??_C@_1M@FGEAHEDM@?$AAf?$AAa?$AA?9?$AAI?$AAR?$AA?$AA@ 10003974     libucrt:lcidtoname_downlevel.obj
 0001:00002980       ??_C@_1M@KBMAIBFN@?$AAv?$AAi?$AA?9?$AAV?$AAN?$AA?$AA@ 10003980     libucrt:lcidtoname_downlevel.obj
 0001:0000298c       ??_C@_1M@GPCBKDJK@?$AAh?$AAy?$AA?9?$AAA?$AAM?$AA?$AA@ 1000398c     libucrt:lcidtoname_downlevel.obj
 0001:00002998       ??_C@_1BG@BECMDDJB@?$AAa?$AAz?$AA?9?$AAA?$AAZ?$AA?9?$AAL?$AAa?$AAt?$AAn?$AA?$AA@ 10003998     libucrt:lcidtoname_downlevel.obj
 0001:000029b0       ??_C@_1M@MAOFCAEA@?$AAe?$AAu?$AA?9?$AAE?$AAS?$AA?$AA@ 100039b0     libucrt:lcidtoname_downlevel.obj
 0001:000029bc       ??_C@_1M@IGHABKPI@?$AAm?$AAk?$AA?9?$AAM?$AAK?$AA?$AA@ 100039bc     libucrt:lcidtoname_downlevel.obj
 0001:000029c8       ??_C@_1M@IAIGNEJG@?$AAt?$AAn?$AA?9?$AAZ?$AAA?$AA?$AA@ 100039c8     libucrt:lcidtoname_downlevel.obj
 0001:000029d4       ??_C@_1M@IIJCOJFA@?$AAx?$AAh?$AA?9?$AAZ?$AAA?$AA?$AA@ 100039d4     libucrt:lcidtoname_downlevel.obj
 0001:000029e0       ??_C@_1M@LGPJHNJH@?$AAz?$AAu?$AA?9?$AAZ?$AAA?$AA?$AA@ 100039e0     libucrt:lcidtoname_downlevel.obj
 0001:000029ec       ??_C@_1M@HOKAOIO@?$AAa?$AAf?$AA?9?$AAZ?$AAA?$AA?$AA@ 100039ec     libucrt:lcidtoname_downlevel.obj
 0001:000029f8       ??_C@_1M@DPCLHLIE@?$AAk?$AAa?$AA?9?$AAG?$AAE?$AA?$AA@ 100039f8     libucrt:lcidtoname_downlevel.obj
 0001:00002a04       ??_C@_1M@BLKMHJBI@?$AAf?$AAo?$AA?9?$AAF?$AAO?$AA?$AA@ 10003a04     libucrt:lcidtoname_downlevel.obj
 0001:00002a10       ??_C@_1M@LGGJAPPB@?$AAh?$AAi?$AA?9?$AAI?$AAN?$AA?$AA@ 10003a10     libucrt:lcidtoname_downlevel.obj
 0001:00002a1c       ??_C@_1M@FIKPIHFE@?$AAm?$AAt?$AA?9?$AAM?$AAT?$AA?$AA@ 10003a1c     libucrt:lcidtoname_downlevel.obj
 0001:00002a28       ??_C@_1M@HEGGPBFA@?$AAs?$AAe?$AA?9?$AAN?$AAO?$AA?$AA@ 10003a28     libucrt:lcidtoname_downlevel.obj
 0001:00002a34       ??_C@_1M@EIBJEEPA@?$AAm?$AAs?$AA?9?$AAM?$AAY?$AA?$AA@ 10003a34     libucrt:lcidtoname_downlevel.obj
 0001:00002a40       ??_C@_1M@FHLBGMPP@?$AAk?$AAk?$AA?9?$AAK?$AAZ?$AA?$AA@ 10003a40     libucrt:lcidtoname_downlevel.obj
 0001:00002a4c       ??_C@_1M@NGJJLCGI@?$AAk?$AAy?$AA?9?$AAK?$AAG?$AA?$AA@ 10003a4c     libucrt:lcidtoname_downlevel.obj
 0001:00002a58       ??_C@_1M@GIENNBFC@?$AAs?$AAw?$AA?9?$AAK?$AAE?$AA?$AA@ 10003a58     libucrt:lcidtoname_downlevel.obj
 0001:00002a64       ??_C@_1BG@NDGMJIMJ@?$AAu?$AAz?$AA?9?$AAU?$AAZ?$AA?9?$AAL?$AAa?$AAt?$AAn?$AA?$AA@ 10003a64     libucrt:lcidtoname_downlevel.obj
 0001:00002a7c       ??_C@_1M@IDCCIHBC@?$AAt?$AAt?$AA?9?$AAR?$AAU?$AA?$AA@ 10003a7c     libucrt:lcidtoname_downlevel.obj
 0001:00002a88       ??_C@_1M@LOICPMOJ@?$AAb?$AAn?$AA?9?$AAI?$AAN?$AA?$AA@ 10003a88     libucrt:lcidtoname_downlevel.obj
 0001:00002a94       ??_C@_1M@KPKKNEAH@?$AAp?$AAa?$AA?9?$AAI?$AAN?$AA?$AA@ 10003a94     libucrt:lcidtoname_downlevel.obj
 0001:00002aa0       ??_C@_1M@PJGPPBOG@?$AAg?$AAu?$AA?9?$AAI?$AAN?$AA?$AA@ 10003aa0     libucrt:lcidtoname_downlevel.obj
 0001:00002aac       ??_C@_1M@KMKMOPHI@?$AAt?$AAa?$AA?9?$AAI?$AAN?$AA?$AA@ 10003aac     libucrt:lcidtoname_downlevel.obj
 0001:00002ab8       ??_C@_1M@KFEHEPAC@?$AAt?$AAe?$AA?9?$AAI?$AAN?$AA?$AA@ 10003ab8     libucrt:lcidtoname_downlevel.obj
 0001:00002ac4       ??_C@_1M@CDCLMGHI@?$AAk?$AAn?$AA?9?$AAI?$AAN?$AA?$AA@ 10003ac4     libucrt:lcidtoname_downlevel.obj
 0001:00002ad0       ??_C@_1M@MIODLDKF@?$AAm?$AAl?$AA?9?$AAI?$AAN?$AA?$AA@ 10003ad0     libucrt:lcidtoname_downlevel.obj
 0001:00002adc       ??_C@_1M@PBIEACPO@?$AAm?$AAr?$AA?9?$AAI?$AAN?$AA?$AA@ 10003adc     libucrt:lcidtoname_downlevel.obj
 0001:00002ae8       ??_C@_1M@NIDEAGPH@?$AAs?$AAa?$AA?9?$AAI?$AAN?$AA?$AA@ 10003ae8     libucrt:lcidtoname_downlevel.obj
 0001:00002af4       ??_C@_1M@FHIHCBIO@?$AAm?$AAn?$AA?9?$AAM?$AAN?$AA?$AA@ 10003af4     libucrt:lcidtoname_downlevel.obj
 0001:00002b00       ??_C@_1M@JAIJPENP@?$AAc?$AAy?$AA?9?$AAG?$AAB?$AA?$AA@ 10003b00     libucrt:lcidtoname_downlevel.obj
 0001:00002b0c       ??_C@_1M@PHGFBEPN@?$AAg?$AAl?$AA?9?$AAE?$AAS?$AA?$AA@ 10003b0c     libucrt:lcidtoname_downlevel.obj
 0001:00002b18       ??_C@_1O@KPIPDNCP@?$AAk?$AAo?$AAk?$AA?9?$AAI?$AAN?$AA?$AA@ 10003b18     libucrt:lcidtoname_downlevel.obj
 0001:00002b28       ??_C@_1O@KNHJLDJA@?$AAs?$AAy?$AAr?$AA?9?$AAS?$AAY?$AA?$AA@ 10003b28     libucrt:lcidtoname_downlevel.obj
 0001:00002b38       ??_C@_1O@MKEKBLAH@?$AAd?$AAi?$AAv?$AA?9?$AAM?$AAV?$AA?$AA@ 10003b38     libucrt:lcidtoname_downlevel.obj
 0001:00002b48       ??_C@_1O@OHDCKDDF@?$AAq?$AAu?$AAz?$AA?9?$AAB?$AAO?$AA?$AA@ 10003b48     libucrt:lcidtoname_downlevel.obj
 0001:00002b58       ??_C@_1M@LEPJNLFD@?$AAn?$AAs?$AA?9?$AAZ?$AAA?$AA?$AA@ 10003b58     libucrt:lcidtoname_downlevel.obj
 0001:00002b64       ??_C@_1M@OMLEIIJB@?$AAm?$AAi?$AA?9?$AAN?$AAZ?$AA?$AA@ 10003b64     libucrt:lcidtoname_downlevel.obj
 0001:00002b70       ??_C@_1M@PMPEAILG@?$AAa?$AAr?$AA?9?$AAI?$AAQ?$AA?$AA@ 10003b70     libucrt:lcidtoname_downlevel.obj
 0001:00002b7c       ??_C@_1M@CNKPNOEE@?$AAd?$AAe?$AA?9?$AAC?$AAH?$AA?$AA@ 10003b7c     libucrt:lcidtoname_downlevel.obj
 0001:00002b88       ??_C@_1M@LKMGMLKO@?$AAe?$AAn?$AA?9?$AAG?$AAB?$AA?$AA@ 10003b88     libucrt:lcidtoname_downlevel.obj
 0001:00002b94       ??_C@_1M@PGKJFFGL@?$AAe?$AAs?$AA?9?$AAM?$AAX?$AA?$AA@ 10003b94     libucrt:lcidtoname_downlevel.obj
 0001:00002ba0       ??_C@_1M@DNNANBDC@?$AAf?$AAr?$AA?9?$AAB?$AAE?$AA?$AA@ 10003ba0     libucrt:lcidtoname_downlevel.obj
 0001:00002bac       ??_C@_1M@HLGMDFHM@?$AAi?$AAt?$AA?9?$AAC?$AAH?$AA?$AA@ 10003bac     libucrt:lcidtoname_downlevel.obj
 0001:00002bb8       ??_C@_1M@CLLBGJH@?$AAn?$AAl?$AA?9?$AAB?$AAE?$AA?$AA@ 10003bb8     libucrt:lcidtoname_downlevel.obj
 0001:00002bc4       ??_C@_1M@BODBOGLF@?$AAn?$AAn?$AA?9?$AAN?$AAO?$AA?$AA@ 10003bc4     libucrt:lcidtoname_downlevel.obj
 0001:00002bd0       ??_C@_1M@HFFAHKAD@?$AAp?$AAt?$AA?9?$AAP?$AAT?$AA?$AA@ 10003bd0     libucrt:lcidtoname_downlevel.obj
 0001:00002bdc       ??_C@_1BG@LNOAKHIE@?$AAs?$AAr?$AA?9?$AAS?$AAP?$AA?9?$AAL?$AAa?$AAt?$AAn?$AA?$AA@ 10003bdc     libucrt:lcidtoname_downlevel.obj
 0001:00002bf4       ??_C@_1M@HBMHBGAK@?$AAs?$AAv?$AA?9?$AAF?$AAI?$AA?$AA@ 10003bf4     libucrt:lcidtoname_downlevel.obj
 0001:00002c00       ??_C@_1BG@DGCJGJBE@?$AAa?$AAz?$AA?9?$AAA?$AAZ?$AA?9?$AAC?$AAy?$AAr?$AAl?$AA?$AA@ 10003c00     libucrt:lcidtoname_downlevel.obj
 0001:00002c18       ??_C@_1M@KEJDAAHB@?$AAs?$AAe?$AA?9?$AAS?$AAE?$AA?$AA@ 10003c18     libucrt:lcidtoname_downlevel.obj
 0001:00002c24       ??_C@_1M@HEIBJJAD@?$AAm?$AAs?$AA?9?$AAB?$AAN?$AA?$AA@ 10003c24     libucrt:lcidtoname_downlevel.obj
 0001:00002c30       ??_C@_1BG@PBGJMCEM@?$AAu?$AAz?$AA?9?$AAU?$AAZ?$AA?9?$AAC?$AAy?$AAr?$AAl?$AA?$AA@ 10003c30     libucrt:lcidtoname_downlevel.obj
 0001:00002c48       ??_C@_1O@LAOBCMDF@?$AAq?$AAu?$AAz?$AA?9?$AAE?$AAC?$AA?$AA@ 10003c48     libucrt:lcidtoname_downlevel.obj
 0001:00002c58       ??_C@_1M@POEEMAIO@?$AAa?$AAr?$AA?9?$AAE?$AAG?$AA?$AA@ 10003c58     libucrt:lcidtoname_downlevel.obj
 0001:00002c64       ??_C@_1M@EFAKDEDL@?$AAz?$AAh?$AA?9?$AAH?$AAK?$AA?$AA@ 10003c64     libucrt:lcidtoname_downlevel.obj
 0001:00002c70       ??_C@_1M@HKKIJHGI@?$AAd?$AAe?$AA?9?$AAA?$AAT?$AA?$AA@ 10003c70     libucrt:lcidtoname_downlevel.obj
 0001:00002c7c       ??_C@_1M@KBFBEHJF@?$AAe?$AAn?$AA?9?$AAA?$AAU?$AA?$AA@ 10003c7c     libucrt:lcidtoname_downlevel.obj
 0001:00002c88       ??_C@_1M@MNPLFAAH@?$AAe?$AAs?$AA?9?$AAE?$AAS?$AA?$AA@ 10003c88     libucrt:lcidtoname_downlevel.obj
 0001:00002c94       ??_C@_1M@HJOOJFMA@?$AAf?$AAr?$AA?9?$AAC?$AAA?$AA?$AA@ 10003c94     libucrt:lcidtoname_downlevel.obj
 0001:00002ca0       ??_C@_1BG@JPOFPNAB@?$AAs?$AAr?$AA?9?$AAS?$AAP?$AA?9?$AAC?$AAy?$AAr?$AAl?$AA?$AA@ 10003ca0     libucrt:lcidtoname_downlevel.obj
 0001:00002cb8       ??_C@_1M@LNFOCMOB@?$AAs?$AAe?$AA?9?$AAF?$AAI?$AA?$AA@ 10003cb8     libucrt:lcidtoname_downlevel.obj
 0001:00002cc4       ??_C@_1O@MGJBOAMB@?$AAq?$AAu?$AAz?$AA?9?$AAP?$AAE?$AA?$AA@ 10003cc4     libucrt:lcidtoname_downlevel.obj
 0001:00002cd4       ??_C@_1M@GJINLBOK@?$AAa?$AAr?$AA?9?$AAL?$AAY?$AA?$AA@ 10003cd4     libucrt:lcidtoname_downlevel.obj
 0001:00002ce0       ??_C@_1M@GGMNHJNL@?$AAz?$AAh?$AA?9?$AAS?$AAG?$AA?$AA@ 10003ce0     libucrt:lcidtoname_downlevel.obj
 0001:00002cec       ??_C@_1M@HOIKODND@?$AAd?$AAe?$AA?9?$AAL?$AAU?$AA?$AA@ 10003cec     libucrt:lcidtoname_downlevel.obj
 0001:00002cf8       ??_C@_1M@DDOCCGFG@?$AAe?$AAn?$AA?9?$AAC?$AAA?$AA?$AA@ 10003cf8     libucrt:lcidtoname_downlevel.obj
 0001:00002d04       ??_C@_1M@BNOEMJLF@?$AAe?$AAs?$AA?9?$AAG?$AAT?$AA?$AA@ 10003d04     libucrt:lcidtoname_downlevel.obj
 0001:00002d10       ??_C@_1M@EOGNKEK@?$AAf?$AAr?$AA?9?$AAC?$AAH?$AA?$AA@ 10003d10     libucrt:lcidtoname_downlevel.obj
 0001:00002d1c       ??_C@_1M@FLIDJFHL@?$AAh?$AAr?$AA?9?$AAB?$AAA?$AA?$AA@ 10003d1c     libucrt:lcidtoname_downlevel.obj
 0001:00002d28       ??_C@_1O@FMCELNAJ@?$AAs?$AAm?$AAj?$AA?9?$AAN?$AAO?$AA?$AA@ 10003d28     libucrt:lcidtoname_downlevel.obj
 0001:00002d38       ??_C@_1M@JHGLJMGJ@?$AAa?$AAr?$AA?9?$AAD?$AAZ?$AA?$AA@ 10003d38     libucrt:lcidtoname_downlevel.obj
 0001:00002d44       ??_C@_1M@JKKFDCNP@?$AAz?$AAh?$AA?9?$AAM?$AAO?$AA?$AA@ 10003d44     libucrt:lcidtoname_downlevel.obj
 0001:00002d50       ??_C@_1M@GEEFALPE@?$AAd?$AAe?$AA?9?$AAL?$AAI?$AA?$AA@ 10003d50     libucrt:lcidtoname_downlevel.obj
 0001:00002d5c       ??_C@_1M@IGEOFBG@?$AAe?$AAn?$AA?9?$AAN?$AAZ?$AA?$AA@ 10003d5c     libucrt:lcidtoname_downlevel.obj
 0001:00002d68       ??_C@_1M@KDBONEHP@?$AAe?$AAs?$AA?9?$AAC?$AAR?$AA?$AA@ 10003d68     libucrt:lcidtoname_downlevel.obj
 0001:00002d74       ??_C@_1M@FHMDOHNN@?$AAf?$AAr?$AA?9?$AAL?$AAU?$AA?$AA@ 10003d74     libucrt:lcidtoname_downlevel.obj
 0001:00002d80       ??_C@_1BG@NFKKMAFG@?$AAb?$AAs?$AA?9?$AAB?$AAA?$AA?9?$AAL?$AAa?$AAt?$AAn?$AA?$AA@ 10003d80     libucrt:lcidtoname_downlevel.obj
 0001:00002d98       ??_C@_1O@IMNBEMCI@?$AAs?$AAm?$AAj?$AA?9?$AAS?$AAE?$AA?$AA@ 10003d98     libucrt:lcidtoname_downlevel.obj
 0001:00002da8       ??_C@_1M@DHHMBNDP@?$AAa?$AAr?$AA?9?$AAM?$AAA?$AA?$AA@ 10003da8     libucrt:lcidtoname_downlevel.obj
 0001:00002db4       ??_C@_1M@BNBLJCGH@?$AAe?$AAn?$AA?9?$AAI?$AAE?$AA?$AA@ 10003db4     libucrt:lcidtoname_downlevel.obj
 0001:00002dc0       ??_C@_1M@GEPAFMDL@?$AAe?$AAs?$AA?9?$AAP?$AAA?$AA?$AA@ 10003dc0     libucrt:lcidtoname_downlevel.obj
 0001:00002dcc       ??_C@_1M@OJONDMDL@?$AAf?$AAr?$AA?9?$AAM?$AAC?$AA?$AA@ 10003dcc     libucrt:lcidtoname_downlevel.obj
 0001:00002dd8       ??_C@_1BG@OBCNFJB@?$AAs?$AAr?$AA?9?$AAB?$AAA?$AA?9?$AAL?$AAa?$AAt?$AAn?$AA?$AA@ 10003dd8     libucrt:lcidtoname_downlevel.obj
 0001:00002df0       ??_C@_1O@KEMEEGPO@?$AAs?$AAm?$AAa?$AA?9?$AAN?$AAO?$AA?$AA@ 10003df0     libucrt:lcidtoname_downlevel.obj
 0001:00002e00       ??_C@_1M@ELMGFODK@?$AAa?$AAr?$AA?9?$AAT?$AAN?$AA?$AA@ 10003e00     libucrt:lcidtoname_downlevel.obj
 0001:00002e0c       ??_C@_1M@BHDLHFAF@?$AAe?$AAn?$AA?9?$AAZ?$AAA?$AA?$AA@ 10003e0c     libucrt:lcidtoname_downlevel.obj
 0001:00002e18       ??_C@_1M@BMGIGLIF@?$AAe?$AAs?$AA?9?$AAD?$AAO?$AA?$AA@ 10003e18     libucrt:lcidtoname_downlevel.obj
 0001:00002e24       ??_C@_1BG@CMBHIPBE@?$AAs?$AAr?$AA?9?$AAB?$AAA?$AA?9?$AAC?$AAy?$AAr?$AAl?$AA?$AA@ 10003e24     libucrt:lcidtoname_downlevel.obj
 0001:00002e3c       ??_C@_1O@HEDBLHNP@?$AAs?$AAm?$AAa?$AA?9?$AAS?$AAE?$AA?$AA@ 10003e3c     libucrt:lcidtoname_downlevel.obj
 0001:00002e4c       ??_C@_1M@DAGCADIM@?$AAa?$AAr?$AA?9?$AAO?$AAM?$AA?$AA@ 10003e4c     libucrt:lcidtoname_downlevel.obj
 0001:00002e58       ??_C@_1M@FODLMICG@?$AAe?$AAn?$AA?9?$AAJ?$AAM?$AA?$AA@ 10003e58     libucrt:lcidtoname_downlevel.obj
 0001:00002e64       ??_C@_1M@DNMLCIHB@?$AAe?$AAs?$AA?9?$AAV?$AAE?$AA?$AA@ 10003e64     libucrt:lcidtoname_downlevel.obj
 0001:00002e70       ??_C@_1O@EOKHMKJK@?$AAs?$AAm?$AAs?$AA?9?$AAF?$AAI?$AA?$AA@ 10003e70     libucrt:lcidtoname_downlevel.obj
 0001:00002e80       ??_C@_1M@CAFJMKOF@?$AAa?$AAr?$AA?9?$AAY?$AAE?$AA?$AA@ 10003e80     libucrt:lcidtoname_downlevel.obj
 0001:00002e8c       ??_C@_1M@CBFHIJLI@?$AAe?$AAn?$AA?9?$AAC?$AAB?$AA?$AA@ 10003e8c     libucrt:lcidtoname_downlevel.obj
 0001:00002e98       ??_C@_1M@BGNFLDN@?$AAe?$AAs?$AA?9?$AAC?$AAO?$AA?$AA@ 10003e98     libucrt:lcidtoname_downlevel.obj
 0001:00002ea4       ??_C@_1O@JMPHMAMC@?$AAs?$AAm?$AAn?$AA?9?$AAF?$AAI?$AA?$AA@ 10003ea4     libucrt:lcidtoname_downlevel.obj
 0001:00002eb4       ??_C@_1M@JLANABKE@?$AAa?$AAr?$AA?9?$AAS?$AAY?$AA?$AA@ 10003eb4     libucrt:lcidtoname_downlevel.obj
 0001:00002ec0       ??_C@_1M@HPKGCFGN@?$AAe?$AAn?$AA?9?$AAB?$AAZ?$AA?$AA@ 10003ec0     libucrt:lcidtoname_downlevel.obj
 0001:00002ecc       ??_C@_1M@OLJCMLGM@?$AAe?$AAs?$AA?9?$AAP?$AAE?$AA?$AA@ 10003ecc     libucrt:lcidtoname_downlevel.obj
 0001:00002ed8       ??_C@_1M@MKKGFKLE@?$AAa?$AAr?$AA?9?$AAJ?$AAO?$AA?$AA@ 10003ed8     libucrt:lcidtoname_downlevel.obj
 0001:00002ee4       ??_C@_1M@EKPGLDNI@?$AAe?$AAn?$AA?9?$AAT?$AAT?$AA?$AA@ 10003ee4     libucrt:lcidtoname_downlevel.obj
 0001:00002ef0       ??_C@_1M@OONGHFHE@?$AAe?$AAs?$AA?9?$AAA?$AAR?$AA?$AA@ 10003ef0     libucrt:lcidtoname_downlevel.obj
 0001:00002efc       ??_C@_1M@OOJFGBHE@?$AAa?$AAr?$AA?9?$AAL?$AAB?$AA?$AA@ 10003efc     libucrt:lcidtoname_downlevel.obj
 0001:00002f08       ??_C@_1M@GCEJHNEG@?$AAe?$AAn?$AA?9?$AAZ?$AAW?$AA?$AA@ 10003f08     libucrt:lcidtoname_downlevel.obj
 0001:00002f14       ??_C@_1M@JNOCAHJI@?$AAe?$AAs?$AA?9?$AAE?$AAC?$AA?$AA@ 10003f14     libucrt:lcidtoname_downlevel.obj
 0001:00002f20       ??_C@_1M@JEFHPGGB@?$AAa?$AAr?$AA?9?$AAK?$AAW?$AA?$AA@ 10003f20     libucrt:lcidtoname_downlevel.obj
 0001:00002f2c       ??_C@_1M@MLKIBJOJ@?$AAe?$AAn?$AA?9?$AAP?$AAH?$AA?$AA@ 10003f2c     libucrt:lcidtoname_downlevel.obj
 0001:00002f38       ??_C@_1M@BDNIPEND@?$AAe?$AAs?$AA?9?$AAC?$AAL?$AA?$AA@ 10003f38     libucrt:lcidtoname_downlevel.obj
 0001:00002f44       ??_C@_1M@MPNMEKBD@?$AAa?$AAr?$AA?9?$AAA?$AAE?$AA?$AA@ 10003f44     libucrt:lcidtoname_downlevel.obj
 0001:00002f50       ??_C@_1M@KBJALCPI@?$AAe?$AAs?$AA?9?$AAU?$AAY?$AA?$AA@ 10003f50     libucrt:lcidtoname_downlevel.obj
 0001:00002f5c       ??_C@_1M@LLCCOAGA@?$AAa?$AAr?$AA?9?$AAB?$AAH?$AA?$AA@ 10003f5c     libucrt:lcidtoname_downlevel.obj
 0001:00002f68       ??_C@_1M@PBFNCDEL@?$AAe?$AAs?$AA?9?$AAP?$AAY?$AA?$AA@ 10003f68     libucrt:lcidtoname_downlevel.obj
 0001:00002f74       ??_C@_1M@EDGINPNP@?$AAa?$AAr?$AA?9?$AAQ?$AAA?$AA?$AA@ 10003f74     libucrt:lcidtoname_downlevel.obj
 0001:00002f80       ??_C@_1M@MKDBIIJI@?$AAe?$AAs?$AA?9?$AAB?$AAO?$AA?$AA@ 10003f80     libucrt:lcidtoname_downlevel.obj
 0001:00002f8c       ??_C@_1M@CPKKEBLD@?$AAe?$AAs?$AA?9?$AAS?$AAV?$AA?$AA@ 10003f8c     libucrt:lcidtoname_downlevel.obj
 0001:00002f98       ??_C@_1M@NDBGMMJL@?$AAe?$AAs?$AA?9?$AAH?$AAN?$AA?$AA@ 10003f98     libucrt:lcidtoname_downlevel.obj
 0001:00002fa4       ??_C@_1M@JIJIBHDP@?$AAe?$AAs?$AA?9?$AAN?$AAI?$AA?$AA@ 10003fa4     libucrt:lcidtoname_downlevel.obj
 0001:00002fb0       ??_C@_1M@CGFMKEEK@?$AAe?$AAs?$AA?9?$AAP?$AAR?$AA?$AA@ 10003fb0     libucrt:lcidtoname_downlevel.obj
 0001:00002fbc       ??_C@_1O@ICJHKIIK@?$AAz?$AAh?$AA?9?$AAC?$AAH?$AAT?$AA?$AA@ 10003fbc     libucrt:lcidtoname_downlevel.obj
 0001:00002fcc       ??_C@_15CLNEJCE@?$AAs?$AAr?$AA?$AA@ 10003fcc     libucrt:lcidtoname_downlevel.obj
 0001:000036f8       ??_C@_1M@KAHEKEIG@?$AAa?$AAf?$AA?9?$AAz?$AAa?$AA?$AA@ 100046f8     libucrt:lcidtoname_downlevel.obj
 0001:00003704       ??_C@_1M@GIECOABL@?$AAa?$AAr?$AA?9?$AAa?$AAe?$AA?$AA@ 10004704     libucrt:lcidtoname_downlevel.obj
 0001:00003710       ??_C@_1M@BMLMEKGI@?$AAa?$AAr?$AA?9?$AAb?$AAh?$AA?$AA@ 10004710     libucrt:lcidtoname_downlevel.obj
 0001:0000371c       ??_C@_1M@DAPFDGGB@?$AAa?$AAr?$AA?9?$AAd?$AAz?$AA?$AA@ 1000471c     libucrt:lcidtoname_downlevel.obj
 0001:00003728       ??_C@_1M@FJNKGKIG@?$AAa?$AAr?$AA?9?$AAe?$AAg?$AA?$AA@ 10004728     libucrt:lcidtoname_downlevel.obj
 0001:00003734       ??_C@_1M@FLGKKCLO@?$AAa?$AAr?$AA?9?$AAi?$AAq?$AA?$AA@ 10004734     libucrt:lcidtoname_downlevel.obj
 0001:00003740       ??_C@_1M@GNDIPALM@?$AAa?$AAr?$AA?9?$AAj?$AAo?$AA?$AA@ 10004740     libucrt:lcidtoname_downlevel.obj
 0001:0000374c       ??_C@_1M@DDMJFMGJ@?$AAa?$AAr?$AA?9?$AAk?$AAw?$AA?$AA@ 1000474c     libucrt:lcidtoname_downlevel.obj
 0001:00003758       ??_C@_1M@EJALMLHM@?$AAa?$AAr?$AA?9?$AAl?$AAb?$AA?$AA@ 10004758     libucrt:lcidtoname_downlevel.obj
 0001:00003764       ??_C@_1M@MOBDBLOC@?$AAa?$AAr?$AA?9?$AAl?$AAy?$AA?$AA@ 10004764     libucrt:lcidtoname_downlevel.obj
 0001:00003770       ??_C@_1M@JAOCLHDH@?$AAa?$AAr?$AA?9?$AAm?$AAa?$AA?$AA@ 10004770     libucrt:lcidtoname_downlevel.obj
 0001:0000377c       ??_C@_1M@JHPMKJIE@?$AAa?$AAr?$AA?9?$AAo?$AAm?$AA?$AA@ 1000477c     libucrt:lcidtoname_downlevel.obj
 0001:00003788       ??_C@_1M@OEPGHFNH@?$AAa?$AAr?$AA?9?$AAq?$AAa?$AA?$AA@ 10004788     libucrt:lcidtoname_downlevel.obj
 0001:00003794       ??_C@_1M@KJDONENM@?$AAa?$AAr?$AA?9?$AAs?$AAa?$AA?$AA@ 10004794     libucrt:lcidtoname_downlevel.obj
 0001:000037a0       ??_C@_1M@DMJDKLKM@?$AAa?$AAr?$AA?9?$AAs?$AAy?$AA?$AA@ 100047a0     libucrt:lcidtoname_downlevel.obj
 0001:000037ac       ??_C@_1M@OMFIPEDC@?$AAa?$AAr?$AA?9?$AAt?$AAn?$AA?$AA@ 100047ac     libucrt:lcidtoname_downlevel.obj
 0001:000037b8       ??_C@_1M@IHMHGAON@?$AAa?$AAr?$AA?9?$AAy?$AAe?$AA?$AA@ 100047b8     libucrt:lcidtoname_downlevel.obj
 0001:000037c4       ??_C@_1BG@KDCPGJGB@?$AAa?$AAz?$AA?9?$AAa?$AAz?$AA?9?$AAc?$AAy?$AAr?$AAl?$AA?$AA@ 100047c4     libucrt:lcidtoname_downlevel.obj
 0001:000037dc       ??_C@_1BG@IBCKDDOE@?$AAa?$AAz?$AA?9?$AAa?$AAz?$AA?9?$AAl?$AAa?$AAt?$AAn?$AA?$AA@ 100047dc     libucrt:lcidtoname_downlevel.obj
 0001:000037f4       ??_C@_1M@EGPFDCPD@?$AAb?$AAe?$AA?9?$AAb?$AAy?$AA?$AA@ 100047f4     libucrt:lcidtoname_downlevel.obj
 0001:00003800       ??_C@_1M@PCMGMCGC@?$AAb?$AAg?$AA?9?$AAb?$AAg?$AA?$AA@ 10004800     libucrt:lcidtoname_downlevel.obj
 0001:0000380c       ??_C@_1M@BJBMFGOB@?$AAb?$AAn?$AA?9?$AAi?$AAn?$AA?$AA@ 1000480c     libucrt:lcidtoname_downlevel.obj
 0001:00003818       ??_C@_1BG@EAKMMACD@?$AAb?$AAs?$AA?9?$AAb?$AAa?$AA?9?$AAl?$AAa?$AAt?$AAn?$AA?$AA@ 10004818     libucrt:lcidtoname_downlevel.obj
 0001:00003830       ??_C@_1M@KGADAODK@?$AAc?$AAa?$AA?9?$AAe?$AAs?$AA?$AA@ 10004830     libucrt:lcidtoname_downlevel.obj
 0001:0000383c       ??_C@_1M@COAJPDHI@?$AAc?$AAs?$AA?9?$AAc?$AAz?$AA?$AA@ 1000483c     libucrt:lcidtoname_downlevel.obj
 0001:00003848       ??_C@_1M@DHBHFONH@?$AAc?$AAy?$AA?9?$AAg?$AAb?$AA?$AA@ 10004848     libucrt:lcidtoname_downlevel.obj
 0001:00003854       ??_C@_1M@IMGKELGA@?$AAd?$AAa?$AA?9?$AAd?$AAk?$AA?$AA@ 10004854     libucrt:lcidtoname_downlevel.obj
 0001:00003860       ??_C@_1M@NNDGDNGA@?$AAd?$AAe?$AA?9?$AAa?$AAt?$AA?$AA@ 10004860     libucrt:lcidtoname_downlevel.obj
 0001:0000386c       ??_C@_1M@IKDBHEEM@?$AAd?$AAe?$AA?9?$AAc?$AAh?$AA?$AA@ 1000486c     libucrt:lcidtoname_downlevel.obj
 0001:00003878       ??_C@_1M@GFFOJMCJ@?$AAd?$AAe?$AA?9?$AAd?$AAe?$AA?$AA@ 10004878     libucrt:lcidtoname_downlevel.obj
 0001:00003884       ??_C@_1M@MDNLKBPM@?$AAd?$AAe?$AA?9?$AAl?$AAi?$AA?$AA@ 10004884     libucrt:lcidtoname_downlevel.obj
 0001:00003890       ??_C@_1M@NJBEEJNL@?$AAd?$AAe?$AA?9?$AAl?$AAu?$AA?$AA@ 10004890     libucrt:lcidtoname_downlevel.obj
 0001:0000389c       ??_C@_1O@GNNELBAP@?$AAd?$AAi?$AAv?$AA?9?$AAm?$AAv?$AA?$AA@ 1000489c     libucrt:lcidtoname_downlevel.obj
 0001:000038ac       ??_C@_1M@EJLEOGAE@?$AAe?$AAl?$AA?9?$AAg?$AAr?$AA?$AA@ 100048ac     libucrt:lcidtoname_downlevel.obj
 0001:000038b8       ??_C@_1M@GMPONJN@?$AAe?$AAn?$AA?9?$AAa?$AAu?$AA?$AA@ 100048b8     libucrt:lcidtoname_downlevel.obj
 0001:000038c4       ??_C@_1M@NIDIIPGF@?$AAe?$AAn?$AA?9?$AAb?$AAz?$AA?$AA@ 100048c4     libucrt:lcidtoname_downlevel.obj
 0001:000038d0       ??_C@_1M@JEHMIMFO@?$AAe?$AAn?$AA?9?$AAc?$AAa?$AA?$AA@ 100048d0     libucrt:lcidtoname_downlevel.obj
 0001:000038dc       ??_C@_1M@IGMJCDLA@?$AAe?$AAn?$AA?9?$AAc?$AAb?$AA?$AA@ 100048dc     libucrt:lcidtoname_downlevel.obj
 0001:000038e8       ??_C@_1M@BNFIGBKG@?$AAe?$AAn?$AA?9?$AAg?$AAb?$AA?$AA@ 100048e8     libucrt:lcidtoname_downlevel.obj
 0001:000038f4       ??_C@_1M@LKIFDIGP@?$AAe?$AAn?$AA?9?$AAi?$AAe?$AA?$AA@ 100048f4     libucrt:lcidtoname_downlevel.obj
 0001:00003900       ??_C@_1M@PJKFGCCO@?$AAe?$AAn?$AA?9?$AAj?$AAm?$AA?$AA@ 10004900     libucrt:lcidtoname_downlevel.obj
 0001:0000390c       ??_C@_1M@KPPKEPBO@?$AAe?$AAn?$AA?9?$AAn?$AAz?$AA?$AA@ 1000490c     libucrt:lcidtoname_downlevel.obj
 0001:00003918       ??_C@_1M@GMDGLDOB@?$AAe?$AAn?$AA?9?$AAp?$AAh?$AA?$AA@ 10004918     libucrt:lcidtoname_downlevel.obj
 0001:00003924       ??_C@_1M@ONGIBJNA@?$AAe?$AAn?$AA?9?$AAt?$AAt?$AA?$AA@ 10004924     libucrt:lcidtoname_downlevel.obj
 0001:00003930       ??_C@_1M@LLODPCMM@?$AAe?$AAn?$AA?9?$AAu?$AAs?$AA?$AA@ 10004930     libucrt:lcidtoname_downlevel.obj
 0001:0000393c       ??_C@_1M@LAKFNPAN@?$AAe?$AAn?$AA?9?$AAz?$AAa?$AA?$AA@ 1000493c     libucrt:lcidtoname_downlevel.obj
 0001:00003948       ??_C@_1M@MFNHNHEO@?$AAe?$AAn?$AA?9?$AAz?$AAw?$AA?$AA@ 10004948     libucrt:lcidtoname_downlevel.obj
 0001:00003954       ??_C@_1M@EJEINPHM@?$AAe?$AAs?$AA?9?$AAa?$AAr?$AA?$AA@ 10004954     libucrt:lcidtoname_downlevel.obj
 0001:00003960       ??_C@_1M@GNKPCCJA@?$AAe?$AAs?$AA?9?$AAb?$AAo?$AA?$AA@ 10004960     libucrt:lcidtoname_downlevel.obj
 0001:0000396c       ??_C@_1M@LEEGFONL@?$AAe?$AAs?$AA?9?$AAc?$AAl?$AA?$AA@ 1000496c     libucrt:lcidtoname_downlevel.obj
 0001:00003978       ??_C@_1M@KGPDPBDF@?$AAe?$AAs?$AA?9?$AAc?$AAo?$AA?$AA@ 10004978     libucrt:lcidtoname_downlevel.obj
 0001:00003984       ??_C@_1M@EIAHOHH@?$AAe?$AAs?$AA?9?$AAc?$AAr?$AA?$AA@ 10004984     libucrt:lcidtoname_downlevel.obj
 0001:00003990       ??_C@_1M@LLPGMBIN@?$AAe?$AAs?$AA?9?$AAd?$AAo?$AA?$AA@ 10004990     libucrt:lcidtoname_downlevel.obj
 0001:0000399c       ??_C@_1M@DKHMKNJA@?$AAe?$AAs?$AA?9?$AAe?$AAc?$AA?$AA@ 1000499c     libucrt:lcidtoname_downlevel.obj
 0001:000039a8       ??_C@_1M@GKGFPKAP@?$AAe?$AAs?$AA?9?$AAe?$AAs?$AA?$AA@ 100049a8     libucrt:lcidtoname_downlevel.obj
 0001:000039b4       ??_C@_1M@LKHKGDLN@?$AAe?$AAs?$AA?9?$AAg?$AAt?$AA?$AA@ 100049b4     libucrt:lcidtoname_downlevel.obj
 0001:000039c0       ??_C@_1M@HEIIGGJD@?$AAe?$AAs?$AA?9?$AAh?$AAn?$AA?$AA@ 100049c0     libucrt:lcidtoname_downlevel.obj
 0001:000039cc       ??_C@_1M@FBDHPPGD@?$AAe?$AAs?$AA?9?$AAm?$AAx?$AA?$AA@ 100049cc     libucrt:lcidtoname_downlevel.obj
 0001:000039d8       ??_C@_1M@DPAGLNDH@?$AAe?$AAs?$AA?9?$AAn?$AAi?$AA?$AA@ 100049d8     libucrt:lcidtoname_downlevel.obj
 0001:000039e4       ??_C@_1M@MDGOPGDD@?$AAe?$AAs?$AA?9?$AAp?$AAa?$AA?$AA@ 100049e4     libucrt:lcidtoname_downlevel.obj
 0001:000039f0       ??_C@_1M@EMAMGBGE@?$AAe?$AAs?$AA?9?$AAp?$AAe?$AA?$AA@ 100049f0     libucrt:lcidtoname_downlevel.obj
 0001:000039fc       ??_C@_1M@IBMCAOEC@?$AAe?$AAs?$AA?9?$AAp?$AAr?$AA?$AA@ 100049fc     libucrt:lcidtoname_downlevel.obj
 0001:00003a08       ??_C@_1M@FGMDIJED@?$AAe?$AAs?$AA?9?$AAp?$AAy?$AA?$AA@ 10004a08     libucrt:lcidtoname_downlevel.obj
 0001:00003a14       ??_C@_1M@IIDEOLLL@?$AAe?$AAs?$AA?9?$AAs?$AAv?$AA?$AA@ 10004a14     libucrt:lcidtoname_downlevel.obj
 0001:00003a20       ??_C@_1M@GAOBIPA@?$AAe?$AAs?$AA?9?$AAu?$AAy?$AA?$AA@ 10004a20     libucrt:lcidtoname_downlevel.obj
 0001:00003a2c       ??_C@_1M@JKFFICHJ@?$AAe?$AAs?$AA?9?$AAv?$AAe?$AA?$AA@ 10004a2c     libucrt:lcidtoname_downlevel.obj
 0001:00003a38       ??_C@_1M@PNMLOJDF@?$AAe?$AAt?$AA?9?$AAe?$AAe?$AA?$AA@ 10004a38     libucrt:lcidtoname_downlevel.obj
 0001:00003a44       ??_C@_1M@GHHLIKEI@?$AAe?$AAu?$AA?9?$AAe?$AAs?$AA?$AA@ 10004a44     libucrt:lcidtoname_downlevel.obj
 0001:00003a50       ??_C@_1M@PBNONODE@?$AAf?$AAa?$AA?9?$AAi?$AAr?$AA?$AA@ 10004a50     libucrt:lcidtoname_downlevel.obj
 0001:00003a5c       ??_C@_1M@JEEHPMIL@?$AAf?$AAi?$AA?9?$AAf?$AAi?$AA?$AA@ 10004a5c     libucrt:lcidtoname_downlevel.obj
 0001:00003a68       ??_C@_1M@LMDCNDBA@?$AAf?$AAo?$AA?9?$AAf?$AAo?$AA?$AA@ 10004a68     libucrt:lcidtoname_downlevel.obj
 0001:00003a74       ??_C@_1M@JKEOHLDK@?$AAf?$AAr?$AA?9?$AAb?$AAe?$AA?$AA@ 10004a74     libucrt:lcidtoname_downlevel.obj
 0001:00003a80       ??_C@_1M@NOHADPMI@?$AAf?$AAr?$AA?9?$AAc?$AAa?$AA?$AA@ 10004a80     libucrt:lcidtoname_downlevel.obj
 0001:00003a8c       ??_C@_1M@KDHIHAEC@?$AAf?$AAr?$AA?9?$AAc?$AAh?$AA?$AA@ 10004a8c     libucrt:lcidtoname_downlevel.obj
 0001:00003a98       ??_C@_1M@MMBBFGAK@?$AAf?$AAr?$AA?9?$AAf?$AAr?$AA?$AA@ 10004a98     libucrt:lcidtoname_downlevel.obj
 0001:00003aa4       ??_C@_1M@PAFNENNF@?$AAf?$AAr?$AA?9?$AAl?$AAu?$AA?$AA@ 10004aa4     libucrt:lcidtoname_downlevel.obj
 0001:00003ab0       ??_C@_1M@EOHDJGDD@?$AAf?$AAr?$AA?9?$AAm?$AAc?$AA?$AA@ 10004ab0     libucrt:lcidtoname_downlevel.obj
 0001:00003abc       ??_C@_1M@FAPLLOPF@?$AAg?$AAl?$AA?9?$AAe?$AAs?$AA?$AA@ 10004abc     libucrt:lcidtoname_downlevel.obj
 0001:00003ac8       ??_C@_1M@FOPBFLOO@?$AAg?$AAu?$AA?9?$AAi?$AAn?$AA?$AA@ 10004ac8     libucrt:lcidtoname_downlevel.obj
 0001:00003ad4       ??_C@_1M@KBMCINPM@?$AAh?$AAe?$AA?9?$AAi?$AAl?$AA?$AA@ 10004ad4     libucrt:lcidtoname_downlevel.obj
 0001:00003ae0       ??_C@_1M@BBPHKFPJ@?$AAh?$AAi?$AA?9?$AAi?$AAn?$AA?$AA@ 10004ae0     libucrt:lcidtoname_downlevel.obj
 0001:00003aec       ??_C@_1M@PMBNDPHD@?$AAh?$AAr?$AA?9?$AAb?$AAa?$AA?$AA@ 10004aec     libucrt:lcidtoname_downlevel.obj
 0001:00003af8       ??_C@_1M@BPCKOEGE@?$AAh?$AAr?$AA?9?$AAh?$AAr?$AA?$AA@ 10004af8     libucrt:lcidtoname_downlevel.obj
 0001:00003b04       ??_C@_1M@GACBMHKE@?$AAh?$AAu?$AA?9?$AAh?$AAu?$AA?$AA@ 10004b04     libucrt:lcidtoname_downlevel.obj
 0001:00003b10       ??_C@_1M@MILPAJJC@?$AAh?$AAy?$AA?9?$AAa?$AAm?$AA?$AA@ 10004b10     libucrt:lcidtoname_downlevel.obj
 0001:00003b1c       ??_C@_1M@BABBICEC@?$AAi?$AAd?$AA?9?$AAi?$AAd?$AA?$AA@ 10004b1c     libucrt:lcidtoname_downlevel.obj
 0001:00003b28       ??_C@_1M@BIKNHHPF@?$AAi?$AAs?$AA?9?$AAi?$AAs?$AA?$AA@ 10004b28     libucrt:lcidtoname_downlevel.obj
 0001:00003b34       ??_C@_1M@NMPCJPHE@?$AAi?$AAt?$AA?9?$AAc?$AAh?$AA?$AA@ 10004b34     libucrt:lcidtoname_downlevel.obj
 0001:00003b40       ??_C@_1M@GHKGFEDF@?$AAi?$AAt?$AA?9?$AAi?$AAt?$AA?$AA@ 10004b40     libucrt:lcidtoname_downlevel.obj
 0001:00003b4c       ??_C@_1M@NIEJCJJA@?$AAj?$AAa?$AA?9?$AAj?$AAp?$AA?$AA@ 10004b4c     libucrt:lcidtoname_downlevel.obj
 0001:00003b58       ??_C@_1M@JILFNBIM@?$AAk?$AAa?$AA?9?$AAg?$AAe?$AA?$AA@ 10004b58     libucrt:lcidtoname_downlevel.obj
 0001:00003b64       ??_C@_1M@PACPMGPH@?$AAk?$AAk?$AA?9?$AAk?$AAz?$AA?$AA@ 10004b64     libucrt:lcidtoname_downlevel.obj
 0001:00003b70       ??_C@_1M@IELFGMHA@?$AAk?$AAn?$AA?9?$AAi?$AAn?$AA?$AA@ 10004b70     libucrt:lcidtoname_downlevel.obj
 0001:00003b7c       ??_C@_1O@IBBJHCH@?$AAk?$AAo?$AAk?$AA?9?$AAi?$AAn?$AA?$AA@ 10004b7c     libucrt:lcidtoname_downlevel.obj
 0001:00003b8c       ??_C@_1M@DMHAEOGC@?$AAk?$AAo?$AA?9?$AAk?$AAr?$AA?$AA@ 10004b8c     libucrt:lcidtoname_downlevel.obj
 0001:00003b98       ??_C@_1M@HBAHBIGA@?$AAk?$AAy?$AA?9?$AAk?$AAg?$AA?$AA@ 10004b98     libucrt:lcidtoname_downlevel.obj
 0001:00003ba4       ??_C@_1M@KPMILCJG@?$AAl?$AAt?$AA?9?$AAl?$AAt?$AA?$AA@ 10004ba4     libucrt:lcidtoname_downlevel.obj
 0001:00003bb0       ??_C@_1M@BDEKKCA@?$AAl?$AAv?$AA?9?$AAl?$AAv?$AA?$AA@ 10004bb0     libucrt:lcidtoname_downlevel.obj
 0001:00003bbc       ??_C@_1M@ELCKCCJJ@?$AAm?$AAi?$AA?9?$AAn?$AAz?$AA?$AA@ 10004bbc     libucrt:lcidtoname_downlevel.obj
 0001:00003bc8       ??_C@_1M@CBOOLAPA@?$AAm?$AAk?$AA?9?$AAm?$AAk?$AA?$AA@ 10004bc8     libucrt:lcidtoname_downlevel.obj
 0001:00003bd4       ??_C@_1M@GPHNBJKN@?$AAm?$AAl?$AA?9?$AAi?$AAn?$AA?$AA@ 10004bd4     libucrt:lcidtoname_downlevel.obj
 0001:00003be0       ??_C@_1M@PABJILIG@?$AAm?$AAn?$AA?9?$AAm?$AAn?$AA?$AA@ 10004be0     libucrt:lcidtoname_downlevel.obj
 0001:00003bec       ??_C@_1M@FGBKKIPG@?$AAm?$AAr?$AA?9?$AAi?$AAn?$AA?$AA@ 10004bec     libucrt:lcidtoname_downlevel.obj
 0001:00003bf8       ??_C@_1M@NDBPDDAL@?$AAm?$AAs?$AA?9?$AAb?$AAn?$AA?$AA@ 10004bf8     libucrt:lcidtoname_downlevel.obj
 0001:00003c04       ??_C@_1M@OPIHOOPI@?$AAm?$AAs?$AA?9?$AAm?$AAy?$AA?$AA@ 10004c04     libucrt:lcidtoname_downlevel.obj
 0001:00003c10       ??_C@_1M@PPDBCNFM@?$AAm?$AAt?$AA?9?$AAm?$AAt?$AA?$AA@ 10004c10     libucrt:lcidtoname_downlevel.obj
 0001:00003c1c       ??_C@_1M@KDJDKMDD@?$AAn?$AAb?$AA?9?$AAn?$AAo?$AA?$AA@ 10004c1c     libucrt:lcidtoname_downlevel.obj
 0001:00003c28       ??_C@_1M@KFCFLMJP@?$AAn?$AAl?$AA?9?$AAb?$AAe?$AA?$AA@ 10004c28     libucrt:lcidtoname_downlevel.obj
 0001:00003c34       ??_C@_1M@KPOPDDGO@?$AAn?$AAl?$AA?9?$AAn?$AAl?$AA?$AA@ 10004c34     libucrt:lcidtoname_downlevel.obj
 0001:00003c40       ??_C@_1M@LJKPEMLN@?$AAn?$AAn?$AA?9?$AAn?$AAo?$AA?$AA@ 10004c40     libucrt:lcidtoname_downlevel.obj
 0001:00003c4c       ??_C@_1M@BDGHHBFL@?$AAn?$AAs?$AA?9?$AAz?$AAa?$AA?$AA@ 10004c4c     libucrt:lcidtoname_downlevel.obj
 0001:00003c58       ??_C@_1M@IDEHOAP@?$AAp?$AAa?$AA?9?$AAi?$AAn?$AA?$AA@ 10004c58     libucrt:lcidtoname_downlevel.obj
 0001:00003c64       ??_C@_1M@HDBKGOGH@?$AAp?$AAl?$AA?9?$AAp?$AAl?$AA?$AA@ 10004c64     libucrt:lcidtoname_downlevel.obj
 0001:00003c70       ??_C@_1M@LJLLCMEH@?$AAp?$AAt?$AA?9?$AAb?$AAr?$AA?$AA@ 10004c70     libucrt:lcidtoname_downlevel.obj
 0001:00003c7c       ??_C@_1M@NCMONAAL@?$AAp?$AAt?$AA?9?$AAp?$AAt?$AA?$AA@ 10004c7c     libucrt:lcidtoname_downlevel.obj
 0001:00003c88       ??_C@_1O@EAKMAJDN@?$AAq?$AAu?$AAz?$AA?9?$AAb?$AAo?$AA?$AA@ 10004c88     libucrt:lcidtoname_downlevel.obj
 0001:00003c98       ??_C@_1O@BHHPIGDN@?$AAq?$AAu?$AAz?$AA?9?$AAe?$AAc?$AA?$AA@ 10004c98     libucrt:lcidtoname_downlevel.obj
 0001:00003ca8       ??_C@_1O@GBAPEKMJ@?$AAq?$AAu?$AAz?$AA?9?$AAp?$AAe?$AA?$AA@ 10004ca8     libucrt:lcidtoname_downlevel.obj
 0001:00003cb8       ??_C@_1M@CLGLEFBO@?$AAr?$AAo?$AA?9?$AAr?$AAo?$AA?$AA@ 10004cb8     libucrt:lcidtoname_downlevel.obj
 0001:00003cc4       ??_C@_1M@CEEDODME@?$AAr?$AAu?$AA?9?$AAr?$AAu?$AA?$AA@ 10004cc4     libucrt:lcidtoname_downlevel.obj
 0001:00003cd0       ??_C@_1M@HPKKKMPP@?$AAs?$AAa?$AA?9?$AAi?$AAn?$AA?$AA@ 10004cd0     libucrt:lcidtoname_downlevel.obj
 0001:00003cdc       ??_C@_1M@BKMAIGOJ@?$AAs?$AAe?$AA?9?$AAf?$AAi?$AA?$AA@ 10004cdc     libucrt:lcidtoname_downlevel.obj
 0001:00003ce8       ??_C@_1M@NDPIFLFI@?$AAs?$AAe?$AA?9?$AAn?$AAo?$AA?$AA@ 10004ce8     libucrt:lcidtoname_downlevel.obj
 0001:00003cf4       ??_C@_1M@DANKKHJ@?$AAs?$AAe?$AA?9?$AAs?$AAe?$AA?$AA@ 10004cf4     libucrt:lcidtoname_downlevel.obj
 0001:00003d00       ??_C@_1M@PNBLONPJ@?$AAs?$AAk?$AA?9?$AAs?$AAk?$AA?$AA@ 10004d00     libucrt:lcidtoname_downlevel.obj
 0001:00003d0c       ??_C@_1M@LFMODOAL@?$AAs?$AAl?$AA?9?$AAs?$AAi?$AA?$AA@ 10004d0c     libucrt:lcidtoname_downlevel.obj
 0001:00003d18       ??_C@_1O@DFKOMPG@?$AAs?$AAm?$AAa?$AA?9?$AAn?$AAo?$AA?$AA@ 10004d18     libucrt:lcidtoname_downlevel.obj
 0001:00003d28       ??_C@_1O@NDKPBNNH@?$AAs?$AAm?$AAa?$AA?9?$AAs?$AAe?$AA?$AA@ 10004d28     libucrt:lcidtoname_downlevel.obj
 0001:00003d38       ??_C@_1O@PLLKBHAB@?$AAs?$AAm?$AAj?$AA?9?$AAn?$AAo?$AA?$AA@ 10004d38     libucrt:lcidtoname_downlevel.obj
 0001:00003d48       ??_C@_1O@CLEPOGCA@?$AAs?$AAm?$AAj?$AA?9?$AAs?$AAe?$AA?$AA@ 10004d48     libucrt:lcidtoname_downlevel.obj
 0001:00003d58       ??_C@_1O@DLGJGKMK@?$AAs?$AAm?$AAn?$AA?9?$AAf?$AAi?$AA?$AA@ 10004d58     libucrt:lcidtoname_downlevel.obj
 0001:00003d68       ??_C@_1O@OJDJGAJC@?$AAs?$AAm?$AAs?$AA?9?$AAf?$AAi?$AA?$AA@ 10004d68     libucrt:lcidtoname_downlevel.obj
 0001:00003d78       ??_C@_1M@BOFOGHPB@?$AAs?$AAq?$AA?9?$AAa?$AAl?$AA?$AA@ 10004d78     libucrt:lcidtoname_downlevel.obj
 0001:00003d84       ??_C@_1BG@LJBBIPGB@?$AAs?$AAr?$AA?9?$AAb?$AAa?$AA?9?$AAc?$AAy?$AAr?$AAl?$AA?$AA@ 10004d84     libucrt:lcidtoname_downlevel.obj
 0001:00003d9c       ??_C@_1BG@JLBENFOE@?$AAs?$AAr?$AA?9?$AAb?$AAa?$AA?9?$AAl?$AAa?$AAt?$AAn?$AA?$AA@ 10004d9c     libucrt:lcidtoname_downlevel.obj
 0001:00003db4       ??_C@_1BG@KODPNHE@?$AAs?$AAr?$AA?9?$AAs?$AAp?$AA?9?$AAc?$AAy?$AAr?$AAl?$AA?$AA@ 10004db4     libucrt:lcidtoname_downlevel.obj
 0001:00003dcc       ??_C@_1BG@CIOGKHPB@?$AAs?$AAr?$AA?9?$AAs?$AAp?$AA?9?$AAl?$AAa?$AAt?$AAn?$AA?$AA@ 10004dcc     libucrt:lcidtoname_downlevel.obj
 0001:00003de4       ??_C@_1M@NGFJLMAC@?$AAs?$AAv?$AA?9?$AAf?$AAi?$AA?$AA@ 10004de4     libucrt:lcidtoname_downlevel.obj
 0001:00003df0       ??_C@_1M@MPJEJAJC@?$AAs?$AAv?$AA?9?$AAs?$AAe?$AA?$AA@ 10004df0     libucrt:lcidtoname_downlevel.obj
 0001:00003dfc       ??_C@_1M@MPNDHLFK@?$AAs?$AAw?$AA?9?$AAk?$AAe?$AA?$AA@ 10004dfc     libucrt:lcidtoname_downlevel.obj
 0001:00003e08       ??_C@_1O@KOHBJJI@?$AAs?$AAy?$AAr?$AA?9?$AAs?$AAy?$AA?$AA@ 10004e08     libucrt:lcidtoname_downlevel.obj
 0001:00003e18       ??_C@_1M@LDCEFHA@?$AAt?$AAa?$AA?9?$AAi?$AAn?$AA?$AA@ 10004e18     libucrt:lcidtoname_downlevel.obj
 0001:00003e24       ??_C@_1M@CNJOFAK@?$AAt?$AAe?$AA?9?$AAi?$AAn?$AA?$AA@ 10004e24     libucrt:lcidtoname_downlevel.obj
 0001:00003e30       ??_C@_1M@GNAECACD@?$AAt?$AAh?$AA?9?$AAt?$AAh?$AA?$AA@ 10004e30     libucrt:lcidtoname_downlevel.obj
 0001:00003e3c       ??_C@_1M@CHBIHOJO@?$AAt?$AAn?$AA?9?$AAz?$AAa?$AA?$AA@ 10004e3c     libucrt:lcidtoname_downlevel.obj
 0001:00003e48       ??_C@_1M@GCCMIGPJ@?$AAt?$AAr?$AA?9?$AAt?$AAr?$AA?$AA@ 10004e48     libucrt:lcidtoname_downlevel.obj
 0001:00003e54       ??_C@_1M@CELMCNBK@?$AAt?$AAt?$AA?9?$AAr?$AAu?$AA?$AA@ 10004e54     libucrt:lcidtoname_downlevel.obj
 0001:00003e60       ??_C@_1M@KLMCELGA@?$AAu?$AAk?$AA?9?$AAu?$AAa?$AA?$AA@ 10004e60     libucrt:lcidtoname_downlevel.obj
 0001:00003e6c       ??_C@_1M@EPAJJAJF@?$AAu?$AAr?$AA?9?$AAp?$AAk?$AA?$AA@ 10004e6c     libucrt:lcidtoname_downlevel.obj
 0001:00003e78       ??_C@_1BG@GEGPMCDJ@?$AAu?$AAz?$AA?9?$AAu?$AAz?$AA?9?$AAc?$AAy?$AAr?$AAl?$AA?$AA@ 10004e78     libucrt:lcidtoname_downlevel.obj
 0001:00003e90       ??_C@_1BG@EGGKJILM@?$AAu?$AAz?$AA?9?$AAu?$AAz?$AA?9?$AAl?$AAa?$AAt?$AAn?$AA?$AA@ 10004e90     libucrt:lcidtoname_downlevel.obj
 0001:00003ea8       ??_C@_1M@GFOCLFF@?$AAv?$AAi?$AA?9?$AAv?$AAn?$AA?$AA@ 10004ea8     libucrt:lcidtoname_downlevel.obj
 0001:00003eb4       ??_C@_1M@CPAMEDFI@?$AAx?$AAh?$AA?9?$AAz?$AAa?$AA?$AA@ 10004eb4     libucrt:lcidtoname_downlevel.obj
 0001:00003ec0       ??_C@_1O@EBKIFIGN@?$AAz?$AAh?$AA?9?$AAc?$AAh?$AAs?$AA?$AA@ 10004ec0     libucrt:lcidtoname_downlevel.obj
 0001:00003ed0       ??_C@_1O@NMHPGANE@?$AAz?$AAh?$AA?9?$AAc?$AAh?$AAt?$AA?$AA@ 10004ed0     libucrt:lcidtoname_downlevel.obj
 0001:00003ee0       ??_C@_1M@LPINJOMC@?$AAz?$AAh?$AA?9?$AAc?$AAn?$AA?$AA@ 10004ee0     libucrt:lcidtoname_downlevel.obj
 0001:00003eec       ??_C@_1M@OCJEJODD@?$AAz?$AAh?$AA?9?$AAh?$AAk?$AA?$AA@ 10004eec     libucrt:lcidtoname_downlevel.obj
 0001:00003ef8       ??_C@_1M@DNDLJINH@?$AAz?$AAh?$AA?9?$AAm?$AAo?$AA?$AA@ 10004ef8     libucrt:lcidtoname_downlevel.obj
 0001:00003f04       ??_C@_1M@MBFDNDND@?$AAz?$AAh?$AA?9?$AAs?$AAg?$AA?$AA@ 10004f04     libucrt:lcidtoname_downlevel.obj
 0001:00003f10       ??_C@_1M@IMEPLEPE@?$AAz?$AAh?$AA?9?$AAt?$AAw?$AA?$AA@ 10004f10     libucrt:lcidtoname_downlevel.obj
 0001:00003f1c       ??_C@_1M@BBGHNHJP@?$AAz?$AAu?$AA?9?$AAz?$AAa?$AA?$AA@ 10004f1c     libucrt:lcidtoname_downlevel.obj
 0001:00004090       __infinity                 10005090     libucrt:87tran.obj
 0001:0000409a       __minfinity                1000509a     libucrt:87tran.obj
 0001:000040a4       __logemax                  100050a4     libucrt:87tran.obj
 0001:000040ca       __OP_EXPjmptab             100050ca     libucrt:87tran.obj
 0001:000040f0       __indefinite               100050f0     libucrt:87disp.obj
 0001:000040fa       __piby2                    100050fa     libucrt:87disp.obj
 0001:00004104       __piby4                    10005104     libucrt:87disp.obj
 0001:00004138       __DEFAULT_CW_in_mem        10005138     libucrt:common.obj
 0001:0000413a       __pi_by_2_to_61            1000513a     libucrt:common.obj
 0001:00004174       ??_C@_03MGHMBJCF@log?$AA@  10005174     libucrt:libm_error.obj
 0001:00004178       ??_C@_05HGHHAHAP@log10?$AA@ 10005178     libucrt:libm_error.obj
 0001:00004180       ??_C@_03KHJOGHMM@exp?$AA@  10005180     libucrt:libm_error.obj
 0001:00004184       ??_C@_03JGHBODFD@pow?$AA@  10005184     libucrt:libm_error.obj
 0001:00004188       ??_C@_04FIHNOPOL@asin?$AA@ 10005188     libucrt:libm_error.obj
 0001:00004190       ??_C@_04PDIFKINK@acos?$AA@ 10005190     libucrt:libm_error.obj
 0001:00004198       ??_C@_04EIAKFFMI@sqrt?$AA@ 10005198     libucrt:libm_error.obj
 0001:000041a0       __real@3ff0000000000000    100051a0     libucrt:libm_error.obj
 0001:000041a8       ??_C@_1BA@BALFACEM@?$AAC?$AAO?$AAN?$AAO?$AAU?$AAT?$AA$?$AA?$AA@ 100051a8     libucrt:initcon.obj
 0001:000041d0       ___acrt_log10_table_t      100051d0     libucrt:log10_tables.obj
 0001:000045e0       ___acrt_log10_table_cb     100055e0     libucrt:log10_tables.obj
 0001:000049f0       __real@3fe0000000000000    100059f0     libucrt:powhlp.obj
 0001:000049f8       ??_C@_04FJHINJAO@tanh?$AA@ 100059f8     libucrt:fpexcept.obj
 0001:00004a00       ??_C@_04MLLJIGOK@atan?$AA@ 10005a00     libucrt:fpexcept.obj
 0001:00004a08       ??_C@_05KNGEOGJB@atan2?$AA@ 10005a08     libucrt:fpexcept.obj
 0001:00004a10       ??_C@_03BLEJJJBH@sin?$AA@  10005a10     libucrt:fpexcept.obj
 0001:00004a14       ??_C@_03LALBNOCG@cos?$AA@  10005a14     libucrt:fpexcept.obj
 0001:00004a18       ??_C@_03IIINPABG@tan?$AA@  10005a18     libucrt:fpexcept.obj
 0001:00004a1c       ??_C@_04GFPJNGEK@ceil?$AA@ 10005a1c     libucrt:fpexcept.obj
 0001:00004a24       ??_C@_05PBJFFIGL@floor?$AA@ 10005a24     libucrt:fpexcept.obj
 0001:00004a2c       ??_C@_04ODHECPBC@fabs?$AA@ 10005a2c     libucrt:fpexcept.obj
 0001:00004a34       ??_C@_04EHEDPDJG@modf?$AA@ 10005a34     libucrt:fpexcept.obj
 0001:00004a3c       ??_C@_05CEJMAHNP@ldexp?$AA@ 10005a3c     libucrt:fpexcept.obj
 0001:00004a44       ??_C@_05KBKMEMPO@_cabs?$AA@ 10005a44     libucrt:fpexcept.obj
 0001:00004a4c       ??_C@_06MEIMCGCF@_hypot?$AA@ 10005a4c     libucrt:fpexcept.obj
 0001:00004a54       ??_C@_04KEPJIHGP@fmod?$AA@ 10005a54     libucrt:fpexcept.obj
 0001:00004a5c       ??_C@_05GKKHEGJL@frexp?$AA@ 10005a5c     libucrt:fpexcept.obj
 0001:00004a64       ??_C@_03MJLDFKDL@_y0?$AA@  10005a64     libucrt:fpexcept.obj
 0001:00004a68       ??_C@_03NAKIGLHK@_y1?$AA@  10005a68     libucrt:fpexcept.obj
 0001:00004a6c       ??_C@_03ONILCKOB@_yn?$AA@  10005a6c     libucrt:fpexcept.obj
 0001:00004a70       ??_C@_05JGDBENOH@_logb?$AA@ 10005a70     libucrt:fpexcept.obj
 0001:00004a78       ??_C@_0L@KDOEJCKC@_nextafter?$AA@ 10005a78     libucrt:fpexcept.obj
 0001:00004b70       ??_C@_04COOMCNPB@sinh?$AA@ 10005b70     libucrt:fpexcept.obj
 0001:00004b78       ??_C@_04HPJJNFIM@cosh?$AA@ 10005b78     libucrt:fpexcept.obj
 0001:00004b80       __d_inf                    10005b80     libucrt:util.obj
 0001:00004b88       __d_max                    10005b88     libucrt:util.obj
 0001:00004b90       __d_mzero                  10005b90     libucrt:util.obj
 0001:00004bc0       __load_config_used         10005bc0     LIBCMT:loadcfg.obj
 0001:00004c1c       ??_R4exception@std@@6B@    10005c1c     LIBCMT:throw_bad_alloc.obj
 0001:00004c30       ??_R3exception@std@@8      10005c30     LIBCMT:throw_bad_alloc.obj
 0001:00004c40       ??_R2exception@std@@8      10005c40     LIBCMT:throw_bad_alloc.obj
 0001:00004c48       ??_R1A@?0A@EA@exception@std@@8 10005c48     LIBCMT:throw_bad_alloc.obj
 0001:00004c64       ??_R4bad_alloc@std@@6B@    10005c64     LIBCMT:throw_bad_alloc.obj
 0001:00004c78       ??_R3bad_alloc@std@@8      10005c78     LIBCMT:throw_bad_alloc.obj
 0001:00004c88       ??_R2bad_alloc@std@@8      10005c88     LIBCMT:throw_bad_alloc.obj
 0001:00004c94       ??_R1A@?0A@EA@bad_alloc@std@@8 10005c94     LIBCMT:throw_bad_alloc.obj
 0001:00004cb0       ??_R4bad_array_new_length@std@@6B@ 10005cb0     LIBCMT:throw_bad_alloc.obj
 0001:00004cc4       ??_R3bad_array_new_length@std@@8 10005cc4     LIBCMT:throw_bad_alloc.obj
 0001:00004cd4       ??_R2bad_array_new_length@std@@8 10005cd4     LIBCMT:throw_bad_alloc.obj
 0001:00004ce4       ??_R1A@?0A@EA@bad_array_new_length@std@@8 10005ce4     LIBCMT:throw_bad_alloc.obj
 0001:00004d00       ??_R4type_info@@6B@        10005d00     LIBCMT:std_type_info_static.obj
 0001:00004d14       ??_R3type_info@@8          10005d14     LIBCMT:std_type_info_static.obj
 0001:00004d24       ??_R2type_info@@8          10005d24     LIBCMT:std_type_info_static.obj
 0001:00004d2c       ??_R1A@?0A@EA@type_info@@8 10005d2c     LIBCMT:std_type_info_static.obj
 0001:00004d50       ___safe_se_handler_table   10005d50     <linker-defined>
 0001:0000500c       ___rtc_iaa                 1000600c     LIBCMT:_initsect_.obj
 0001:00005010       ___rtc_izz                 10006010     LIBCMT:_initsect_.obj
 0001:00005014       ___rtc_taa                 10006014     LIBCMT:_initsect_.obj
 0001:00005018       ___rtc_tzz                 10006018     LIBCMT:_initsect_.obj
 0001:00005020       __chkstk                   10006020 f   chkstk.obj
 0001:00005020       __alloca_probe             10006020 f   chkstk.obj
 0001:00005050       ??0?$DialogBuilderBase@UFarDialogItem@@@@IAE@XZ 10006050 f i Align.obj
 0001:000050c0       ??0PluginDialogBuilder@@QAE@ABUPluginStartupInfo@@ABU_GUID@@1HPB_WP6GHPAXHH3@Z3_K@Z 100060c0 f i Align.obj
 0001:000051a0       ??0PluginIntEditFieldBinding@@QAE@ABUPluginStartupInfo@@PAPAXHPAHH@Z 100061a0 f i Align.obj
 0001:00005240       ??0PluginUIntEditFieldBinding@@QAE@ABUPluginStartupInfo@@PAPAXHPAIH@Z 10006240 f i Align.obj
 0001:000052e0       ??1?$DialogBuilderBase@UFarDialogItem@@@@MAE@XZ 100062e0 f i Align.obj
 0001:00005320       ??_E?$DialogBuilderBase@UFarDialogItem@@@@MAEPAXI@Z 10006320 f i Align.obj
 0001:00005320       ??_G?$DialogBuilderBase@UFarDialogItem@@@@MAEPAXI@Z 10006320 f i Align.obj
 0001:00005340       ??_E?$DialogItemBinding@UFarDialogItem@@@@UAEPAXI@Z 10006340 f i Align.obj
 0001:00005340       ??_G?$DialogItemBinding@UFarDialogItem@@@@UAEPAXI@Z 10006340 f i Align.obj
 0001:00005370       ??_GPluginCheckBoxBinding@@UAEPAXI@Z 10006370 f i Align.obj
 0001:00005370       ??_EPluginCheckBoxBinding@@UAEPAXI@Z 10006370 f i Align.obj
 0001:000053a0       ??_EPluginDialogBuilder@@UAEPAXI@Z 100063a0 f i Align.obj
 0001:000053a0       ??_GPluginDialogBuilder@@UAEPAXI@Z 100063a0 f i Align.obj
 0001:000053e0       ??_GPluginUIntEditFieldBinding@@UAEPAXI@Z 100063e0 f i Align.obj
 0001:000053e0       ??_EPluginIntEditFieldBinding@@UAEPAXI@Z 100063e0 f i Align.obj
 0001:000053e0       ??_EPluginUIntEditFieldBinding@@UAEPAXI@Z 100063e0 f i Align.obj
 0001:000053e0       ??_GPluginIntEditFieldBinding@@UAEPAXI@Z 100063e0 f i Align.obj
 0001:00005410       ??_EPluginRadioButtonBinding@@UAEPAXI@Z 10006410 f i Align.obj
 0001:00005410       ??_GPluginRadioButtonBinding@@UAEPAXI@Z 10006410 f i Align.obj
 0001:00005440       ?AddButtons@?$DialogBuilderBase@UFarDialogItem@@@@QAEXHPBHHH@Z 10006440 f i Align.obj
 0001:000055a0       ?AddIntEditField@PluginDialogBuilder@@UAEPAUFarDialogItem@@PAHH@Z 100065a0 f i Align.obj
 0001:00005660       ?AddSeparator@?$DialogBuilderBase@UFarDialogItem@@@@QAEXPB_W@Z 10006660 f i Align.obj
 0001:000056d0       ?AddTextAfter@?$DialogBuilderBase@UFarDialogItem@@@@QAEPAUFarDialogItem@@PAU2@PB_WH@Z 100066d0 f i Align.obj
 0001:00005770       ?AddIntEditField@?$DialogBuilderBase@UFarDialogItem@@@@UAEPAUFarDialogItem@@PAHH@Z 10006770 f i Align.obj
 0001:00005770       ?CreateCheckBoxBinding@?$DialogBuilderBase@UFarDialogItem@@@@MAEPAU?$DialogItemBinding@UFarDialogItem@@@@PAHH@Z 10006770 f i Align.obj
 0001:00005770       ?AddUIntEditField@?$DialogBuilderBase@UFarDialogItem@@@@UAEPAUFarDialogItem@@PAIH@Z 10006770 f i Align.obj
 0001:00005780       ?AddUIntEditField@PluginDialogBuilder@@UAEPAUFarDialogItem@@PAIH@Z 10006780 f i Align.obj
 0001:00005840       ?CreateCheckBoxBinding@PluginDialogBuilder@@MAEPAU?$DialogItemBinding@UFarDialogItem@@@@PAHH@Z 10006840 f i Align.obj
 0001:000058a0       ?CreateRadioButtonBinding@PluginDialogBuilder@@MAEPAU?$DialogItemBinding@UFarDialogItem@@@@PAH@Z 100068a0 f i Align.obj
 0001:000058f0       ?DoShowDialog@?$DialogBuilderBase@UFarDialogItem@@@@MAEHXZ 100068f0 f i Align.obj
 0001:00005900       ?DoShowDialog@PluginDialogBuilder@@MAEHXZ 10006900 f i Align.obj
 0001:00005950       ?GetLangString@?$DialogBuilderBase@UFarDialogItem@@@@MAEPB_WH@Z 10006950 f i Align.obj
 0001:00005950       ?CreateRadioButtonBinding@?$DialogBuilderBase@UFarDialogItem@@@@MAEPAU?$DialogItemBinding@UFarDialogItem@@@@PAH@Z 10006950 f i Align.obj
 0001:00005960       ?GetLangString@PluginDialogBuilder@@MAEPB_WH@Z 10006960 f i Align.obj
 0001:00005980       ?SaveValue@?$DialogItemBinding@UFarDialogItem@@@@UAEXPAUFarDialogItem@@H@Z 10006980 f i Align.obj
 0001:00005980       ?InitDialogItem@?$DialogBuilderBase@UFarDialogItem@@@@MAEXPAUFarDialogItem@@PB_W@Z 10006980 f i Align.obj
 0001:00005990       ?InitDialogItem@PluginDialogBuilder@@MAEXPAUFarDialogItem@@PB_W@Z 10006990 f i Align.obj
 0001:000059b0       ?ItemWidth@?$DialogBuilderBase@UFarDialogItem@@@@IAEHABUFarDialogItem@@@Z 100069b0 f i Align.obj
 0001:00005e50       ?MaxTextWidth@?$DialogBuilderBase@UFarDialogItem@@@@IAEHXZ 10006e50 f i Align.obj
 0001:00005f10       ?ReallocDialogItems@?$DialogBuilderBase@UFarDialogItem@@@@IAEXXZ 10006f10 f i Align.obj
 0001:00006650       ?SaveValue@PluginCheckBoxBinding@@UAEXPAUFarDialogItem@@H@Z 10007650 f i Align.obj
 0001:00006690       ?SaveValue@PluginIntEditFieldBinding@@UAEXPAUFarDialogItem@@H@Z 10007690 f i Align.obj
 0001:000066c0       ?SaveValue@PluginRadioButtonBinding@@UAEXPAUFarDialogItem@@H@Z 100076c0 f i Align.obj
 0001:000066f0       ?SaveValue@PluginUIntEditFieldBinding@@UAEXPAUFarDialogItem@@H@Z 100076f0 f i Align.obj
 0001:00006720       ?SaveValues@?$DialogBuilderBase@UFarDialogItem@@@@IAEXXZ 10007720 f i Align.obj
 0001:00006770       ?TextWidth@?$DialogBuilderBase@UFarDialogItem@@@@MAEHABUFarDialogItem@@@Z 10007770 f i Align.obj
 0001:00006780       ?TextWidth@PluginDialogBuilder@@MAEHABUFarDialogItem@@@Z 10007780 f i Align.obj
 0001:00006790       ?UpdateBorderSize@?$DialogBuilderBase@UFarDialogItem@@@@IAEXXZ 10007790 f i Align.obj
 0001:00006830       ?UpdateSecondColumnPosition@?$DialogBuilderBase@UFarDialogItem@@@@IAEXXZ 10007830 f i Align.obj
 0001:00006890       _GetGlobalInfoW@4          10007890 f   Align.obj
 0001:00006920       _GetPluginInfoW@4          10007920 f   Align.obj
 0001:00006970       _OpenW@4                   10007970 f   Align.obj
 0001:00006fa0       _SetStartupInfoW@4         10007fa0 f   Align.obj
 0001:00007060       _DecodePointerWrapper@4    10008060 f   vc_crt_fix_impl.obj
 0001:000070a0       _EncodePointerWrapper@4    100080a0 f   vc_crt_fix_impl.obj
 0001:000070e0       _GetModuleHandleExWWrapper@12 100080e0 f   vc_crt_fix_impl.obj
 0001:00007120       _InitializeSListHeadWrapper@4 10008120 f   vc_crt_fix_impl.obj
 0001:00007170       _InterlockedFlushSListWrapper@4 10008170 f   vc_crt_fix_impl.obj
 0001:000071b0       _InterlockedPopEntrySListWrapper@4 100081b0 f   vc_crt_fix_impl.obj
 0001:000071f0       _InterlockedPushEntrySListWrapper@8 100081f0 f   vc_crt_fix_impl.obj
 0001:00007230       _InterlockedPushListSListExWrapper@16 10008230 f   vc_crt_fix_impl.obj
 0001:00007270       _QueryDepthSListWrapper@4  10008270 f   vc_crt_fix_impl.obj
 0001:000072b0       _RtlFirstEntrySListWrapper@4 100082b0 f   vc_crt_fix_impl.obj
 0001:000072f0       ___vcrt_uninitialize_telemetry_provider 100082f0 f   vc_crt_fix_impl.obj
 0001:000072f0       ___telemetry_main_return_trigger 100082f0 f   vc_crt_fix_impl.obj
 0001:000072f0       ___telemetry_main_invoke_trigger 100082f0 f   vc_crt_fix_impl.obj
 0001:000072f0       ___except_validate_jump_buffer 100082f0 f   libvcruntime:jbcxrval.obj
 0001:000072f0       @_guard_check_icall_nop@4  100082f0 f   LIBCMT:guard_support.obj
 0001:000072f0       ___except_validate_context_record 100082f0 f   libvcruntime:jbcxrval.obj
 0001:000072f0       ___vcrt_initialize_telemetry_provider 100082f0 f   vc_crt_fix_impl.obj
 0001:000072f1       ??2@YAPAXI@Z               100082f1 f   LIBCMT:new_scalar.obj
 0001:00007324       ??3@YAXPAXI@Z              10008324 f   LIBCMT:delete_scalar_size.obj
 0001:00007332       ??_U@YAPAXI@Z              10008332 f   LIBCMT:new_array.obj
 0001:0000733b       ??_V@YAXPAX@Z              1000833b f   LIBCMT:delete_array.obj
 0001:00007668       __DllMainCRTStartup@12     10008668 f   LIBCMT:dll_dllmain.obj
 0001:0000768b       ??0bad_alloc@std@@QAE@ABV01@@Z 1000868b f i LIBCMT:throw_bad_alloc.obj
 0001:000076a6       ??0bad_alloc@std@@QAE@XZ   100086a6 f i LIBCMT:throw_bad_alloc.obj
 0001:000076be       ??0bad_array_new_length@std@@QAE@ABV01@@Z 100086be f i LIBCMT:throw_bad_alloc.obj
 0001:000076d9       ??0bad_array_new_length@std@@QAE@XZ 100086d9 f i LIBCMT:throw_bad_alloc.obj
 0001:000076f1       ??0exception@std@@QAE@ABV01@@Z 100086f1 f i LIBCMT:throw_bad_alloc.obj
 0001:0000771d       ??1bad_array_new_length@std@@UAE@XZ 1000871d f i LIBCMT:throw_bad_alloc.obj
 0001:0000771d       ??1bad_alloc@std@@UAE@XZ   1000871d f i LIBCMT:throw_bad_alloc.obj
 0001:0000772e       ??_Ebad_array_new_length@std@@UAEPAXI@Z 1000872e f i LIBCMT:throw_bad_alloc.obj
 0001:0000772e       ??_Eexception@std@@UAEPAXI@Z 1000872e f i LIBCMT:throw_bad_alloc.obj
 0001:0000772e       ??_Gexception@std@@UAEPAXI@Z 1000872e f i LIBCMT:throw_bad_alloc.obj
 0001:0000772e       ??_Ebad_alloc@std@@UAEPAXI@Z 1000872e f i LIBCMT:throw_bad_alloc.obj
 0001:0000772e       ??_Gbad_alloc@std@@UAEPAXI@Z 1000872e f i LIBCMT:throw_bad_alloc.obj
 0001:0000772e       ??_Gbad_array_new_length@std@@UAEPAXI@Z 1000872e f i LIBCMT:throw_bad_alloc.obj
 0001:0000775b       ?__scrt_throw_std_bad_alloc@@YAXXZ 1000875b f   LIBCMT:throw_bad_alloc.obj
 0001:00007778       ?__scrt_throw_std_bad_array_new_length@@YAXXZ 10008778 f   LIBCMT:throw_bad_alloc.obj
 0001:00007795       ?what@exception@std@@UBEPBDXZ 10008795 f i LIBCMT:throw_bad_alloc.obj
 0001:000077a2       ??3@YAXPAX@Z               100087a2 f   LIBCMT:delete_scalar.obj
 0001:000077a7       ??$__crt_fast_encode_pointer@PAX@@YAPAXQAX@Z 100087a7 f i libvcruntime:winapi_downlevel.obj
 0001:000077a7       ??$__crt_fast_encode_pointer@PAP6AXXZ@@YAPAP6AXXZQAP6AXXZ@Z 100087a7 f i LIBCMT:utility.obj
 0001:00007808       ___scrt_acquire_startup_lock 10008808 f   LIBCMT:utility.obj
 0001:0000783d       ___scrt_dllmain_after_initialize_c 1000883d f   LIBCMT:utility.obj
 0001:00007868       ___scrt_dllmain_before_initialize_c 10008868 f   LIBCMT:utility.obj
 0001:00007876       ___scrt_dllmain_crt_thread_attach 10008876 f   LIBCMT:utility.obj
 0001:00007895       ___scrt_dllmain_crt_thread_detach 10008895 f   LIBCMT:utility.obj
 0001:000078a2       ___scrt_dllmain_exception_filter 100088a2 f   LIBCMT:utility.obj
 0001:000078d5       ___scrt_dllmain_uninitialize_c 100088d5 f   LIBCMT:utility.obj
 0001:000078f8       ___scrt_dllmain_uninitialize_critical 100088f8 f   LIBCMT:utility.obj
 0001:00007905       ___scrt_initialize_crt     10008905 f   LIBCMT:utility.obj
 0001:0000793e       ___scrt_initialize_onexit_tables 1000893e f   LIBCMT:utility.obj
 0001:000079d5       ___scrt_is_nonwritable_in_current_image 100089d5 f   LIBCMT:utility.obj
 0001:00007a62       ___scrt_release_startup_lock 10008a62 f   LIBCMT:utility.obj
 0001:00007a7f       ___scrt_uninitialize_crt   10008a7f f   LIBCMT:utility.obj
 0001:00007aa7       __onexit                   10008aa7 f   LIBCMT:utility.obj
 0001:00007ae2       _atexit                    10008ae2 f   LIBCMT:utility.obj
 0001:00007af7       ___security_init_cookie    10008af7 f   LIBCMT:gs_support.obj
 0001:00007b93       _DllMain@12                10008b93 f   LIBCMT:dll_dllmain_stub.obj
 0001:00007b99       ?__scrt_initialize_type_info@@YAXXZ 10008b99 f   LIBCMT:tncleanup.obj
 0001:00007ba5       ?__scrt_uninitialize_type_info@@YAXXZ 10008ba5 f   LIBCMT:tncleanup.obj
 0001:00007bb1       ___local_stdio_printf_options 10008bb1 f i LIBCMT:default_local_stdio_options.obj
 0001:00007bb7       ___local_stdio_scanf_options 10008bb7 f i LIBCMT:default_local_stdio_options.obj
 0001:00007bbd       ___scrt_initialize_default_local_stdio_options 10008bbd f   LIBCMT:default_local_stdio_options.obj
 0001:00007bda       ___scrt_get_dyn_tls_init_callback 10008bda f   LIBCMT:dyn_tls_init.obj
 0001:00007be0       ___scrt_fastfail           10008be0 f   LIBCMT:utility_desktop.obj
 0001:00007cfb       __crt_debugger_hook        10008cfb f   LIBCMT:utility_desktop.obj
 0001:00007d03       __RTC_Initialize           10008d03 f   LIBCMT:_initsect_.obj
 0001:00007d2e       __RTC_Terminate            10008d2e f   LIBCMT:_initsect_.obj
 0001:00007d59       @_guard_check_icall@4      10008d59 f i LIBCMT:checkcfg.obj
 0001:00007d60       __SEH_prolog4              10008d60 f   LIBCMT:_sehprolg4_.obj
 0001:00007da6       __SEH_epilog4              10008da6 f   LIBCMT:_sehprolg4_.obj
 0001:00007dbb       ??_Etype_info@@UAEPAXI@Z   10008dbb f i LIBCMT:std_type_info_static.obj
 0001:00007dbb       ??_Gtype_info@@UAEPAXI@Z   10008dbb f i LIBCMT:std_type_info_static.obj
 0001:00007dde       ___isa_available_init      10008dde f   LIBCMT:_cpu_disp_.obj
 0001:00007f7f       __get_startup_argv_mode    10008f7f f   LIBCMT:argv_mode.obj
 0001:00007f83       ___scrt_is_ucrt_dll_in_use 10008f83 f   LIBCMT:ucrt_detection.obj
 0001:00007f8f       @__security_check_cookie@4 10008f8f f   LIBCMT:_secchk_.obj
 0001:00007fa0       ___raise_securityfailure   10008fa0 f   LIBCMT:gs_report.obj
 0001:00007fc8       ___report_gsfailure        10008fc8 f   LIBCMT:gs_report.obj
 0001:000080d0       _memmove                   100090d0 f   libvcruntime:memmove.obj
 0001:00008650       _memcpy                    10009650 f   libvcruntime:memcpy.obj
 0001:00008bd0       _memset                    10009bd0 f   libvcruntime:memset.obj
 0001:00008d70       __except_handler4          10009d70 f   libvcruntime:_chandler4_.obj
 0001:00008eca       ___std_exception_copy      10009eca f   libvcruntime:std_exception.obj
 0001:00008f2d       ___std_exception_destroy   10009f2d f   libvcruntime:std_exception.obj
 0001:00008f4c       __CxxThrowException@8      10009f4c f   libvcruntime:throw.obj
 0001:00008fba       ___vcrt_initialize         10009fba f   libvcruntime:initialization.obj
 0001:00008fe8       ___vcrt_thread_attach      10009fe8 f   libvcruntime:initialization.obj
 0001:00008ff3       ___vcrt_thread_detach      10009ff3 f   libvcruntime:initialization.obj
 0001:00008ffe       ___vcrt_uninitialize       10009ffe f   libvcruntime:initialization.obj
 0001:00009022       ___vcrt_uninitialize_critical 1000a022 f   libvcruntime:initialization.obj
 0001:0000902a       ___std_type_info_destroy_list 1000a02a f   libvcruntime:std_type_info.obj
 0001:00009050       __local_unwind4            1000a050 f   libvcruntime:_exsup4_.obj
 0001:00009126       __seh_longjmp_unwind4@4    1000a126 f   libvcruntime:_exsup4_.obj
 0001:0000914e       @_EH4_CallFilterFunc@8     1000a14e f   libvcruntime:_exsup4_.obj
 0001:00009165       @_EH4_TransferToHandler@8  1000a165 f   libvcruntime:_exsup4_.obj
 0001:0000917e       @_EH4_GlobalUnwind2@8      1000a17e f   libvcruntime:_exsup4_.obj
 0001:00009197       @_EH4_LocalUnwind@16       1000a197 f   libvcruntime:_exsup4_.obj
 0001:000091ae       ___vcrt_freefls@4          1000a1ae f   libvcruntime:per_thread_data.obj
 0001:000091ca       ___vcrt_freeptd            1000a1ca f   libvcruntime:per_thread_data.obj
 0001:00009200       ___vcrt_getptd_noexit      1000a200 f   libvcruntime:per_thread_data.obj
 0001:00009292       ___vcrt_initialize_ptd     1000a292 f   libvcruntime:per_thread_data.obj
 0001:000092c5       ___vcrt_uninitialize_ptd   1000a2c5 f   libvcruntime:per_thread_data.obj
 0001:000092e0       ___vcrt_initialize_locks   1000a2e0 f   libvcruntime:locks.obj
 0001:0000931c       ___vcrt_uninitialize_locks 1000a31c f   libvcruntime:locks.obj
 0001:0000946c       ___vcrt_FlsAlloc           1000a46c f   libvcruntime:winapi_downlevel.obj
 0001:000094a6       ___vcrt_FlsFree            1000a4a6 f   libvcruntime:winapi_downlevel.obj
 0001:000094e0       ___vcrt_FlsGetValue        1000a4e0 f   libvcruntime:winapi_downlevel.obj
 0001:0000951a       ___vcrt_FlsSetValue        1000a51a f   libvcruntime:winapi_downlevel.obj
 0001:00009557       ___vcrt_InitializeCriticalSectionEx 1000a557 f   libvcruntime:winapi_downlevel.obj
 0001:0000959d       ___vcrt_initialize_winapi_thunks 1000a59d f   libvcruntime:winapi_downlevel.obj
 0001:000095c1       ___vcrt_uninitialize_winapi_thunks 1000a5c1 f   libvcruntime:winapi_downlevel.obj
 0001:000095f3       ___vcrt_initialize_pure_virtual_call_handler 1000a5f3 f   libvcruntime:purevirt_data.obj
 0001:00009610       __global_unwind2           1000a610 f   libvcruntime:_exsup_.obj
 0001:00009675       __local_unwind2            1000a675 f   libvcruntime:_exsup_.obj
 0001:000096f9       __abnormal_termination     1000a6f9 f   libvcruntime:_exsup_.obj
 0001:0000971c       __NLG_Notify1              1000a71c f   libvcruntime:_exsup_.obj
 0001:00009725       __NLG_Notify               1000a725 f   libvcruntime:_exsup_.obj
 0001:0000973c       __NLG_Dispatch             1000a73c     libvcruntime:_exsup_.obj
 0001:0000973c       __NLG_Dispatch2            1000a73c     libvcruntime:_exsup_.obj
 0001:00009744       __NLG_Call                 1000a744 f   libvcruntime:_exsup_.obj
 0001:00009746       __NLG_Return2              1000a746     libvcruntime:_exsup_.obj
 0001:00009747       _free                      1000a747 f   libucrt:free.obj
 0001:0000974c       _malloc                    1000a74c f   libucrt:malloc.obj
 0001:00009757       _realloc                   1000a757 f   libucrt:realloc.obj
 0001:00009762       ___acrt_initialize_new_handler 1000a762 f   libucrt:new_handler.obj
 0001:00009776       __callnewh                 1000a776 f   libucrt:new_handler.obj
 0001:000097ba       __query_new_handler        1000a7ba f   libucrt:new_handler.obj
 0001:0000980c       __initterm                 1000a80c f   libucrt:initterm.obj
 0001:00009868       __initterm_e               1000a868 f   libucrt:initterm.obj
 0001:000098ad       __seh_filter_dll           1000a8ad f   libucrt:exception_filter.obj
 0001:000098cd       __seh_filter_exe           1000a8cd f   libucrt:exception_filter.obj
 0001:00009c5b       ___acrt_initialize_thread_local_exit_callback 1000ac5b f   libucrt:exit.obj
 0001:00009c6a       __cexit                    1000ac6a f   libucrt:exit.obj
 0001:00009c79       __exit                     1000ac79 f   libucrt:exit.obj
 0001:00009c8f       __is_c_termination_complete 1000ac8f f   libucrt:exit.obj
 0001:00009f2e       ___acrt_allocate_buffer_for_argv 1000af2e f   libucrt:argv_parsing.obj
 0001:00009f83       __configure_narrow_argv    1000af83 f   libucrt:argv_parsing.obj
 0001:0000a0e7       ??$uninitialize@A6AXAAPAPAD@Z@?$dual_state_global@PAPAD@__crt_state_management@@QAEXA6AXAAPAPAD@Z@Z 1000b0e7 f i libucrt:environment_initialization.obj
 0001:0000a0e7       ??$uninitialize@A6AXAAPAPA_W@Z@?$dual_state_global@PAPA_W@__crt_state_management@@QAEXA6AXAAPAPA_W@Z@Z 1000b0e7 f i libucrt:environment_initialization.obj
 0001:0000a15d       ___dcrt_uninitialize_environments_nolock 1000b15d f   libucrt:environment_initialization.obj
 0001:0000a194       __initialize_narrow_environment 1000b194 f   libucrt:environment_initialization.obj
 0001:0000a199       ??$?RV<lambda_800076c951b434888f4765a74a194fcc>@@AAV<lambda_4e60a939b0d047cfe11ddc22648dfba9>@@V<lambda_6dbb1268764f43b569ce7b67e331d33a>@@@?$__crt_seh_guarded_call@H@@QAEH$$QAV<lambda_800076c951b434888f4765a74a194fcc>@@AAV<lambda_4e60a939b0d047cfe11ddc22648dfba9>@@$$QAV<lambda_6dbb1268764f43b569ce7b67e331d33a>@@@Z 1000b199 f i libucrt:onexit.obj
 0001:0000a1ea       ??$?RV<lambda_995298e7d72eb4c2aab26c0585b3abe5>@@AAV<lambda_275893d493268fdec8709772e3fcec0e>@@V<lambda_293819299cbf9a7022e18b56a874bb5c>@@@?$__crt_seh_guarded_call@H@@QAEH$$QAV<lambda_995298e7d72eb4c2aab26c0585b3abe5>@@AAV<lambda_275893d493268fdec8709772e3fcec0e>@@$$QAV<lambda_293819299cbf9a7022e18b56a874bb5c>@@@Z 1000b1ea f i libucrt:onexit.obj
 0001:0000a23b       ??$__acrt_lock_and_call@V<lambda_275893d493268fdec8709772e3fcec0e>@@@@YAHW4__acrt_lock_id@@$$QAV<lambda_275893d493268fdec8709772e3fcec0e>@@@Z 1000b23b f i libucrt:onexit.obj
 0001:0000a263       ??$__acrt_lock_and_call@V<lambda_4e60a939b0d047cfe11ddc22648dfba9>@@@@YAHW4__acrt_lock_id@@$$QAV<lambda_4e60a939b0d047cfe11ddc22648dfba9>@@@Z 1000b263 f i libucrt:onexit.obj
 0001:0000a28b       ??$__crt_fast_encode_pointer@P6AHXZ@@YAP6AHXZQ6AHXZ@Z 1000b28b f i libucrt:onexit.obj
 0001:0000a50b       __crt_atexit               1000b50b f   libucrt:onexit.obj
 0001:0000a521       __execute_onexit_table     1000b521 f   libucrt:onexit.obj
 0001:0000a53e       __initialize_onexit_table  1000b53e f   libucrt:onexit.obj
 0001:0000a57b       __register_onexit_function 1000b57b f   libucrt:onexit.obj
 0001:0000a690       ___acrt_uninitialize_command_line 1000b690 f   libucrt:argv_data.obj
 0001:0000a693       ___acrt_initialize         1000b693 f   libucrt:initialization.obj
 0001:0000a6a5       ___acrt_thread_attach      1000b6a5 f   libucrt:initialization.obj
 0001:0000a6b0       ___acrt_thread_detach      1000b6b0 f   libucrt:initialization.obj
 0001:0000a6b8       ___acrt_uninitialize       1000b6b8 f   libucrt:initialization.obj
 0001:0000a6ca       ___acrt_uninitialize_critical 1000b6ca f   libucrt:initialization.obj
 0001:0000a6dc       _terminate                 1000b6dc f   libucrt:terminate.obj
 0001:0000a718       _strcpy_s                  1000b718 f   libucrt:strcpy_s.obj
 0001:0000a772       __free_base                1000b772 f   libucrt:free_base.obj
 0001:0000a7ac       __malloc_base              1000b7ac f   libucrt:malloc_base.obj
 0001:0000a7fa       _abort                     1000b7fa f   libucrt:abort.obj
 0001:0000a83d       __calloc_base              1000b83d f   libucrt:calloc_base.obj
 0001:0000a89a       ??0_LocaleUpdate@@QAE@QAU__crt_locale_pointers@@@Z 1000b89a f i libucrt:output.obj
 0001:0000a91d       __realloc_base             1000b91d f   libucrt:realloc_base.obj
 0001:0000a986       ___acrt_initialize_locks   1000b986 f   libucrt:locks.obj
 0001:0000a9c7       ___acrt_lock               1000b9c7 f   libucrt:locks.obj
 0001:0000a9de       ___acrt_uninitialize_locks 1000b9de f   libucrt:locks.obj
 0001:0000aa0f       ___acrt_unlock             1000ba0f f   libucrt:locks.obj
 0001:0000aa26       ??$?RV<lambda_3518db117f0e7cdb002338c5d3c47b6c>@@AAV<lambda_b2ea41f6bbb362cd97d94c6828d90b61>@@V<lambda_abdedf541bb04549bc734292b4a045d4>@@@?$__crt_seh_guarded_call@X@@QAEX$$QAV<lambda_3518db117f0e7cdb002338c5d3c47b6c>@@AAV<lambda_b2ea41f6bbb362cd97d94c6828d90b61>@@$$QAV<lambda_abdedf541bb04549bc734292b4a045d4>@@@Z 1000ba26 f i libucrt:per_thread_data.obj
 0001:0000aa76       ??$?RV<lambda_51b6e8b1eb166f2a3faf91f424b38130>@@AAV<lambda_6250bd4b2a391816dd638c3bf72b0bcb>@@V<lambda_0b5a4a3e68152e1d9b943535f5f47bed>@@@?$__crt_seh_guarded_call@X@@QAEX$$QAV<lambda_51b6e8b1eb166f2a3faf91f424b38130>@@AAV<lambda_6250bd4b2a391816dd638c3bf72b0bcb>@@$$QAV<lambda_0b5a4a3e68152e1d9b943535f5f47bed>@@@Z 1000ba76 f i libucrt:per_thread_data.obj
 0001:0000aad7       ??$?RV<lambda_5b71d36f03204c0beab531769a5b5694>@@AAV<lambda_be2b3da3f62db62e9dad5dc70221a656>@@V<lambda_8f9ce462984622f9bf76b59e2aaaf805>@@@?$__crt_seh_guarded_call@X@@QAEX$$QAV<lambda_5b71d36f03204c0beab531769a5b5694>@@AAV<lambda_be2b3da3f62db62e9dad5dc70221a656>@@$$QAV<lambda_8f9ce462984622f9bf76b59e2aaaf805>@@@Z 1000bad7 f i libucrt:per_thread_data.obj
 0001:0000ab22       ??$?RV<lambda_9df27f884b057bc3edfc946cb5b7cf47>@@AAV<lambda_e69574bed617af4e071282c136b37893>@@V<lambda_cc0d902bcbbeb830f749456577db4721>@@@?$__crt_seh_guarded_call@X@@QAEX$$QAV<lambda_9df27f884b057bc3edfc946cb5b7cf47>@@AAV<lambda_e69574bed617af4e071282c136b37893>@@$$QAV<lambda_cc0d902bcbbeb830f749456577db4721>@@@Z 1000bb22 f i libucrt:per_thread_data.obj
 0001:0000ab6a       ??$__acrt_lock_and_call@V<lambda_6250bd4b2a391816dd638c3bf72b0bcb>@@@@YAXW4__acrt_lock_id@@$$QAV<lambda_6250bd4b2a391816dd638c3bf72b0bcb>@@@Z 1000bb6a f i libucrt:per_thread_data.obj
 0001:0000ab92       ??$__acrt_lock_and_call@V<lambda_b2ea41f6bbb362cd97d94c6828d90b61>@@@@YAXW4__acrt_lock_id@@$$QAV<lambda_b2ea41f6bbb362cd97d94c6828d90b61>@@@Z 1000bb92 f i libucrt:per_thread_data.obj
 0001:0000abba       ??$__acrt_lock_and_call@V<lambda_be2b3da3f62db62e9dad5dc70221a656>@@@@YAXW4__acrt_lock_id@@$$QAV<lambda_be2b3da3f62db62e9dad5dc70221a656>@@@Z 1000bbba f i libucrt:per_thread_data.obj
 0001:0000abe2       ??$__acrt_lock_and_call@V<lambda_e69574bed617af4e071282c136b37893>@@@@YAXW4__acrt_lock_id@@$$QAV<lambda_e69574bed617af4e071282c136b37893>@@@Z 1000bbe2 f i libucrt:per_thread_data.obj
 0001:0000ad98       ___acrt_freeptd            1000bd98 f   libucrt:per_thread_data.obj
 0001:0000adc4       ___acrt_getptd             1000bdc4 f   libucrt:per_thread_data.obj
 0001:0000ae48       ___acrt_getptd_noexit      1000be48 f   libucrt:per_thread_data.obj
 0001:0000aecd       ___acrt_initialize_ptd     1000becd f   libucrt:per_thread_data.obj
 0001:0000aef9       ___acrt_uninitialize_ptd   1000bef9 f   libucrt:per_thread_data.obj
 0001:0000b02d       ___acrt_FlsAlloc@4         1000c02d f   libucrt:winapi_thunks.obj
 0001:0000b083       ___acrt_FlsFree@4          1000c083 f   libucrt:winapi_thunks.obj
 0001:0000b0d9       ___acrt_FlsGetValue@4      1000c0d9 f   libucrt:winapi_thunks.obj
 0001:0000b12f       ___acrt_FlsSetValue@8      1000c12f f   libucrt:winapi_thunks.obj
 0001:0000b188       ___acrt_InitializeCriticalSectionEx@12 1000c188 f   libucrt:winapi_thunks.obj
 0001:0000b1ea       ___acrt_LCMapStringEx@36   1000c1ea f   libucrt:winapi_thunks.obj
 0001:0000b272       ___acrt_LocaleNameToLCID@8 1000c272 f   libucrt:winapi_thunks.obj
 0001:0000b2ce       ___acrt_initialize_winapi_thunks 1000c2ce f   libucrt:winapi_thunks.obj
 0001:0000b2f4       ___acrt_is_packaged_app    1000c2f4 f   libucrt:winapi_thunks.obj
 0001:0000b37b       ___acrt_uninitialize_winapi_thunks 1000c37b f   libucrt:winapi_thunks.obj
 0001:0000b3b1       ___acrt_call_reportfault   1000c3b1 f   libucrt:invalid_parameter.obj
 0001:0000b4ec       ___acrt_initialize_invalid_parameter_handler 1000c4ec f   libucrt:invalid_parameter.obj
 0001:0000b500       __invalid_parameter        1000c500 f   libucrt:invalid_parameter.obj
 0001:0000b57b       __invalid_parameter_noinfo 1000c57b f   libucrt:invalid_parameter.obj
 0001:0000b58b       __invoke_watson            1000c58b f   libucrt:invalid_parameter.obj
 0001:0000b5be       ___acrt_errno_from_os_error 1000c5be f   libucrt:errno.obj
 0001:0000b601       ___acrt_errno_map_os_error 1000c601 f   libucrt:errno.obj
 0001:0000b624       ___doserrno                1000c624 f   libucrt:errno.obj
 0001:0000b637       __errno                    1000c637 f   libucrt:errno.obj
 0001:0000ba0c       ??1?$argument_list@D@?A0xb0e4b824@@QAE@XZ 1000ca0c f i libucrt:argv_wildcards.obj
 0001:0000ba31       ?append@?$argument_list@D@?A0xb0e4b824@@QAEHQAD@Z 1000ca31 f i libucrt:argv_wildcards.obj
 0001:0000ba66       ?expand_if_necessary@?$argument_list@D@?A0xb0e4b824@@AAEHXZ 1000ca66 f i libucrt:argv_wildcards.obj
 0001:0000baed       ___acrt_expand_narrow_argv_wildcards 1000caed f   libucrt:argv_wildcards.obj
 0001:0000baf8       ??$?RV<lambda_978dc153c237d78434369da87b74ff60>@@AAV<lambda_ad1ced32f4ac17aa236e5ef05d6b3b7c>@@V<lambda_4a8533e2866a575feecb8298ce776b0d>@@@?$__crt_seh_guarded_call@X@@QAEX$$QAV<lambda_978dc153c237d78434369da87b74ff60>@@AAV<lambda_ad1ced32f4ac17aa236e5ef05d6b3b7c>@@$$QAV<lambda_4a8533e2866a575feecb8298ce776b0d>@@@Z 1000caf8 f i libucrt:mbctype.obj
 0001:0000bb3b       ??$__acrt_lock_and_call@V<lambda_ad1ced32f4ac17aa236e5ef05d6b3b7c>@@@@YAXW4__acrt_lock_id@@$$QAV<lambda_ad1ced32f4ac17aa236e5ef05d6b3b7c>@@@Z 1000cb3b f i libucrt:mbctype.obj
 0001:0000bfd2       ___acrt_initialize_multibyte 1000cfd2 f   libucrt:mbctype.obj
 0001:0000bff0       ___acrt_update_thread_multibyte_data 1000cff0 f   libucrt:mbctype.obj
 0001:0000c092       __setmbcp_nolock           1000d092 f   libucrt:mbctype.obj
 0001:0000c35d       __ismbblead                1000d35d f   libucrt:ismbbyte.obj
 0001:0000c375       ___acrt_initialize_command_line 1000d375 f   libucrt:argv_data.obj
 0001:0000c3c5       ___dcrt_get_narrow_environment_from_os 1000d3c5 f   libucrt:get_environment_from_os.obj
 0001:0000c448       __recalloc                 1000d448 f   libucrt:recalloc.obj
 0001:0000c453       __recalloc_base            1000d453 f   libucrt:recalloc.obj
 0001:0000c4c0       ___acrt_initialize_heap    1000d4c0 f   libucrt:heap_handle.obj
 0001:0000c4d1       ___acrt_uninitialize_heap  1000d4d1 f   libucrt:heap_handle.obj
 0001:0000c647       ___acrt_initialize_lowio   1000d647 f   libucrt:ioinit.obj
 0001:0000c69d       ___acrt_uninitialize_lowio 1000d69d f   libucrt:ioinit.obj
 0001:0000c6c9       ___acrt_execute_initializers 1000d6c9 f   libucrt:shared_initialization.obj
 0001:0000c74c       ___acrt_execute_uninitializers 1000d74c f   libucrt:shared_initialization.obj
 0001:0000c799       ??$?RV<lambda_a048d3beccc847880fc8490e18b82769>@@AAV<lambda_ec61778202f4f5fc7e7711acc23c3bca>@@V<lambda_f7496a158712204296dd6628a163878e>@@@?$__crt_seh_guarded_call@P6AXH@Z@@QAEP6AXH@Z$$QAV<lambda_a048d3beccc847880fc8490e18b82769>@@AAV<lambda_ec61778202f4f5fc7e7711acc23c3bca>@@$$QAV<lambda_f7496a158712204296dd6628a163878e>@@@Z 1000d799 f i libucrt:signal.obj
 0001:0000c7f3       ??$__acrt_lock_and_call@V<lambda_ec61778202f4f5fc7e7711acc23c3bca>@@@@YAP6AXH@ZW4__acrt_lock_id@@$$QAV<lambda_ec61778202f4f5fc7e7711acc23c3bca>@@@Z 1000d7f3 f i libucrt:signal.obj
 0001:0000c85d       ?initialize@?$dual_state_global@P6AXH@Z@__crt_state_management@@QAEXQ6AXH@Z@Z 1000d85d f i libucrt:signal.obj
 0001:0000c85d       ?initialize@?$dual_state_global@P6AHPAU_exception@@@Z@__crt_state_management@@QAEXQ6AHPAU_exception@@@Z@Z 1000d85d f i libucrt:matherr.obj
 0001:0000c85d       ?initialize@?$dual_state_global@P6AHI@Z@__crt_state_management@@QAEXQ6AHI@Z@Z 1000d85d f i libucrt:new_handler.obj
 0001:0000c85d       ?initialize@?$dual_state_global@PAPAD@__crt_state_management@@QAEXQAPAD@Z 1000d85d f i libucrt:environment_initialization.obj
 0001:0000c85d       ?initialize@?$dual_state_global@PAU__crt_locale_data@@@__crt_state_management@@QAEXQAU__crt_locale_data@@@Z 1000d85d f i libucrt:initialization.obj
 0001:0000c85d       ?initialize@?$dual_state_global@P6AXPB_W00II@Z@__crt_state_management@@QAEXQ6AXPB_W00II@Z@Z 1000d85d f i libucrt:invalid_parameter.obj
 0001:0000c8b6       ___acrt_get_sigabrt_handler 1000d8b6 f   libucrt:signal.obj
 0001:0000c8cd       ___acrt_initialize_signal_handlers 1000d8cd f   libucrt:signal.obj
 0001:0000c908       ___fpecode                 1000d908 f   libucrt:signal.obj
 0001:0000c911       _raise                     1000d911 f   libucrt:signal.obj
 0001:0000cb19       ___acrt_has_user_matherr   1000db19 f   libucrt:matherr.obj
 0001:0000cb32       ___acrt_initialize_user_matherr 1000db32 f   libucrt:matherr.obj
 0001:0000cb46       ___acrt_invoke_user_matherr 1000db46 f   libucrt:matherr.obj
 0001:0000cb8f       __query_new_mode           1000db8f f   libucrt:new_mode.obj
 0001:0000cb95       __mbtowc_l                 1000db95 f   libucrt:mbtowc.obj
 0001:0000cc8f       _mbtowc                    1000dc8f f   libucrt:mbtowc.obj
 0001:0000cca9       ___acrt_update_locale_info 1000dca9 f   libucrt:locale_update.obj
 0001:0000ccd6       ___acrt_update_multibyte_info 1000dcd6 f   libucrt:locale_update.obj
 0001:0000cd03       __fileno                   1000dd03 f   libucrt:fileno.obj
 0001:0000cd29       ___acrt_initialize_stdio   1000dd29 f   libucrt:_file.obj
 0001:0000cdf1       ___acrt_uninitialize_stdio 1000ddf1 f   libucrt:_file.obj
 0001:0000ce3d       __lock_file                1000de3d f   libucrt:_file.obj
 0001:0000ce51       __unlock_file              1000de51 f   libucrt:_file.obj
 0001:0000ce65       ___acrt_set_locale_changed 1000de65 f   libucrt:wsetlocale.obj
 0001:0000ce70       ___acrt_uninitialize_locale 1000de70 f   libucrt:wsetlocale.obj
 0001:0000cec2       ___pctype_func             1000dec2 f   libucrt:ctype.obj
 0001:0000cee8       ___acrt_add_locale_ref     1000dee8 f   libucrt:locale_refcounting.obj
 0001:0000cf65       ___acrt_free_locale        1000df65 f   libucrt:locale_refcounting.obj
 0001:0000d0af       ___acrt_locale_add_lc_time_reference 1000e0af f   libucrt:locale_refcounting.obj
 0001:0000d0d8       ___acrt_locale_free_lc_time_if_unreferenced 1000e0d8 f   libucrt:locale_refcounting.obj
 0001:0000d108       ___acrt_locale_release_lc_time_reference 1000e108 f   libucrt:locale_refcounting.obj
 0001:0000d131       ___acrt_release_locale_ref 1000e131 f   libucrt:locale_refcounting.obj
 0001:0000d1b2       ___acrt_update_thread_locale_data 1000e1b2 f   libucrt:locale_refcounting.obj
 0001:0000d229       __updatetlocinfoEx_nolock  1000e229 f   libucrt:locale_refcounting.obj
 0001:0000d335       ___acrt_DownlevelLocaleNameToLCID 1000e335 f   libucrt:lcidtoname_downlevel.obj
 0001:0000d450       _qsort                     1000e450 f   libucrt:qsort.obj
 0001:0000d89b       _strncpy_s                 1000e89b f   libucrt:strncpy_s.obj
 0001:0000d8b0       _strpbrk                   1000e8b0 f   libucrt:strpbrk.obj
 0001:0000d8f0       __mbsdec                   1000e8f0 f   libucrt:mbsdec.obj
 0001:0000d907       __mbsdec_l                 1000e907 f   libucrt:mbsdec.obj
 0001:0000d9a3       ___acrt_GetStringTypeA     1000e9a3 f   libucrt:getstringtypea.obj
 0001:0000dac0       __freea_crt                1000eac0 f i libucrt:getstringtypea.obj
 0001:0000dcfd       ___acrt_LCMapStringA       1000ecfd f   libucrt:lcmapstringa.obj
 0001:0000dd48       __msize                    1000ed48 f   libucrt:msize.obj
 0001:0000dd7b       ___acrt_lowio_create_handle_array 1000ed7b f   libucrt:osfinfo.obj
 0001:0000ddf5       ___acrt_lowio_destroy_handle_array 1000edf5 f   libucrt:osfinfo.obj
 0001:0000de2a       ___acrt_lowio_ensure_fh_exists 1000ee2a f   libucrt:osfinfo.obj
 0001:0000dec2       ___acrt_lowio_lock_fh      1000eec2 f   libucrt:osfinfo.obj
 0001:0000dee5       ___acrt_lowio_unlock_fh    1000eee5 f   libucrt:osfinfo.obj
 0001:0000df08       __free_osfhnd              1000ef08 f   libucrt:osfinfo.obj
 0001:0000df99       __get_osfhandle            1000ef99 f   libucrt:osfinfo.obj
 0001:0000e003       __isatty                   1000f003 f   libucrt:isatty.obj
 0001:0000e059       ___acrt_stdio_flush_nolock 1000f059 f   libucrt:fflush.obj
 0001:0000e0bf       __fflush_nolock            1000f0bf f   libucrt:fflush.obj
 0001:0000e106       __flushall                 1000f106 f   libucrt:fflush.obj
 0001:0000e1e7       __isleadbyte_l             1000f1e7 f i libucrt:_wctype.obj
 0001:0000e220       __fcloseall                1000f220 f   libucrt:closeall.obj
 0001:0000e2c0       ___acrt_stdio_free_buffer_nolock 1000f2c0 f   libucrt:_freebuf.obj
 0001:0000e2fe       ___acrt_locale_free_monetary 1000f2fe f   libucrt:initmon.obj
 0001:0000e3fc       ___acrt_locale_free_numeric 1000f3fc f   libucrt:initnum.obj
 0001:0000e4a1       ___acrt_locale_free_time   1000f4a1 f   libucrt:inittime.obj
 0001:0000e585       ___strncnt                 1000f585 f   libucrt:strncnt.obj
 0001:0000e5a1       __query_app_type           1000f5a1 f   libucrt:report_runtime_error.obj
 0001:0000e5a7       ??$?RV<lambda_61cee617f5178ae960314fd4d05640a0>@@AAV<lambda_6978c1fb23f02e42e1d9e99668cc68aa>@@V<lambda_9cd88cf8ad10232537feb2133f08c833>@@@?$__crt_seh_guarded_call@H@@QAEH$$QAV<lambda_61cee617f5178ae960314fd4d05640a0>@@AAV<lambda_6978c1fb23f02e42e1d9e99668cc68aa>@@$$QAV<lambda_9cd88cf8ad10232537feb2133f08c833>@@@Z 1000f5a7 f i libucrt:commit.obj
 0001:0000e63f       ??$__acrt_lowio_lock_fh_and_call@V<lambda_6978c1fb23f02e42e1d9e99668cc68aa>@@@@YAHH$$QAV<lambda_6978c1fb23f02e42e1d9e99668cc68aa>@@@Z 1000f63f f i libucrt:commit.obj
 0001:0000e667       __commit                   1000f667 f   libucrt:commit.obj
 0001:0000ec66       __write                    1000fc66 f   libucrt:write.obj
 0001:0000ed51       __write_nolock             1000fd51 f   libucrt:write.obj
 0001:0000ef60       _log10                     1000ff60 f   libucrt:log10.obj
 0001:0000efa0       __CIlog10                  1000ffa0 f   libucrt:log10.obj
 0001:0000efdb       __CIlog10_default          1000ffdb f   libucrt:log10.obj
 0001:0000efef       __log10_default            1000ffef     libucrt:log10.obj
 0001:0000f0b0       _ceil                      100100b0 f   libucrt:ceil_pentium4.obj
 0001:0000f0f0       __ceil_pentium4            100100f0 f   libucrt:ceil_pentium4.obj
 0001:0000f24b       __lseeki64_nolock          1001024b f   libucrt:lseek.obj
 0001:0000f266       __fclose_nolock            10010266 f   libucrt:fclose.obj
 0001:0000f2dc       _fclose                    100102dc f   libucrt:fclose.obj
 0001:0000f360       ___ascii_strnicmp          10010360 f   libucrt:_strnicm.obj
 0001:0000f3c1       __putwch_nolock            100103c1 f   libucrt:putwch.obj
 0001:0000f406       ___acrt_initialize_sse2    10010406 f   libucrt:mathfcns.obj
 0001:0000f420       __CIlog10_pentium4         10010420 f   libucrt:log10_pentium4.obj
 0001:0000f438       __log10_pentium4           10010438     libucrt:log10_pentium4.obj
 0001:0000f6c1       __fFEXP                    100106c1     libucrt:87tran.obj
 0001:0000f718       __rtinfpopse               10010718     libucrt:87tran.obj
 0001:0000f71a       __rtinfnpopse              1001071a     libucrt:87tran.obj
 0001:0000f72a       __fFLN                     1001072a     libucrt:87tran.obj
 0001:0000f7df       __rtinfpop                 100107df     libucrt:87tran.obj
 0001:0000f7e1       __rtinfnpop                100107e1     libucrt:87tran.obj
 0001:0000f7fe       __ffexpm1                  100107fe     libucrt:87tran.obj
 0001:0000f8b0       __trandisp1                100108b0 f   libucrt:87disp.obj
 0001:0000f917       __trandisp2                10010917 f   libucrt:87disp.obj
 0001:0000f9a3       __rttospopde               100109a3     libucrt:87disp.obj
 0001:0000f9a8       __rttospop                 100109a8     libucrt:87disp.obj
 0001:0000f9aa       __rtnospop                 100109aa     libucrt:87disp.obj
 0001:0000f9ac       __rttosnpop                100109ac     libucrt:87disp.obj
 0001:0000f9ad       __rtnospopde               100109ad     libucrt:87disp.obj
 0001:0000f9b4       __rtzeropop                100109b4     libucrt:87disp.obj
 0001:0000f9b6       __rtzeronpop               100109b6     libucrt:87disp.obj
 0001:0000f9bb       __rtzerospop               100109bb     libucrt:87disp.obj
 0001:0000f9c8       __rtonepop                 100109c8     libucrt:87disp.obj
 0001:0000f9ca       __rtonenpop                100109ca     libucrt:87disp.obj
 0001:0000f9cf       __tosnan1                  100109cf     libucrt:87disp.obj
 0001:0000f9fa       __nosnan2                  100109fa     libucrt:87disp.obj
 0001:0000f9fc       __tosnan2                  100109fc     libucrt:87disp.obj
 0001:0000fa24       __nan2                     10010a24     libucrt:87disp.obj
 0001:0000fa63       __rtindfpop                10010a63     libucrt:87disp.obj
 0001:0000fa65       __rtindfnpop               10010a65     libucrt:87disp.obj
 0001:0000fa76       __rttosnpopde              10010a76     libucrt:87disp.obj
 0001:0000fa80       __rtatan2inf               10010a80     libucrt:87disp.obj
 0001:0000fa9d       __rtchsifneg               10010a9d     libucrt:87disp.obj
 0001:0000fab0       __twoToTOS                 10010ab0 f   libucrt:common.obj
 0001:0000fac5       __load_CW                  10010ac5 f   libucrt:common.obj
 0001:0000fadc       __convertTOStoQNaN         10010adc f   libucrt:common.obj
 0001:0000faf5       __fload_withFB             10010af5 f   libucrt:common.obj
 0001:0000fb38       __checkTOS_withFB          10010b38 f   libucrt:common.obj
 0001:0000fb4e       __fast_exit                10010b4e f   libucrt:common.obj
 0001:0000fb5b       __math_exit                10010b5b f   libucrt:common.obj
 0001:0000fb85       __check_overflow_exit      10010b85 f   libucrt:common.obj
 0001:0000fb99       __check_range_exit         10010b99 f   libucrt:common.obj
 0001:0000fc40       __startTwoArgErrorHandling 10010c40 f   libucrt:genexcep.obj
 0001:0000fc57       __startOneArgErrorHandling 10010c57 f   libucrt:genexcep.obj
 0001:0000fc93       ___libm_error_support      10010c93 f   libucrt:libm_error.obj
 0001:0000feab       __ceil_default             10010eab f   libucrt:ceil.obj
 0001:0000ff64       ??$?RV<lambda_123407a5e2ac06da108355a851863b7a>@@AAV<lambda_2fe9b910cf3cbf4a0ab98a02ba45b3ec>@@V<lambda_ae55bdf541ad94d75914d381c370e64d>@@@?$__crt_seh_guarded_call@H@@QAEH$$QAV<lambda_123407a5e2ac06da108355a851863b7a>@@AAV<lambda_2fe9b910cf3cbf4a0ab98a02ba45b3ec>@@$$QAV<lambda_ae55bdf541ad94d75914d381c370e64d>@@@Z 10010f64 f i libucrt:close.obj
 0001:0000ffe6       ??$__acrt_lowio_lock_fh_and_call@V<lambda_2fe9b910cf3cbf4a0ab98a02ba45b3ec>@@@@YAHH$$QAV<lambda_2fe9b910cf3cbf4a0ab98a02ba45b3ec>@@@Z 10010fe6 f i libucrt:close.obj
 0001:0001000e       __close                    1001100e f   libucrt:close.obj
 0001:0001008d       __close_nolock             1001108d f   libucrt:close.obj
 0001:00010129       ?__acrt_stdio_free_stream@@YAXV__crt_stdio_stream@@@Z 10011129 f   libucrt:stream.obj
 0001:00010164       ___dcrt_lowio_initialize_console_output 10011164 f   libucrt:initcon.obj
 0001:00010183       ___dcrt_terminate_console_output 10011183 f   libucrt:initcon.obj
 0001:0001019a       __clrfp                    1001119a f   libucrt:fpctrl.obj
 0001:000101ad       __ctrlfp                   100111ad f   libucrt:fpctrl.obj
 0001:000101d9       __set_statfp               100111d9 f   libucrt:fpctrl.obj
 0001:00010234       __statfp                   10011234 f   libucrt:fpctrl.obj
 0001:00010246       __d_inttype                10011246 f   libucrt:powhlp.obj
 0001:000102b0       __powhlp                   100112b0 f   libucrt:powhlp.obj
 0001:000103db       __87except                 100113db f   libucrt:87except.obj
 0001:000104e6       __frnd                     100114e6 f   libucrt:frnd.obj
 0001:000104fc       __errcode                  100114fc f   libucrt:fpexcept.obj
 0001:00010530       __except1                  10011530 f   libucrt:fpexcept.obj
 0001:000105fe       __handle_exc               100115fe f   libucrt:fpexcept.obj
 0001:000107de       __raise_exc                100117de f   libucrt:fpexcept.obj
 0001:00010801       __raise_exc_ex             10011801 f   libucrt:fpexcept.obj
 0001:00010af2       __set_errno_from_matherr   10011af2 f   libucrt:fpexcept.obj
 0001:00010b21       __umatherr                 10011b21 f   libucrt:fpexcept.obj
 0001:00010bc3       __decomp                   10011bc3 f   libucrt:util.obj
 0001:00010c97       __set_exp                  10011c97 f   libucrt:util.obj
 0001:00010cc6       __sptype                   10011cc6 f   libucrt:util.obj
 0001:00010d24       __fpclass                  10011d24 f   libucrt:ieeemisc.obj
 0001:00010dc8       _IsProcessorFeaturePresent@4 10011dc8 f   kernel32:KERNEL32.dll
 0001:00010dce       _RtlUnwind@16              10011dce f   kernel32:KERNEL32.dll
 0001:00010de0       __FindPESection            10011de0 f   LIBCMT:pesect.obj
 0001:00010e30       __IsNonwritableInCurrentImage 10011e30 f   LIBCMT:pesect.obj
 0001:00010ef0       __ValidateImageBase        10011ef0 f   LIBCMT:pesect.obj
 0001:00010f30       __aulldvrm                 10011f30 f   LIBCMT:ulldvrm.obj
 0001:00010fd0       __SEH_prolog4_GS           10011fd0 f   LIBCMT:_sehprolg4gs_.obj
 0001:00011019       __SEH_epilog4_GS           10012019 f   LIBCMT:_sehprolg4gs_.obj
 0001:00011030       __allmul                   10012030 f   LIBCMT:llmul.obj
 0001:00011070       __alldvrm                  10012070 f   LIBCMT:lldvrm.obj
 0001:00011150       __aullshr                  10012150 f   LIBCMT:ullshr.obj
 0001:00011170       __alloca_probe_16          10012170 f   LIBCMT:alloca16.obj
 0001:00011186       __alloca_probe_8           10012186     LIBCMT:alloca16.obj
 0001:000111a0       __allshl                   100121a0 f   LIBCMT:llshl.obj
 0001:000111c0       __ftol2_sse                100121c0 f   LIBCMT:_ftol2_.obj
 0001:000111c9       __ftol2_pentium4           100121c9 f   LIBCMT:_ftol2_.obj
 0001:000111dc       __ftol2_sse_excpt          100121dc f   LIBCMT:_ftol2_.obj
 0001:00011200       __ftol2                    10012200 f   LIBCMT:_ftol2_.obj
 0001:00011280       _strchr                    10012280 f   libvcruntime:strchr.obj
 0001:000112ee       ___from_strstr_to_strchr   100122ee     libvcruntime:strchr.obj
 0001:000113b0       _strrchr                   100123b0 f   libvcruntime:strrchr.obj
 0001:00011544       __TI2?AVbad_alloc@std@@    10012544     LIBCMT:throw_bad_alloc.obj
 0001:00011554       __CTA2?AVbad_alloc@std@@   10012554     LIBCMT:throw_bad_alloc.obj
 0001:00011560       __CT??_R0?AVbad_alloc@std@@@8??0bad_alloc@std@@QAE@ABV01@@Z12 10012560     LIBCMT:throw_bad_alloc.obj
 0001:0001157c       __CT??_R0?AVexception@std@@@8??0exception@std@@QAE@ABV01@@Z12 1001257c     LIBCMT:throw_bad_alloc.obj
 0001:00011598       __TI3?AVbad_array_new_length@std@@ 10012598     LIBCMT:throw_bad_alloc.obj
 0001:000115a8       __CTA3?AVbad_array_new_length@std@@ 100125a8     LIBCMT:throw_bad_alloc.obj
 0001:000115b8       __CT??_R0?AVbad_array_new_length@std@@@8??0bad_array_new_length@std@@QAE@ABV01@@Z12 100125b8     LIBCMT:throw_bad_alloc.obj
 0002:00000000       ___scrt_native_dllmain_reason 10013000     LIBCMT:utility.obj
 0002:00000010       ___isa_enabled             10013010     LIBCMT:_cpu_disp_.obj
 0002:00000014       ___security_cookie_complement 10013014     LIBCMT:gs_cookie.obj
 0002:00000018       ___security_cookie         10013018     LIBCMT:gs_cookie.obj
 0002:00000030       __NLG_Destination          10013030     libvcruntime:_exsup_.obj
 0002:00000040       ___abort_behavior          10013040     libucrt:abort.obj
 0002:00000148       __mbctype                  10013148     libucrt:mbctype.obj
 0002:00000250       __mbcasemap                10013250     libucrt:mbctype.obj
 0002:00000350       ___acrt_initial_multibyte_data 10013350     libucrt:mbctype.obj
 0002:00000570       ___acrt_current_multibyte_data 10013570     libucrt:mbctype.obj
 0002:00000578       ___acrt_initial_locale_data 10013578     libucrt:nlsdata.obj
 0002:00000630       ___acrt_initial_locale_pointers 10013630     libucrt:nlsdata.obj
 0002:00000638       ___acrt_wide_c_locale_string 10013638     libucrt:nlsdata.obj
 0002:00000640       __iob                      10013640     libucrt:_file.obj
 0002:000006f0       ___globallocalestatus      100136f0     libucrt:glstatus.obj
 0002:000006f4       ___acrt_lconv_static_decimal 100136f4     libucrt:localeconv.obj
 0002:000006f8       ___acrt_lconv_static_W_decimal 100136f8     libucrt:localeconv.obj
 0002:00000700       ___acrt_lconv_c            10013700     libucrt:localeconv.obj
 0002:00000750       ___dcrt_lowio_console_output_handle 10013750     libucrt:initcon.obj
 0002:00000760       __fltused                  10013760     LIBCMT:fltused.obj
 0002:00000770       ??_R0?AVbad_alloc@std@@@8  10013770     LIBCMT:throw_bad_alloc.obj
 0002:0000078c       ??_R0?AVexception@std@@@8  1001378c     LIBCMT:throw_bad_alloc.obj
 0002:000007a8       ??_R0?AVbad_array_new_length@std@@@8 100137a8     LIBCMT:throw_bad_alloc.obj
 0002:000007d0       ??_R0?AVtype_info@@@8      100137d0     LIBCMT:std_type_info_static.obj
 0002:00000988       ___scrt_current_native_startup_state 10013988     LIBCMT:utility.obj
 0002:0000098c       ___scrt_native_startup_lock 1001398c     LIBCMT:utility.obj
 0002:000009b0       ?__type_info_root_node@@3U__type_info_node@@A 100139b0     LIBCMT:tncleanup.obj
 0002:000009b8       ?_OptionsStorage@?1??__local_stdio_printf_options@@9@4_KA 100139b8     LIBCMT:default_local_stdio_options.obj
 0002:000009c0       ?_OptionsStorage@?1??__local_stdio_scanf_options@@9@4_KA 100139c0     LIBCMT:default_local_stdio_options.obj
 0002:000009c8       ___scrt_debugger_hook_flag 100139c8     LIBCMT:utility_desktop.obj
 0002:000009cc       ___isa_available           100139cc     LIBCMT:_cpu_disp_.obj
 0002:000009d0       ___favor                   100139d0     LIBCMT:_cpu_disp_.obj
 0002:00000d6c       ___pPurecall               10013d6c     libvcruntime:purevirt_data.obj
 0002:00000d70       ?pArgList@UnDecorator@@0PAVReplicator@@A 10013d70     libvcruntime:undname.obj
 0002:00000d74       ?pZNameList@UnDecorator@@0PAVReplicator@@A 10013d74     libvcruntime:undname.obj
 0002:00000d78       ?pTemplateArgList@UnDecorator@@0PAVReplicator@@A 10013d78     libvcruntime:undname.obj
 0002:00000d7c       ?gName@UnDecorator@@0PBDB  10013d7c     libvcruntime:undname.obj
 0002:00000d80       ?name@UnDecorator@@0PBDB   10013d80     libvcruntime:undname.obj
 0002:00000d84       ?outputString@UnDecorator@@0PADA 10013d84     libvcruntime:undname.obj
 0002:00000d88       ?maxStringLength@UnDecorator@@0HA 10013d88     libvcruntime:undname.obj
 0002:00000d8c       ?disableFlags@UnDecorator@@0KA 10013d8c     libvcruntime:undname.obj
 0002:00000d90       ?fExplicitTemplateParams@UnDecorator@@0_NA 10013d90     libvcruntime:undname.obj
 0002:00000d91       ?fGetTemplateArgumentList@UnDecorator@@0_NA 10013d91     libvcruntime:undname.obj
 0002:00000d94       ?m_pGetParameter@UnDecorator@@0P6APADJ@ZA 10013d94     libvcruntime:undname.obj
 0002:00000ec8       __environ_table            10013ec8     libucrt:environment_initialization.obj
 0002:00000ecc       __wenviron_table           10013ecc     libucrt:environment_initialization.obj
 0002:00000ed0       ___dcrt_initial_wide_environment 10013ed0     libucrt:environment_initialization.obj
 0002:00000ed4       ___dcrt_initial_narrow_environment 10013ed4     libucrt:environment_initialization.obj
 0002:00000ed8       ___acrt_atexit_table       10013ed8     libucrt:onexit.obj
 0002:00000ee4       ___acrt_at_quick_exit_table 10013ee4     libucrt:onexit.obj
 0002:00001108       ___mblocalename            10014108     libucrt:mbctype.obj
 0002:0000110c       ___mbcodepage              1001410c     libucrt:mbctype.obj
 0002:00001110       ___ismbcodepage            10014110     libucrt:mbctype.obj
 0002:00001114       ___mbulinfo                10014114     libucrt:mbctype.obj
 0002:00001128       ___argc                    10014128     libucrt:argv_data.obj
 0002:0000112c       ___argv                    1001412c     libucrt:argv_data.obj
 0002:00001130       ___wargv                   10014130     libucrt:argv_data.obj
 0002:00001134       __acmdln                   10014134     libucrt:argv_data.obj
 0002:00001138       __wcmdln                   10014138     libucrt:argv_data.obj
 0002:0000113c       __pgmptr                   1001413c     libucrt:argv_data.obj
 0002:00001140       ___acrt_heap               10014140     libucrt:heap_handle.obj
 0002:00001148       ___pioinfo                 10014148     libucrt:ioinit.obj
 0002:00001348       __nhandle                  10014348     libucrt:ioinit.obj
 0002:00001360       ___acrt_current_locale_data 10014360     libucrt:nlsdata.obj
 0002:00001364       ___acrt_stdout_buffer      10014364     libucrt:_sftbuf.obj
 0002:00001368       ___acrt_stderr_buffer      10014368     libucrt:_sftbuf.obj
 0002:00001370       __nstream                  10014370     libucrt:_file.obj
 0002:00001374       ___piob                    10014374     libucrt:_file.obj
 0002:00001378       ___acrt_locale_changed_data 10014378     libucrt:wsetlocale.obj
 0002:0000137c       ___acrt_lconv_static_null  1001437c     libucrt:localeconv.obj
 0002:00001380       ___acrt_lconv_static_W_null 10014380     libucrt:localeconv.obj
 0002:00001388       ___fastflag                10014388     libucrt:fp_flags.obj
 0002:00001390       ___scrt_ucrt_dll_is_in_use 10014390     <common>
 0002:00001394       ___dyn_tls_init_callback   10014394     <common>
 0002:00001398       __pDestructExceptionObject 10014398     <common>
 0002:0000139c       __pmatherr                 1001439c     <common>
 0002:000013a0       ___use_sse2_mathfcns       100143a0     <common>
 0003:00000000       __imp__lstrlenW@4          10015000     kernel32:KERNEL32.dll
 0003:00000004       __imp__SetLastError@4      10015004     kernel32:KERNEL32.dll
 0003:00000008       __imp__GetModuleHandleW@4  10015008     kernel32:KERNEL32.dll
 0003:0000000c       __imp__GetProcAddress@8    1001500c     kernel32:KERNEL32.dll
 0003:00000010       __imp__QueryPerformanceCounter@4 10015010     kernel32:KERNEL32.dll
 0003:00000014       __imp__GetCurrentProcessId@0 10015014     kernel32:KERNEL32.dll
 0003:00000018       __imp__GetCurrentThreadId@0 10015018     kernel32:KERNEL32.dll
 0003:0000001c       __imp__GetSystemTimeAsFileTime@4 1001501c     kernel32:KERNEL32.dll
 0003:00000020       __imp__IsDebuggerPresent@0 10015020     kernel32:KERNEL32.dll
 0003:00000024       __imp__UnhandledExceptionFilter@4 10015024     kernel32:KERNEL32.dll
 0003:00000028       __imp__SetUnhandledExceptionFilter@4 10015028     kernel32:KERNEL32.dll
 0003:0000002c       __imp__GetStartupInfoW@4   1001502c     kernel32:KERNEL32.dll
 0003:00000030       __imp__IsProcessorFeaturePresent@4 10015030     kernel32:KERNEL32.dll
 0003:00000034       __imp__GetCurrentProcess@0 10015034     kernel32:KERNEL32.dll
 0003:00000038       __imp__TerminateProcess@8  10015038     kernel32:KERNEL32.dll
 0003:0000003c       __imp__RaiseException@16   1001503c     kernel32:KERNEL32.dll
 0003:00000040       __imp__RtlUnwind@16        10015040     kernel32:KERNEL32.dll
 0003:00000044       __imp__GetLastError@0      10015044     kernel32:KERNEL32.dll
 0003:00000048       __imp__EnterCriticalSection@4 10015048     kernel32:KERNEL32.dll
 0003:0000004c       __imp__LeaveCriticalSection@4 1001504c     kernel32:KERNEL32.dll
 0003:00000050       __imp__DeleteCriticalSection@4 10015050     kernel32:KERNEL32.dll
 0003:00000054       __imp__InitializeCriticalSectionAndSpinCount@8 10015054     kernel32:KERNEL32.dll
 0003:00000058       __imp__TlsAlloc@0          10015058     kernel32:KERNEL32.dll
 0003:0000005c       __imp__TlsGetValue@4       1001505c     kernel32:KERNEL32.dll
 0003:00000060       __imp__TlsSetValue@8       10015060     kernel32:KERNEL32.dll
 0003:00000064       __imp__TlsFree@4           10015064     kernel32:KERNEL32.dll
 0003:00000068       __imp__FreeLibrary@4       10015068     kernel32:KERNEL32.dll
 0003:0000006c       __imp__LoadLibraryExW@12   1001506c     kernel32:KERNEL32.dll
 0003:00000070       __imp__ExitProcess@4       10015070     kernel32:KERNEL32.dll
 0003:00000074       __imp__GetModuleFileNameA@12 10015074     kernel32:KERNEL32.dll
 0003:00000078       __imp__MultiByteToWideChar@24 10015078     kernel32:KERNEL32.dll
 0003:0000007c       __imp__WideCharToMultiByte@32 1001507c     kernel32:KERNEL32.dll
 0003:00000080       __imp__HeapFree@12         10015080     kernel32:KERNEL32.dll
 0003:00000084       __imp__HeapAlloc@12        10015084     kernel32:KERNEL32.dll
 0003:00000088       __imp__HeapReAlloc@16      10015088     kernel32:KERNEL32.dll
 0003:0000008c       __imp__LCMapStringW@24     1001508c     kernel32:KERNEL32.dll
 0003:00000090       __imp__FindClose@4         10015090     kernel32:KERNEL32.dll
 0003:00000094       __imp__FindFirstFileExA@24 10015094     kernel32:KERNEL32.dll
 0003:00000098       __imp__FindNextFileA@8     10015098     kernel32:KERNEL32.dll
 0003:0000009c       __imp__IsValidCodePage@4   1001509c     kernel32:KERNEL32.dll
 0003:000000a0       __imp__GetACP@0            100150a0     kernel32:KERNEL32.dll
 0003:000000a4       __imp__GetOEMCP@0          100150a4     kernel32:KERNEL32.dll
 0003:000000a8       __imp__GetCPInfo@8         100150a8     kernel32:KERNEL32.dll
 0003:000000ac       __imp__GetCommandLineA@0   100150ac     kernel32:KERNEL32.dll
 0003:000000b0       __imp__GetCommandLineW@0   100150b0     kernel32:KERNEL32.dll
 0003:000000b4       __imp__GetEnvironmentStringsW@0 100150b4     kernel32:KERNEL32.dll
 0003:000000b8       __imp__FreeEnvironmentStringsW@4 100150b8     kernel32:KERNEL32.dll
 0003:000000bc       __imp__GetProcessHeap@0    100150bc     kernel32:KERNEL32.dll
 0003:000000c0       __imp__GetStdHandle@4      100150c0     kernel32:KERNEL32.dll
 0003:000000c4       __imp__GetFileType@4       100150c4     kernel32:KERNEL32.dll
 0003:000000c8       __imp__GetStringTypeW@16   100150c8     kernel32:KERNEL32.dll
 0003:000000cc       __imp__HeapSize@12         100150cc     kernel32:KERNEL32.dll
 0003:000000d0       __imp__SetStdHandle@8      100150d0     kernel32:KERNEL32.dll
 0003:000000d4       __imp__WriteFile@20        100150d4     kernel32:KERNEL32.dll
 0003:000000d8       __imp__FlushFileBuffers@4  100150d8     kernel32:KERNEL32.dll
 0003:000000dc       __imp__GetConsoleCP@0      100150dc     kernel32:KERNEL32.dll
 0003:000000e0       __imp__GetConsoleMode@8    100150e0     kernel32:KERNEL32.dll
 0003:000000e4       __imp__SetFilePointerEx@20 100150e4     kernel32:KERNEL32.dll
 0003:000000e8       __imp__CloseHandle@4       100150e8     kernel32:KERNEL32.dll
 0003:000000ec       __imp__WriteConsoleW@20    100150ec     kernel32:KERNEL32.dll
 0003:000000f0       __imp__CreateFileW@28      100150f0     kernel32:KERNEL32.dll
 0003:000000f4       \177KERNEL32_NULL_THUNK_DATA 100150f4     kernel32:KERNEL32.dll
 0003:000000f8       __IMPORT_DESCRIPTOR_KERNEL32 100150f8     kernel32:KERNEL32.dll
 0003:0000010c       __NULL_IMPORT_DESCRIPTOR   1001510c     kernel32:KERNEL32.dll

 entry point at        0001:00007668

 Static symbols

 0001:000001e8       ?kernel32@@3QB_WB          100011e8     vc_crt_fix_impl.obj
 0001:00000340       _GS_ExceptionPointers      10001340     LIBCMT:gs_report.obj
 0001:00000348       ?ExceptionTemplate@?1??_CxxThrowException@@9@8@4UEHExceptionRecord@@B 10001348     libvcruntime:throw.obj
 0001:00000368       ?module_names@?A0xe4141595@@3QBQB_WB 10001368     libvcruntime:winapi_downlevel.obj
 0001:00000418       ?candidate_modules@?1??try_get_FlsAlloc@@YAP6GKP6GXPAX@Z@ZXZ@4QBW4module_id@?A0xe4141595@@B 10001418     libvcruntime:winapi_downlevel.obj
 0001:0000042c       ?candidate_modules@?1??try_get_FlsFree@@YAP6GHK@ZXZ@4QBW4module_id@?A0xe4141595@@B 1000142c     libvcruntime:winapi_downlevel.obj
 0001:0000043c       ?candidate_modules@?1??try_get_FlsGetValue@@YAP6GPAXK@ZXZ@4QBW4module_id@?A0xe4141595@@B 1000143c     libvcruntime:winapi_downlevel.obj
 0001:00000450       ?candidate_modules@?1??try_get_FlsSetValue@@YAP6GHKPAX@ZXZ@4QBW4module_id@?A0xe4141595@@B 10001450     libvcruntime:winapi_downlevel.obj
 0001:00000464       ?candidate_modules@?1??try_get_InitializeCriticalSectionEx@@YAP6GHPAU_RTL_CRITICAL_SECTION@@KK@ZXZ@4QBW4module_id@?A0xe4141595@@B 10001464     libvcruntime:winapi_downlevel.obj
 0001:00000488       ?tokenTable@@3QBQBDB       10001488     libvcruntime:undname.obj
 0001:000004c0       ?nameTable@@3QBQBDB        100014c0     libvcruntime:undname.obj
 0001:00000604       ?rttiTable@@3QBQBDB        10001604     libvcruntime:undname.obj
 0001:00000cb0       ___acrt_initializers       10001cb0     libucrt:initialization.obj
 0001:00000d28       _module_names              10001d28     libucrt:winapi_thunks.obj
 0001:000011c8       ?candidate_modules@?1??try_get_FlsAlloc@@YAP6GKP6GXPAX@Z@ZXZ@4QBW4module_id@?A0x352e5c4b@@B 100021c8     libucrt:winapi_thunks.obj
 0001:000011d0       ?candidate_modules@?1??try_get_FlsFree@@YAP6GHK@ZXZ@4QBW4module_id@?A0x352e5c4b@@B 100021d0     libucrt:winapi_thunks.obj
 0001:000011d8       ?candidate_modules@?1??try_get_FlsGetValue@@YAP6GPAXK@ZXZ@4QBW4module_id@?A0x352e5c4b@@B 100021d8     libucrt:winapi_thunks.obj
 0001:000011e0       ?candidate_modules@?1??try_get_FlsSetValue@@YAP6GHKPAX@ZXZ@4QBW4module_id@?A0x352e5c4b@@B 100021e0     libucrt:winapi_thunks.obj
 0001:000011e8       ?candidate_modules@?1??try_get_GetCurrentPackageId@@YAP6GJPAIPAE@ZXZ@4QBW4module_id@?A0x352e5c4b@@B 100021e8     libucrt:winapi_thunks.obj
 0001:00001204       ?candidate_modules@?1??try_get_InitializeCriticalSectionEx@@YAP6GHPAU_RTL_CRITICAL_SECTION@@KK@ZXZ@4QBW4module_id@?A0x352e5c4b@@B 10002204     libucrt:winapi_thunks.obj
 0001:0000120c       ?candidate_modules@?1??try_get_LCMapStringEx@@YAP6GHPB_WK0HPA_WHPAU_nlsversioninfo@@PAXJ@ZXZ@4QBW4module_id@?A0x352e5c4b@@B 1000220c     libucrt:winapi_thunks.obj
 0001:00001224       ?candidate_modules@?1??try_get_LocaleNameToLCID@@YAP6GKPB_WK@ZXZ@4QBW4module_id@?A0x352e5c4b@@B 10002224     libucrt:winapi_thunks.obj
 0001:00001240       _errtable                  10002240     libucrt:errno.obj
 0001:000013a8       __mb_locale_names          100023a8     libucrt:mbctype.obj
 0001:00001eb0       _LcidToLocaleNameTable     10002eb0     libucrt:lcidtoname_downlevel.obj
 0001:00002fd8       _LocaleNameToIndexTable    10003fd8     libucrt:lcidtoname_downlevel.obj
 0001:00003f30       LOG_name                   10004f30     libucrt:log10.obj
 0001:00003f40       _One                       10004f40     libucrt:ceil_pentium4.obj
 0001:00003f50       _Bns                       10004f50     libucrt:ceil_pentium4.obj
 0001:00003f60       _Zero                      10004f60     libucrt:ceil_pentium4.obj
 0001:00003f70       _S                         10004f70     libucrt:ceil_pentium4.obj
 0001:00003f80       _NegZero                   10004f80     libucrt:ceil_pentium4.obj
 0001:00003f90       emask                      10004f90     libucrt:log10_pentium4.obj
 0001:00003fa0       CC                         10004fa0     libucrt:log10_pentium4.obj
 0001:00003fb0       Magic                      10004fb0     libucrt:log10_pentium4.obj
 0001:00003fc0       hi_mask                    10004fc0     libucrt:log10_pentium4.obj
 0001:00003fd0       LOG10_2                    10004fd0     libucrt:log10_pentium4.obj
 0001:00003fe0       place_L                    10004fe0     libucrt:log10_pentium4.obj
 0001:00004000       One                        10005000     libucrt:log10_pentium4.obj
 0001:00004010       Zero                       10005010     libucrt:log10_pentium4.obj
 0001:00004020       Two52                      10005020     libucrt:log10_pentium4.obj
 0001:00004030       Infs                       10005030     libucrt:log10_pentium4.obj
 0001:00004040       NaN                        10005040     libucrt:log10_pentium4.obj
 0001:00004050       coeff                      10005050     libucrt:log10_pentium4.obj
 0001:000040ae       _log2max                   100050ae     libucrt:87tran.obj
 0001:000040b8       _smallarg                  100050b8     libucrt:87tran.obj
 0001:000040c2       _half                      100050c2     libucrt:87tran.obj
 0001:0000410e       One                        1000510e     libucrt:87disp.obj
 0001:00004116       Three                      10005116     libucrt:87disp.obj
 0001:0000411e       XAMtoTagTab                1000511e     libucrt:87disp.obj
 0001:00004130       One                        10005130     libucrt:common.obj
 0001:00004144       DblMax                     10005144     libucrt:common.obj
 0001:0000414c       DblMin                     1000514c     libucrt:common.obj
 0001:00004154       IeeeAdjO                   10005154     libucrt:common.obj
 0001:0000415c       IeeeAdjU                   1000515c     libucrt:common.obj
 0001:00004164       _infinity                  10005164     libucrt:common.obj
 0001:0000416c       _zero                      1000516c     libucrt:common.obj
 0001:000041b8       _over                      100051b8     libucrt:fpctrl.obj
 0001:000041c4       _under                     100051c4     libucrt:fpctrl.obj
 0001:00004a88       ?_names@?1??_get_fname@@9@9 10005a88     libucrt:fpexcept.obj
 0001:00005020       $$000000                   10006020     chkstk.obj
 0001:0000557c       $LN28                      1000657c     Align.obj
 0001:0000558c       $LN26                      1000658c     Align.obj
 0001:00005a04       $LN12                      10006a04     Align.obj
 0001:00005a14       $LN10                      10006a14     Align.obj
 0001:00005a20       ?JustifyBlock@@YAXH@Z      10006a20 f   Align.obj
 0001:00005cc0       ?JustifyString@@YA_NHAAUEditorSetString@@@Z 10006cc0 f   Align.obj
 0001:00005eec       $LN24                      10006eec     Align.obj
 0001:00005efc       $LN22                      10006efc     Align.obj
 0001:00005ff0       ?ReformatBlock@@YAXHHH@Z   10006ff0 f   Align.obj
 0001:00006fe0       ?DecodePointer@implementation@?1??DecodePointerWrapper@@YGPAXPAX@Z@SGPAX0@Z 10007fe0 f   vc_crt_fix_impl.obj
 0001:00006fe0       ?EncodePointer@implementation@?1??EncodePointerWrapper@@YGPAXPAX@Z@SGPAX0@Z 10007fe0 f   vc_crt_fix_impl.obj
 0001:00006ff0       ?GetModuleHandleExW@implementation@?1??GetModuleHandleExWWrapper@@YGHKPB_WPAPAUHINSTANCE__@@@Z@SGHK01@Z 10007ff0 f   vc_crt_fix_impl.obj
 0001:00007020       ?InitializeSListHead@implementation@?1??InitializeSListHeadWrapper@@YGXPAT_SLIST_HEADER@@@Z@SGX0@Z 10008020 f   vc_crt_fix_impl.obj
 0001:00007030       ?InterlockedPushEntrySList@implementation@?1??InterlockedPushEntrySListWrapper@@YGPAU_SINGLE_LIST_ENTRY@@PAT_SLIST_HEADER@@PAU3@@Z@SGPAU3@01@Z 10008030 f   vc_crt_fix_impl.obj
 0001:00007040       ?InterlockedPushListSListEx@implementation@?1??InterlockedPushListSListExWrapper@@YGPAU_SINGLE_LIST_ENTRY@@PAT_SLIST_HEADER@@PAU3@1K@Z@SGPAU3@011K@Z 10008040 f   vc_crt_fix_impl.obj
 0001:00007050       ?InterlockedPopEntrySList@implementation@?1??InterlockedPopEntrySListWrapper@@YGPAU_SINGLE_LIST_ENTRY@@PAT_SLIST_HEADER@@@Z@SGPAU3@0@Z 10008050 f   vc_crt_fix_impl.obj
 0001:00007050       ?InterlockedFlushSList@implementation@?1??InterlockedFlushSListWrapper@@YGPAU_SINGLE_LIST_ENTRY@@PAT_SLIST_HEADER@@@Z@SGPAU3@0@Z 10008050 f   vc_crt_fix_impl.obj
 0001:00007050       ?RtlFirstEntrySList@implementation@?1??RtlFirstEntrySListWrapper@@YGPAU_SINGLE_LIST_ENTRY@@PAT_SLIST_HEADER@@@Z@SGPAU3@0@Z 10008050 f   vc_crt_fix_impl.obj
 0001:00007050       ?QueryDepthSList@implementation@?1??QueryDepthSListWrapper@@YGGPAT_SLIST_HEADER@@@Z@SGG0@Z 10008050 f   vc_crt_fix_impl.obj
 0001:00007340       ?dllmain_crt_dispatch@@YGHQAUHINSTANCE__@@KQAX@Z 10008340 f   LIBCMT:dll_dllmain.obj
 0001:00007393       ?dllmain_crt_process_attach@@YAHQAUHINSTANCE__@@QAX@Z 10008393 f   LIBCMT:dll_dllmain.obj
 0001:000074a5       ?dllmain_crt_process_detach@@YAH_N@Z 100084a5 f   LIBCMT:dll_dllmain.obj
 0001:00007522       ?dllmain_dispatch@@YAHQAUHINSTANCE__@@KQAX@Z 10008522 f   LIBCMT:dll_dllmain.obj
 0001:0000763e       ?dllmain_raw@@YGHQAUHINSTANCE__@@KQAX@Z 1000863e f   LIBCMT:dll_dllmain.obj
 0001:000077c4       ?find_pe_section@@YAPAU_IMAGE_SECTION_HEADER@@QAEI@Z 100087c4 f   LIBCMT:utility.obj
 0001:00007d60       $$000000                   10008d60     LIBCMT:_sehprolg4_.obj
 0001:000080d0       $$000000                   100090d0     libvcruntime:memmove.obj
 0001:00008334       TrailingUpVec              10009334     libvcruntime:memmove.obj
 0001:000083e0       TrailingDownVec            100093e0     libvcruntime:memmove.obj
 0001:00008650       $$000000                   10009650     libvcruntime:memcpy.obj
 0001:000088b4       TrailingUpVec              100098b4     libvcruntime:memcpy.obj
 0001:00008960       TrailingDownVec            10009960     libvcruntime:memcpy.obj
 0001:00008bd0       $$000000                   10009bd0     libvcruntime:memset.obj
 0001:00008d30       _ValidateLocalCookies      10009d30 f   libvcruntime:_chandler4_.obj
 0001:00009050       $$000000                   1000a050     libvcruntime:_exsup4_.obj
 0001:000090e0       __unwind_handler4          1000a0e0 f   libvcruntime:_exsup4_.obj
 0001:0000934b       ?try_get_function@@YAPAXW4function_id@?A0xe4141595@@QBDQBW4module_id@2@2@Z 1000a34b f   libvcruntime:winapi_downlevel.obj
 0001:000093eb       ?try_get_module@@YAPAUHINSTANCE__@@W4module_id@?A0xe4141595@@@Z 1000a3eb f   libvcruntime:winapi_downlevel.obj
 0001:00009610       $$000000                   1000a610     libvcruntime:_exsup_.obj
 0001:00009630       __unwind_handler           1000a630 f   libvcruntime:_exsup_.obj
 0001:00009a40       ?atexit_exception_filter@@YAHK@Z 1000aa40 f   libucrt:exit.obj
 0001:00009a53       ?common_exit@@YAXHW4_crt_exit_cleanup_mode@@W4_crt_exit_return_mode@@@Z 1000aa53 f   libucrt:exit.obj
 0001:00009b6c       ?exit_or_terminate_process@@YAXI@Z 1000ab6c f   libucrt:exit.obj
 0001:00009bad       ?is_managed_app@@YA_NXZ    1000abad f   libucrt:exit.obj
 0001:00009bf1       ?try_cor_exit_process@@YAXI@Z 1000abf1 f   libucrt:exit.obj
 0001:00009c95       ??$common_configure_argv@D@@YAHW4_crt_argv_mode@@@Z 1000ac95 f   libucrt:argv_parsing.obj
 0001:00009db9       ??$parse_command_line@D@@YAXPADPAPAD0PAI2@Z 1000adb9 f   libucrt:argv_parsing.obj
 0001:00009f8e       ??$common_initialize_environment_nolock@D@@YAHXZ 1000af8e f   libucrt:environment_initialization.obj
 0001:00009fe7       ??$create_environment@D@@YAQAPADQAD@Z 1000afe7 f   libucrt:environment_initialization.obj
 0001:0000a0b8       ??$free_environment@D@@YAXQAPAD@Z 1000b0b8 f   libucrt:environment_initialization.obj
 0001:0000a0b8       ??$free_environment@_W@@YAXQAPA_W@Z 1000b0b8 f   libucrt:environment_initialization.obj
 0001:0000a127       ??$uninitialize_environment_internal@D@@YAXAAPAPAD@Z 1000b127 f   libucrt:environment_initialization.obj
 0001:0000a142       ??$uninitialize_environment_internal@_W@@YAXAAPAPA_W@Z 1000b142 f   libucrt:environment_initialization.obj
 0001:0000a2aa       ??R<lambda_275893d493268fdec8709772e3fcec0e>@@QBEHXZ 1000b2aa f   libucrt:onexit.obj
 0001:0000a3ca       ??R<lambda_4e60a939b0d047cfe11ddc22648dfba9>@@QBEHXZ 1000b3ca f   libucrt:onexit.obj
 0001:0000a59f       _initialize_global_variables 1000b59f f   libucrt:initialization.obj
 0001:0000a5b1       _initialize_c              1000b5b1 f   libucrt:initialization.obj
 0001:0000a5cb       _uninitialize_environment  1000b5cb f   libucrt:initialization.obj
 0001:0000a5d3       _initialize_pointers       1000b5d3 f   libucrt:initialization.obj
 0001:0000a610       _uninitialize_vcruntime    1000b610 f   libucrt:initialization.obj
 0001:0000a619       _uninitialize_allocated_memory 1000b619 f   libucrt:initialization.obj
 0001:0000a690       _uninitialize_global_state_isolation 1000b690 f   libucrt:initialization.obj
 0001:0000a690       _initialize_global_state_isolation 1000b690 f   libucrt:initialization.obj
 0001:0000a690       _initialize_environment    1000b690 f   libucrt:initialization.obj
 0001:0000a690       _uninitialize_c            1000b690 f   libucrt:initialization.obj
 0001:0000a690       _report_memory_leaks       1000b690 f   libucrt:initialization.obj
 0001:0000ac0a       ?construct_ptd@@YAXQAU__acrt_ptd@@QAPAU__crt_locale_data@@@Z 1000bc0a f   libucrt:per_thread_data.obj
 0001:0000ac83       ?destroy_fls@@YGXPAX@Z     1000bc83 f   libucrt:per_thread_data.obj
 0001:0000aca4       ?destroy_ptd@@YAXQAU__acrt_ptd@@@Z 1000bca4 f   libucrt:per_thread_data.obj
 0001:0000ad4d       ?replace_current_thread_locale_nolock@@YAXQAU__acrt_ptd@@QAU__crt_locale_data@@@Z 1000bd4d f   libucrt:per_thread_data.obj
 0001:0000af13       ?try_get_function@@YAPAXW4function_id@?A0x352e5c4b@@QBDQBW4module_id@2@2@Z 1000bf13 f   libucrt:winapi_thunks.obj
 0001:0000afb2       ?try_get_module@@YAPAUHINSTANCE__@@W4module_id@?A0x352e5c4b@@@Z 1000bfb2 f   libucrt:winapi_thunks.obj
 0001:0000b64a       ?<helper_func_cdecl>@<lambda_62bb7ecb46d0a77b591a051c43eb5ad1>@@CAHPBX0@Z 1000c64a f   libucrt:argv_wildcards.obj
 0001:0000b662       ??$common_expand_argv_wildcards@D@@YAHQAPADQAPAPAD@Z 1000c662 f   libucrt:argv_wildcards.obj
 0001:0000b7f2       ??$copy_and_add_argument_to_buffer@D@@YAHQBD0IAAV?$argument_list@D@?A0xb0e4b824@@@Z 1000c7f2 f   libucrt:argv_wildcards.obj
 0001:0000b888       ??$expand_argument_wildcards@D@@YAHQAD0AAV?$argument_list@D@?A0xb0e4b824@@@Z 1000c888 f   libucrt:argv_wildcards.obj
 0001:0000bb63       ??R<lambda_ad1ced32f4ac17aa236e5ef05d6b3b7c>@@QBEXXZ 1000cb63 f   libucrt:mbctype.obj
 0001:0000bc27       ?CPtoLocaleName@@YAPB_WH@Z 1000cc27 f   libucrt:mbctype.obj
 0001:0000bc65       ?getSystemCP@@YAHH@Z       1000cc65 f   libucrt:mbctype.obj
 0001:0000bcd8       ?setSBCS@@YAXPAU__crt_multibyte_data@@@Z 1000ccd8 f   libucrt:mbctype.obj
 0001:0000bd3d       ?setSBUpLow@@YAXPAU__crt_multibyte_data@@@Z 1000cd3d f   libucrt:mbctype.obj
 0001:0000bed1       ?setmbcp_internal@@YAHH_N@Z 1000ced1 f   libucrt:mbctype.obj
 0001:0000c283       _memcpy_s                  1000d283 f   libucrt:mbctype.obj
 0001:0000c304       ?x_ismbbtype_l@@YAHPAU__crt_locale_pointers@@IHH@Z 1000d304 f   libucrt:ismbbyte.obj
 0001:0000c38e       ?find_end_of_double_null_terminated_sequence@@YAPB_WQB_W@Z 1000d38e f   libucrt:get_environment_from_os.obj
 0001:0000c4db       ?initialize_inherited_file_handles_nolock@@YAXXZ 1000d4db f   libucrt:ioinit.obj
 0001:0000c591       ?initialize_stdio_handles_nolock@@YAXXZ 1000d591 f   libucrt:ioinit.obj
 0001:0000c81b       ?get_global_action_nolock@@YAPAP6AXH@ZH@Z 1000d81b f   libucrt:signal.obj
 0001:0000c88e       ?siglookup@@YAPAU__crt_signal_action_t@@HQAU1@@Z 1000d88e f   libucrt:signal.obj
 0001:0000d279       ?GetTableIndexFromLocaleName@@YAHPB_W@Z 1000e279 f   libucrt:lcidtoname_downlevel.obj
 0001:0000d370       ?shortsort@@YAXPAD0IP6AHPBX1@Z@Z 1000e370 f   libucrt:qsort.obj
 0001:0000d410       ?swap@@YAXPAD0I@Z          1000e410 f   libucrt:qsort.obj
 0001:0000d7ea       ??$common_tcsncpy_s@D@@YAHQADIQBDI@Z 1000e7ea f   libucrt:strncpy_s.obj
 0001:0000d8b0       $$000000                   1000e8b0     libucrt:strpbrk.obj
 0001:0000d994       ?initialize_multibyte@@YAHXZ 1000e994 f   libucrt:multibyte_initializer.obj
 0001:0000dae0       ?__acrt_LCMapStringA_stat@@YAHPAU__crt_locale_pointers@@PB_WKPBDHPADHHH@Z 1000eae0 f   libucrt:lcmapstringa.obj
 0001:0000e10f       _common_flush_all          1000f10f f   libucrt:fflush.obj
 0001:0000e465       ?free_crt_array_internal@@YAXQAPBXI@Z 1000f465 f   libucrt:inittime.obj
 0001:0000e6d6       ?write_double_translated_ansi_nolock@@YA?AUwrite_result@?A0x47fa6670@@HQBDI@Z 1000f6d6 f   libucrt:write.obj
 0001:0000e889       ?write_double_translated_unicode_nolock@@YA?AUwrite_result@?A0x47fa6670@@QBDI@Z 1000f889 f   libucrt:write.obj
 0001:0000e8f6       ?write_requires_double_translation_nolock@@YA_NH@Z 1000f8f6 f   libucrt:write.obj
 0001:0000e96c       ?write_text_ansi_nolock@@YA?AUwrite_result@?A0x47fa6670@@HQBDI@Z 1000f96c f   libucrt:write.obj
 0001:0000ea4b       ?write_text_utf16le_nolock@@YA?AUwrite_result@?A0x47fa6670@@HQBDI@Z 1000fa4b f   libucrt:write.obj
 0001:0000eb39       ?write_text_utf8_nolock@@YA?AUwrite_result@?A0x47fa6670@@HQBDI@Z 1000fb39 f   libucrt:write.obj
 0001:0000ef60       $$000000                   1000ff60     libucrt:log10.obj
 0001:0000f0b0       $$000000                   100100b0     libucrt:ceil_pentium4.obj
 0001:0000f1cd       ??$common_lseek_nolock@_J@@YA_JH_JH@Z 100101cd f   libucrt:lseek.obj
 0001:0000f360       $$000000                   10010360     libucrt:_strnicm.obj
 0001:0000f420       $$000000                   10010420     libucrt:log10_pentium4.obj
 0001:0000f6b0       $$000000                   100106b0     libucrt:87tran.obj
 0001:0000f8b0       $$000000                   100108b0     libucrt:87disp.obj
 0001:0000fab0       $$000000                   10010ab0     libucrt:common.obj
 0001:0000fc40       $$000000                   10010c40     libucrt:genexcep.obj
 0001:00010f30       $$000000                   10011f30     LIBCMT:ulldvrm.obj
 0001:00010fd0       $$000000                   10011fd0     LIBCMT:_sehprolg4gs_.obj
 0001:00011030       $$000000                   10012030     LIBCMT:llmul.obj
 0001:00011070       $$000000                   10012070     LIBCMT:lldvrm.obj
 0001:00011150       $$000000                   10012150     LIBCMT:ullshr.obj
 0001:00011170       $$000000                   10012170     LIBCMT:alloca16.obj
 0001:000111a0       $$000000                   100121a0     LIBCMT:llshl.obj
 0001:000111c0       $$000000                   100121c0     LIBCMT:_ftol2_.obj
 0001:00011280       $$000000                   10012280     libvcruntime:strchr.obj
 0001:000113b0       $$000000                   100123b0     libvcruntime:strrchr.obj
 0001:000114e8       __sehtable$?dllmain_crt_process_attach@@YAHQAUHINSTANCE__@@QAX@Z 100124e8     LIBCMT:dll_dllmain.obj
 0001:00011508       __sehtable$?dllmain_crt_process_detach@@YAH_N@Z 10012508     LIBCMT:dll_dllmain.obj
 0001:00011528       __sehtable$?dllmain_dispatch@@YAHQAUHINSTANCE__@@KQAX@Z 10012528     LIBCMT:dll_dllmain.obj
 0001:000115d8       __sehtable$___scrt_is_nonwritable_in_current_image 100125d8     LIBCMT:utility.obj
 0001:000115f8       __sehtable$__query_new_handler 100125f8     libucrt:new_handler.obj
 0001:00011618       __sehtable$?common_exit@@YAXHW4_crt_exit_cleanup_mode@@W4_crt_exit_return_mode@@@Z 10012618     libucrt:exit.obj
 0001:00011640       __sehtable$??$?RV<lambda_800076c951b434888f4765a74a194fcc>@@AAV<lambda_4e60a939b0d047cfe11ddc22648dfba9>@@V<lambda_6dbb1268764f43b569ce7b67e331d33a>@@@?$__crt_seh_guarded_call@H@@QAEH$$QAV<lambda_800076c951b434888f4765a74a194fcc>@@AAV<lambda_4e60a939b0d047cfe11ddc22648dfba9>@@$$QAV<lambda_6dbb1268764f43b569ce7b67e331d33a>@@@Z 10012640     libucrt:onexit.obj
 0001:00011660       __sehtable$??$?RV<lambda_995298e7d72eb4c2aab26c0585b3abe5>@@AAV<lambda_275893d493268fdec8709772e3fcec0e>@@V<lambda_293819299cbf9a7022e18b56a874bb5c>@@@?$__crt_seh_guarded_call@H@@QAEH$$QAV<lambda_995298e7d72eb4c2aab26c0585b3abe5>@@AAV<lambda_275893d493268fdec8709772e3fcec0e>@@$$QAV<lambda_293819299cbf9a7022e18b56a874bb5c>@@@Z 10012660     libucrt:onexit.obj
 0001:00011680       __sehtable$_terminate      10012680     libucrt:terminate.obj
 0001:000116a0       __sehtable$??$?RV<lambda_9df27f884b057bc3edfc946cb5b7cf47>@@AAV<lambda_e69574bed617af4e071282c136b37893>@@V<lambda_cc0d902bcbbeb830f749456577db4721>@@@?$__crt_seh_guarded_call@X@@QAEX$$QAV<lambda_9df27f884b057bc3edfc946cb5b7cf47>@@AAV<lambda_e69574bed617af4e071282c136b37893>@@$$QAV<lambda_cc0d902bcbbeb830f749456577db4721>@@@Z 100126a0     libucrt:per_thread_data.obj
 0001:000116c0       __sehtable$??$?RV<lambda_3518db117f0e7cdb002338c5d3c47b6c>@@AAV<lambda_b2ea41f6bbb362cd97d94c6828d90b61>@@V<lambda_abdedf541bb04549bc734292b4a045d4>@@@?$__crt_seh_guarded_call@X@@QAEX$$QAV<lambda_3518db117f0e7cdb002338c5d3c47b6c>@@AAV<lambda_b2ea41f6bbb362cd97d94c6828d90b61>@@$$QAV<lambda_abdedf541bb04549bc734292b4a045d4>@@@Z 100126c0     libucrt:per_thread_data.obj
 0001:000116e0       __sehtable$??$?RV<lambda_51b6e8b1eb166f2a3faf91f424b38130>@@AAV<lambda_6250bd4b2a391816dd638c3bf72b0bcb>@@V<lambda_0b5a4a3e68152e1d9b943535f5f47bed>@@@?$__crt_seh_guarded_call@X@@QAEX$$QAV<lambda_51b6e8b1eb166f2a3faf91f424b38130>@@AAV<lambda_6250bd4b2a391816dd638c3bf72b0bcb>@@$$QAV<lambda_0b5a4a3e68152e1d9b943535f5f47bed>@@@Z 100126e0     libucrt:per_thread_data.obj
 0001:00011700       __sehtable$??$?RV<lambda_5b71d36f03204c0beab531769a5b5694>@@AAV<lambda_be2b3da3f62db62e9dad5dc70221a656>@@V<lambda_8f9ce462984622f9bf76b59e2aaaf805>@@@?$__crt_seh_guarded_call@X@@QAEX$$QAV<lambda_5b71d36f03204c0beab531769a5b5694>@@AAV<lambda_be2b3da3f62db62e9dad5dc70221a656>@@$$QAV<lambda_8f9ce462984622f9bf76b59e2aaaf805>@@@Z 10012700     libucrt:per_thread_data.obj
 0001:00011720       __sehtable$___acrt_update_thread_multibyte_data 10012720     libucrt:mbctype.obj
 0001:00011740       __sehtable$??$?RV<lambda_978dc153c237d78434369da87b74ff60>@@AAV<lambda_ad1ced32f4ac17aa236e5ef05d6b3b7c>@@V<lambda_4a8533e2866a575feecb8298ce776b0d>@@@?$__crt_seh_guarded_call@X@@QAEX$$QAV<lambda_978dc153c237d78434369da87b74ff60>@@AAV<lambda_ad1ced32f4ac17aa236e5ef05d6b3b7c>@@$$QAV<lambda_4a8533e2866a575feecb8298ce776b0d>@@@Z 10012740     libucrt:mbctype.obj
 0001:00011760       __sehtable$___acrt_initialize_lowio 10012760     libucrt:ioinit.obj
 0001:00011780       __sehtable$_raise          10012780     libucrt:signal.obj
 0001:000117a0       __sehtable$??$?RV<lambda_a048d3beccc847880fc8490e18b82769>@@AAV<lambda_ec61778202f4f5fc7e7711acc23c3bca>@@V<lambda_f7496a158712204296dd6628a163878e>@@@?$__crt_seh_guarded_call@P6AXH@Z@@QAEP6AXH@Z$$QAV<lambda_a048d3beccc847880fc8490e18b82769>@@AAV<lambda_ec61778202f4f5fc7e7711acc23c3bca>@@$$QAV<lambda_f7496a158712204296dd6628a163878e>@@@Z 100127a0     libucrt:signal.obj
 0001:000117c0       __sehtable$___acrt_uninitialize_locale 100127c0     libucrt:wsetlocale.obj
 0001:000117e0       __sehtable$___acrt_update_thread_locale_data 100127e0     libucrt:locale_refcounting.obj
 0001:00011800       __sehtable$___acrt_lowio_ensure_fh_exists 10012800     libucrt:osfinfo.obj
 0001:00011820       __sehtable$_common_flush_all 10012820     libucrt:fflush.obj
 0001:00011848       __sehtable$__fcloseall     10012848     libucrt:closeall.obj
 0001:00011868       __sehtable$??$?RV<lambda_61cee617f5178ae960314fd4d05640a0>@@AAV<lambda_6978c1fb23f02e42e1d9e99668cc68aa>@@V<lambda_9cd88cf8ad10232537feb2133f08c833>@@@?$__crt_seh_guarded_call@H@@QAEH$$QAV<lambda_61cee617f5178ae960314fd4d05640a0>@@AAV<lambda_6978c1fb23f02e42e1d9e99668cc68aa>@@$$QAV<lambda_9cd88cf8ad10232537feb2133f08c833>@@@Z 10012868     libucrt:commit.obj
 0001:00011888       __sehtable$__write         10012888     libucrt:write.obj
 0001:000118a8       __sehtable$_fclose         100128a8     libucrt:fclose.obj
 0001:000118c8       __sehtable$??$?RV<lambda_123407a5e2ac06da108355a851863b7a>@@AAV<lambda_2fe9b910cf3cbf4a0ab98a02ba45b3ec>@@V<lambda_ae55bdf541ad94d75914d381c370e64d>@@@?$__crt_seh_guarded_call@H@@QAEH$$QAV<lambda_123407a5e2ac06da108355a851863b7a>@@AAV<lambda_2fe9b910cf3cbf4a0ab98a02ba45b3ec>@@$$QAV<lambda_ae55bdf541ad94d75914d381c370e64d>@@@Z 100128c8     libucrt:close.obj
 0001:000118e8       __sehtable$__IsNonwritableInCurrentImage 100128e8     LIBCMT:pesect.obj
 0001:00011910       .edata                     10012910     Align.exp
 0001:00011938       rgpv                       10012938     Align.exp
 0001:00011948       rgszName                   10012948     Align.exp
 0001:00011958       rgwOrd                     10012958     Align.exp
 0001:00011960       szName                     10012960     Align.exp
 0001:0001196a       $N00001                    1001296a     Align.exp
 0001:00011979       $N00002                    10012979     Align.exp
 0001:00011988       $N00003                    10012988     Align.exp
 0001:0001198e       $N00004                    1001298e     Align.exp
 0002:00000020       ?__vcrt_flsindex@@3KA      10013020     libvcruntime:per_thread_data.obj
 0002:00000044       ___acrt_flsindex           10013044     libucrt:per_thread_data.obj
 0002:00000048       _errno_no_memory           10013048     libucrt:errno.obj
 0002:0000004c       _doserrno_no_memory        1001304c     libucrt:errno.obj
 0002:00000050       ___rgctypeflag             10013050     libucrt:mbctype.obj
 0002:00000058       ___rgcode_page_info        10013058     libucrt:mbctype.obj
 0002:000007e8       ?Info@@3UPluginStartupInfo@@A 100137e8     Align.obj
 0002:00000870       ?FSF@@3UFarStandardFunctions@@A 10013870     Align.obj
 0002:00000930       ?PluginMenuStrings@?1??GetPluginInfoW@@9@4@4PAPB_WA 10013930     Align.obj
 0002:00000934       ?Function@?1??EncodePointerWrapper@@9@4@4Q6GPAXPAX@ZA 10013934     vc_crt_fix_impl.obj
 0002:00000938       ?$S1@?1??EncodePointerWrapper@@9@4@4IA 10013938     vc_crt_fix_impl.obj
 0002:0000093c       ?Function@?1??DecodePointerWrapper@@9@4@4Q6GPAXPAX@ZA 1001393c     vc_crt_fix_impl.obj
 0002:00000940       ?$S2@?1??DecodePointerWrapper@@9@4@4IA 10013940     vc_crt_fix_impl.obj
 0002:00000944       ?Function@?1??GetModuleHandleExWWrapper@@9@12@4Q6GHKPB_WPAPAUHINSTANCE__@@@ZA 10013944     vc_crt_fix_impl.obj
 0002:00000948       ?$S3@?1??GetModuleHandleExWWrapper@@9@12@4IA 10013948     vc_crt_fix_impl.obj
 0002:0000094c       ?Function@?1??InitializeSListHeadWrapper@@9@4@4Q6GXPAT_SLIST_HEADER@@@ZA 1001394c     vc_crt_fix_impl.obj
 0002:00000950       ?$S4@?1??InitializeSListHeadWrapper@@9@4@4IA 10013950     vc_crt_fix_impl.obj
 0002:00000954       ?Function@?1??InterlockedFlushSListWrapper@@9@4@4Q6GPAU_SINGLE_LIST_ENTRY@@PAT_SLIST_HEADER@@@ZA 10013954     vc_crt_fix_impl.obj
 0002:00000958       ?$S5@?1??InterlockedFlushSListWrapper@@9@4@4IA 10013958     vc_crt_fix_impl.obj
 0002:0000095c       ?Function@?1??InterlockedPopEntrySListWrapper@@9@4@4Q6GPAU_SINGLE_LIST_ENTRY@@PAT_SLIST_HEADER@@@ZA 1001395c     vc_crt_fix_impl.obj
 0002:00000960       ?$S6@?1??InterlockedPopEntrySListWrapper@@9@4@4IA 10013960     vc_crt_fix_impl.obj
 0002:00000964       ?Function@?1??InterlockedPushEntrySListWrapper@@9@8@4Q6GPAU_SINGLE_LIST_ENTRY@@PAT_SLIST_HEADER@@PAU2@@ZA 10013964     vc_crt_fix_impl.obj
 0002:00000968       ?$S7@?1??InterlockedPushEntrySListWrapper@@9@8@4IA 10013968     vc_crt_fix_impl.obj
 0002:0000096c       ?Function@?1??InterlockedPushListSListExWrapper@@9@16@4Q6GPAU_SINGLE_LIST_ENTRY@@PAT_SLIST_HEADER@@PAU2@1K@ZA 1001396c     vc_crt_fix_impl.obj
 0002:00000970       ?$S8@?1??InterlockedPushListSListExWrapper@@9@16@4IA 10013970     vc_crt_fix_impl.obj
 0002:00000974       ?Function@?1??RtlFirstEntrySListWrapper@@9@4@4Q6GPAU_SINGLE_LIST_ENTRY@@PAT_SLIST_HEADER@@@ZA 10013974     vc_crt_fix_impl.obj
 0002:00000978       ?$S9@?1??RtlFirstEntrySListWrapper@@9@4@4IA 10013978     vc_crt_fix_impl.obj
 0002:0000097c       ?Function@?1??QueryDepthSListWrapper@@9@4@4Q6GGPAT_SLIST_HEADER@@@ZA 1001397c     vc_crt_fix_impl.obj
 0002:00000980       ?$S10@?1??QueryDepthSListWrapper@@9@4@4IA 10013980     vc_crt_fix_impl.obj
 0002:00000984       ?__proc_attached@@3HA      10013984     LIBCMT:dll_dllmain.obj
 0002:00000990       ?module_local_atexit_table@@3U_onexit_table_t@@A 10013990     LIBCMT:utility.obj
 0002:0000099c       ?module_local_at_quick_exit_table@@3U_onexit_table_t@@A 1001399c     LIBCMT:utility.obj
 0002:000009a8       ?is_initialized_as_dll@@3_NA 100139a8     LIBCMT:utility.obj
 0002:000009d8       _GS_ExceptionRecord        100139d8     LIBCMT:gs_report.obj
 0002:00000a28       _GS_ContextRecord          10013a28     LIBCMT:gs_report.obj
 0002:00000cf4       ?__vcrt_startup_thread_ptd@@3U__vcrt_ptd@@A 10013cf4     libvcruntime:per_thread_data.obj
 0002:00000d1c       ___vcrt_lock_table         10013d1c     libvcruntime:locks.obj
 0002:00000d34       ___vcrt_locks_initialized  10013d34     libvcruntime:locks.obj
 0002:00000d38       ?module_handles@@3PAPAUHINSTANCE__@@A 10013d38     libvcruntime:winapi_downlevel.obj
 0002:00000d48       ?encoded_function_pointers@@3PAPAXA 10013d48     libvcruntime:winapi_downlevel.obj
 0002:00000d98       ?heap@@3V_HeapManager@@A   10013d98     libvcruntime:undname.obj
 0002:00000dac       ___acrt_new_handler        10013dac     libucrt:new_handler.obj
 0002:00000db0       _c_termination_complete    10013db0     libucrt:exit.obj
 0002:00000db4       _thread_local_exit_callback_func 10013db4     libucrt:exit.obj
 0002:00000db8       ?c_exit_complete@?5??common_exit@@YAXHW4_crt_exit_cleanup_mode@@W4_crt_exit_return_mode@@@Z@4_NA 10013db8     libucrt:exit.obj
 0002:00000dc0       ?program_name@?5???$common_configure_argv@D@@YAHW4_crt_argv_mode@@@Z@4PADA 10013dc0     libucrt:argv_parsing.obj
 0002:00000ef0       ___acrt_lock_table         10013ef0     libucrt:locks.obj
 0002:00001028       ___acrt_locks_initialized  10014028     libucrt:locks.obj
 0002:00001030       _module_handles            10014030     libucrt:winapi_thunks.obj
 0002:00001080       _encoded_function_pointers 10014080     libucrt:winapi_thunks.obj
 0002:00001100       ?state_cache@?1??__acrt_is_packaged_app@@9@4JA 10014100     libucrt:winapi_thunks.obj
 0002:00001104       ___acrt_invalid_parameter_handler 10014104     libucrt:invalid_parameter.obj
 0002:00001120       _fSystemSet                10014120     libucrt:mbctype.obj
 0002:00001124       ?initialized@?1??__acrt_initialize_multibyte@@9@4_NA 10014124     libucrt:mbctype.obj
 0002:0000134c       _ctrlc_action              1001434c     libucrt:signal.obj
 0002:00001350       _ctrlbreak_action          10014350     libucrt:signal.obj
 0002:00001354       _abort_action              10014354     libucrt:signal.obj
 0002:00001358       _term_action               10014358     libucrt:signal.obj
 0002:0000135c       _user_matherr              1001435c     libucrt:matherr.obj
 0002:0000136c       ___acrt_global_new_mode    1001436c     libucrt:new_mode.obj
 0002:00001384       ___acrt_app_type           10014384     libucrt:report_runtime_error.obj
 0002:0000138c       __pmatherr_set             1001438c     libucrt:libm_error.obj
 0003:0000025a       .idata$6                   1001525a     kernel32:KERNEL32.dll
 0004:00000000       __guard_fids____dcrt_uninitialize_environments_nolock 10016000     libucrt:environment_initialization.obj
 0004:00000008       __guard_fids__             10016008     libucrt:initialization.obj
 0004:00000068       __guard_fids____acrt_initialize_ptd 10016068     libucrt:per_thread_data.obj
 0004:0000006c       __guard_fids_??$expand_argument_wildcards@D@@YAHQAD0AAV?$argument_list@D@?A0xb0e4b824@@@Z 1001606c     libucrt:argv_wildcards.obj
 0004:00000070       __guard_fids__             10016070     libucrt:multibyte_initializer.obj
 0004:00000074       __guard_fids__             10016074     libucrt:stdio_initializer.obj
 0004:00000078       __guard_fids__             10016078     libucrt:stdio_initializer.obj
 0004:0000007c       __guard_fids__             1001607c     libucrt:locale_initializer.obj
 0004:00000080       __guard_fids____libm_error_support 10016080     libucrt:libm_error.obj
 0004:00000084       __guard_fids__             10016084     libucrt:sse2_initializer.obj
 0004:00000088       __guard_fids__             10016088     libucrt:console_output_initializer.obj
 0004:0000008c       __guard_fids_?dllmain_crt_process_attach@@YAHQAUHINSTANCE__@@QAX@Z 1001608c     LIBCMT:dll_dllmain.obj
 0004:00000094       __guard_fids_?dllmain_dispatch@@YAHQAUHINSTANCE__@@KQAX@Z 10016094     LIBCMT:dll_dllmain.obj
 0004:00000098       __guard_fids__             10016098     LIBCMT:throw_bad_alloc.obj
 0004:000000a0       __guard_fids__             100160a0     LIBCMT:throw_bad_alloc.obj
 0004:000000a8       __guard_fids__             100160a8     LIBCMT:throw_bad_alloc.obj
 0004:000000b0       __guard_fids__             100160b0     LIBCMT:throw_bad_alloc.obj
 0004:000000b4       __guard_fids__             100160b4     LIBCMT:throw_bad_alloc.obj
 0004:000000b8       __guard_fids__             100160b8     LIBCMT:throw_bad_alloc.obj
 0004:000000bc       __guard_fids__             100160bc     LIBCMT:throw_bad_alloc.obj
 0004:000000c0       __guard_fids__             100160c0     LIBCMT:throw_bad_alloc.obj
 0004:000000c4       __guard_fids__             100160c4     LIBCMT:std_type_info_static.obj
 0004:000000c8       __guard_fids__             100160c8     LIBCMT:guard_support.obj
 0004:000000cc       __guard_fids____vcrt_initialize_ptd 100160cc     libvcruntime:per_thread_data.obj
 0005:00000060       $R000000                   10017060     Align.res
